:100000000C9472180C94A3180C94A3180C94A318B5
:100010000C94A3180C94A3180C94A3180C94A31874
:100020000C94A3180C94A3180C94A3180C94A31864
:100030000C94A3180C94A3180C94A3180C94A31854
:100040000C94A3180C9403A10C94A3180C94A3185B
:100050000C94A3180C94A3180C94679C0C94F0F8BF
:100060000C94A3180C94C3520C94B9520C94A3187A
:100070000C94A3180C94A3180C94A3180C94A31814
:100080000C94A3180C94A3180C94A3180C94A31804
:100090000C94A3180C94A3180C94A3180C94A318F4
:1000A0000C94A3180C94A3180C94A3180C94A318E4
:1000B0000C94A3180C94A3180C94A3180C94A318D4
:1000C0000C94A3180C94A3180C94A3180C9419293D
:1000D0000C94E3280C94A3180C94A3180C94A31864
:1000E0000C94A318084AD73B3BCE016E84BCBFFDDD
:1000F000C12F3D6C74319ABD56833DDA3D00C77FF8
:1001000011BED9E4BB4C3E916BAAAABE0000008090
:100110003F05A84CCDB2D44EB93836A9020C50B91F
:10012000918688083CA6AAAA2ABE000000803F004B
:100130000D94D6110C9464F30D946D0B0C9485F210
:100140000C9437F30C94ABF20C9457290C945AF39B
:100150000D94DC080C94AB290C9430530D941D0DB8
:100160000C94A3F20C941DF30C94B7290C94BB29A6
:100170000C94C5FB0D9427050C9487530C945D5388
:100180000C942DF30C9461530C9478F30C947EF240
:100190000C9469830C9464F20D94B8110C94695317
:1001A0000D94170B0C943F530C9495F20D94FE0F85
:1001B0000C946F820D94420B0C9465530C948483C1
:1001C0000C940B850D942B080C94D5290C9495292F
:1001D0000C9441F30D944C0B0C94CA290C945DFFC4
:1001E0000C94FAF20D94E70A0C9455530C94F2F225
:1001F0000C94C3290C948C820C94A7F20D94330BAD
:100200000C946D530C9463370C9441840C949DF2C0
:100210000D94E1030C9467370C9404830C945953A8
:100220000C94B5F20C94DD290C94A4290C94015380
:100230000C94387E0C948CF30C94B3290C9486297E
:100240000C9409F30C94B1F20D94600B0C94E6FC41
:100250000C944E530C9414370C945FF20C948BF264
:100260000C9425830C947AF20C945B390D94490C10
:100270000C949C390C9402840C9414840C946EF3AA
:100280000C94397E0C94CBFD0C9425F30D948B01CA
:100290000C9474530C94D4390C942F390C9482F22E
:1002A0000C9482F30C9499F20D940D000C94F5FDCE
:1002B0000C9476F20D940E0B0C9413F30C948FF2B5
:1002C0000C947F530C94FFF20D945A0C0D94140B64
:1002D0000D945A050C94AF290C94BF290C944BF340
:1002E0000C94B67D4E414E494E495459494E46CD27
:1002F000CCCC3D0AD7233C17B7D13877CC2B3295DD
:1003000095E6241FB14F0A000020410000C84200BA
:10031000401C4620BCBE4CCA1B0E5AAEC59D740084
:10032000407A10F35A00A0724E18090010A5D4E8C4
:100330000000E87648170000E40B54020000CA9A57
:100340003B000000E1F505000080969800000040A9
:10035000420F000000A086010000001027000000EE
:1003600000E803000000006400000000000A000034
:100370000000000100000000002C76D888DC674FE8
:100380000823DFC1DFAE59E1B1B796E5E3E453C618
:100390003AE651997696E8E6C28426EB898C9B6210
:1003A000ED407C6FFCEFBC9C9F40F2BAA56FA5F4BA
:1003B00090055A2AF75C936B6CF9676DC11BFCE0E2
:1003C000E40D47FEF520E6B500D0ED902E03009435
:1003D0003577050080841E080000204E0A000000CA
:1003E000C80C333333330F986E12831141EF8D21D4
:1003F00014893BE65516CFFEE6DB18D1844B381B3B
:10040000F77C1D901DA4BBE424203284725E2281FF
:1004100000C9F124ECA1E53D27434F4D4D554E4910
:10042000434154494F4E0044525952554E00455293
:10043000524F525300494E464F004543484F0045E6
:1004400072726F722077726974696E6720746F20A0
:10045000454550524F4D210A0053544F505045448A
:100460002E20005072696E7465722073746F707004
:1004700065642064756520746F206572726F727395
:100480002E2046697820746865206572726F72202C
:10049000616E6420757365204D39393920746F2081
:1004A000726573746172742E202854656D70657264
:1004B00061747572652069732072657365742E208E
:1004C0005365742069742061667465722072657367
:1004D00074617274696E67290A004E6F2043686503
:1004E000636B73756D2077697468206C696E652025
:1004F0006E756D6265722C204C617374204C696E50
:10050000653A20004E6F20436865636B73756D20FC
:1005100077697468206C696E65206E756D626572AE
:100520002C204C617374204C696E653A200063681E
:1005300065636B73756D206D69736D617463682C91
:10054000204C617374204C696E653A20004C696ED2
:1005500065204E756D626572206973206E6F742020
:100560004C617374204C696E65204E756D626572C6
:100570002B312C204C617374204C696E653A20003D
:100580004D3131300053657269616C207374617450
:100590007573206D69736D617463680A00776169B2
:1005A000740A0053442072656164206572726F7230
:1005B0000A002121204B494C4C206361757365640E
:1005C00020627920746F6F206D75636820696E6199
:1005D00063746976652074696D65202D206375727A
:1005E00072656E7420636F6D6D616E643A200048B1
:1005F0006F74656E642049646C652054696D656F25
:10060000757400486F74656E642049646C6520548D
:10061000696D656F75740A002A2A2A496E697469C2
:100620006E672063617264206973204F4B2A2A2A07
:10063000004D6564696120496E736572746564007C
:100640004D656469612052656D6F766564004D315A
:100650003030305300627573793A2070617573657C
:100660006420666F7220696E7075740A006275731B
:10067000793A2070617573656420666F72207573B6
:1006800065720A00627573793A2070726F636573E0
:1006900073696E670A002A2A2A6B696C6C2A2A2AF7
:1006A00000706F7765726F6666004B494C4C45442D
:1006B0002E20005072696E7465722068616C7465DA
:1006C000642E206B696C6C28292063616C6C6564F6
:1006D000210A006563686F3A004572726F723A00D2
:1006E0000A4D6561737572656420706F696E74730D
:1006F0003A0A00357835206D6573682E205A206FD0
:1007000066667365743A20002F2F616374696F6E9B
:100710003A00656E640053656E64204D31303820B8
:10072000746F20726573756D650A00496E7365722A
:10073000742066696C616D656E7420616E642073EF
:10074000656E64204D3130380A0052656865617409
:100750002066696E69736865642E0052656865611C
:100760007420446F6E6500526568656174696E67D8
:100770002E2E2E00526568656174004865617465AF
:10078000722054696D656F75740053656E64204DF9
:1007900031303820746F2068656174206E6F7A7A0A
:1007A0006C650A004E6F7A7A6C65205061726B65D9
:1007B0006400486F74656E6420746F6F20636F6CA3
:1007C000640A00706175736564005061757365003B
:1007D00050757267654D6F72650050617573656421
:1007E0000070726F6D70745F0073686F7700627570
:1007F00074746F6E00626567696E004C6F6164208F
:1008000046696C616D656E74004C6F616420466969
:100810006C616D656E74205400496E73657274204E
:1008200066696C616D656E7420616E642073656EBF
:1008300064204D3130380A00726573756D6564004F
:10084000526573756D696E670057616974696E678B
:1008500020666F72206865617475702E0A004C65A1
:100860006176696E6720473236003F537065636971
:100870006669656420582C5920636F6F7264696ED5
:10088000617465206F7574206F6620626F756E6489
:10089000732E0A003F2852296570656174207661C5
:1008A0006C7565206E6F7420706C61757369626C15
:1008B000653B206D757374206265206174206C65E2
:1008C00061737420312E0A003F28522965706561DA
:1008D00074206D757374206265207370656369663A
:1008E000696564207768656E206E6F742075736922
:1008F0006E6720616E204C43442E0A003F537065A2
:10090000636966696564206E6F7A7A6C65207465C8
:100910006D7065726174757265206E6F7420706C95
:1009200061757369626C652E0A003F537065636977
:10093000666965642066696C616D656E74207369B3
:100940007A65206E6F7420706C61757369626C6576
:100950002E0A003F53706563696669656420707292
:10096000696D65206C656E677468206E6F742070A9
:100970006C61757369626C652E0A003F5072696D17
:1009800065206C656E677468206D75737420626590
:1009900020737065636966696564207768656E2099
:1009A0006E6F74207573696E6720616E204C4344CE
:1009B0002E0A003F537065636966696564206E6F37
:1009C0007A7A6C652073697A65206E6F7420706C1A
:1009D00061757369626C652E0A003F5265747261BD
:1009E0006374696F6E204D756C7469706C696572A3
:1009F000206D757374206265207370656369666924
:100A000065642E0A003F53706563696669656420FA
:100A100052657472616374696F6E204D756C746990
:100A2000706C696572206E6F7420706C617573698B
:100A3000626C652E0A003F53706563696669656480
:100A4000206C6179657220686569676874206E6FD3
:100A50007420706C61757369626C652E0A0043299D
:100A60002E0A003F5370656369666965642062659C
:100A7000642074656D7065726174757265206E6F47
:100A80007420706C61757369626C65202834302D38
:100A900000473236207374617274696E672E2E2E91
:100AA0000A004F46460A004661646520486569674A
:100AB00068742000426564204C6576656C696E67D9
:100AC00020004661696C656420746F20656E616208
:100AD0006C6520426564204C6576656C696E670ABA
:100AE000004D65736820426564204C6576656C2016
:100AF000646174613A0A00496E76616C6964206DC4
:100B00006573682E0A00206E6F7420656E746572BE
:100B100065642E0A0050726F62696E6720506F69BB
:100B20006E740025532025692F256900206F6620EB
:100B3000004D424C2047323920706F696E7420009E
:100B4000290A004A206F7574206F662072616E67F3
:100B5000652028302D00290A0049206F7574206F08
:100B6000662072616E67652028302D004732384C50
:100B700030004D6573682070726F62696E67206423
:100B80006F6E65004D6573682070726F62696E6785
:100B900020646F6E652E0A005374617274206D6557
:100BA00073682070726F62696E672077697468205D
:100BB00022473239205331222066697273742E0A1B
:100BC000004732395332004732384C300A47323905
:100BD000533200686173206E6F20646174612E0A65
:100BE000004D65736820426564204C6576656C69CC
:100BF0006E67200053206F7574206F662072616EDF
:100C000067652028302D35292E0A004D6573682030
:100C1000706F696E74206F7574206F662072616EDC
:100C200067650A004D34323120696E636F727265F8
:100C3000637420706172616D657465722075736193
:100C400067650A00546F6F6C6368616E67653A0090
:100C500020204D32313700205700204C0020410029
:100C60002047002046002055002052002053003D20
:100C70003D4F6E506F7765724C6F7373526573752D
:100C80006D653D3D004D32342053256C6420542564
:100C90006C64004739322E392045257300473120D6
:100CA000462564004739322E39205A2573004731D2
:100CB000205A3020463230300047312058257320EA
:100CC00059257320463330303000473132004D34DF
:100CD000323020532569205A2573004D313036209B
:100CE00050256920532569005425692053004D3251
:100CF000303020542569204430004D3230302054AB
:100D0000256920442573004732385230585900472E
:100D100039322E39204530205A300A47315A25734E
:100D2000004D31303920532569004D313930205381
:100D30002569004D343230205330205A300020498C
:100D40006E76616C69642065787472756465722072
:100D50000047322F47332062616420706172616DF9
:100D600065746572730A00536C6565702E2E2E00D3
:100D70004D65736820706F696E74206F7574206F95
:100D8000662072616E67650A004D302053746F7083
:100D9000004D312053746F7000436F6E74696E752F
:100DA0006500436C69636B20746F20526573756DC9
:100DB000652E2E2E004E6F204D6F76652E00456EEF
:100DC000642066696C65206C6973740A004265670B
:100DD000696E2066696C65206C6973740A004E6FD9
:100DE000206D656469610A00526573756D696E678F
:100DF00020534400286E6F2066696C652900437596
:100E00007272656E742066696C653A200050726972
:100E10006E742074696D653A20000A5374617473AE
:100E20003A2046696C616D656E7420757365643A2D
:100E300020002C204C6F6E67657374206A6F623AD5
:100E40002000546F74616C2074696D653A20005302
:100E5000746174733A20002C204661696C65643AB1
:100E600020002C2046696E69736865643A20005042
:100E700072696E74733A200053746174733A20007F
:100E80006F6B006F6666003A0435042E0427041960
:100E90000444454255473A004D3131332053004216
:100EA000656420436F6F6C696E672E2E2E0042655D
:100EB000642048656174696E672E2E2E00544D3390
:100EC000442043522D58204F46462E002F2F0020FD
:100ED0005200416363656C65726174696F6E3A209C
:100EE00050005741524E494E4721204C6F77205AAF
:100EF000204A65726B206D6179206C656164207495
:100F00006F20756E77616E746564207061757365AE
:100F1000732E0A004D3230362058004F4646004F9F
:100F20004E0020204D61783A2000200020204D699D
:100F30006E3A2000536F667420656E6473746F7030
:100F4000733A200046523A0020466C6F773A2000F0
:100F50004261627973746570205A004D424C2041A1
:100F6000646A757374205A0020643A0020693A005C
:100F700020703A00496E76616C69642065787472FD
:100F8000756465720A0020643A0020693A00207096
:100F90003A0064697300656E0043290A0061626C5F
:100FA000656420286D696E2074656D702000436F44
:100FB0006C64206578747275646573206172652055
:100FC00000504944204175746F74756E6500504936
:100FD00044204175746F74756E65206661696C6537
:100FE00064212042616420686561746572206964CF
:100FF0000A004F666673657473204170706C696592
:1010000064004572723A20546F6F2066617221004D
:10101000546F6F206661722066726F6D2072656614
:101020006572656E636520706F696E740A00454570
:1010300050524F4D204F4B0A002E0A002028302DD1
:10104000313029002076616C7565206F7574206FD2
:10105000662072616E676500416476616E6365202B
:101060004B00506F7765722D6C6F737320726563E0
:101070006F7665727920004D383400446F6E6520BC
:101080007072696E74696E672066696C650A004DDE
:101090003737004D3331004361703A004D454154BC
:1010A0005041434B00434F4F4C45525F54454D50C8
:1010B00045524154555245004348414D4245525FC7
:1010C00054454D50455241545552450042414259B4
:1010D0005354455050494E470041524353004D4FE1
:1010E00054494F4E5F4D4F44455300544845524D6F
:1010F000414C5F50524F54454354494F4E004C4F62
:101100004E475F46494C454E414D45004155544F71
:101110005245504F52545F53445F535441545553BA
:101120000053445F5752495445005245504541547D
:10113000005344434152440050524F4D50545F536A
:101140005550504F525400454D455247454E435916
:101150005F50415253455200434153455F4C49470C
:1011600048545F4252494748544E45535300544FE8
:1011700047474C455F4C494748545300534F4654EA
:10118000574152455F504F574552004255494C44D4
:101190005F50455243454E54004C4556454C494ED0
:1011A000475F44415441005A5F50524F42450052FC
:1011B000554E4F5554004155544F4C4556454C00E3
:1011C0005052494E545F4A4F420050524F47524589
:1011D0005353004155544F5245504F52545F54455C
:1011E0004D5000564F4C554D4554524943004545CE
:1011F00050524F4D0042494E4152595F46494C456D
:101200005F5452414E534645520053455249414C5A
:101210005F584F4E5F584F4646004649524D574122
:1012200052455F4E414D453A4D61726C696E2032B8
:101230002E302E375F4457372E3320544D33442001
:1012400053534D444E4E2028417072203234203288
:101250003032312032303A35353A32342920534F4A
:10126000555243455F434F44455F55524C3A68746D
:101270007470733A2F2F6769746875622E636F6D8F
:101280002F496E73616E6974794175746F6D617405
:10129000696F6E2F4D61726C696E2F747265652F68
:1012A000437265616C6974794477696E5F322E3080
:1012B0002050524F544F434F4C5F56455253494F65
:1012C0004E3A312E30204D414348494E455F5459E6
:1012D00050453A544D33442043522D5820455854DC
:1012E00052554445525F434F554E543A322055555E
:1012F00049443A63656465326132662D3431613246
:101300002D343734382D396231322D63353563361B
:10131000326633363766660A0043616E6E6F74203C
:101320006F70656E20737562646972200025697341
:101330000025696D20256973002569682025696D80
:101340002025697300256964202569682025696D59
:10135000202569730025697920256964202569683D
:101360002025696D20256973003D3D4477696E2015
:10137000496E697420436F6D706C6574653D3D0006
:101380002A2A2A4E6F7A7A6C6554656D705374619F
:101390007475735B325D203D003D3D486561746945
:1013A0006E6720446F6E65204368616E67652046F6
:1013B000696C616D656E743D3D00202073746172CF
:1013C0007470726F677265737320003D3D77616959
:1013D0007477617920353D3D003D3D7761697477D3
:1013E000617920343D3D003D3D77616974776179D5
:1013F00020333D3D003D3D7761697477617920314F
:101400003D3D003D3D6F6E5072696E7454696D656F
:101410007253746F707065643D3D003D3D6F6E4664
:101420006163746F727952657365743D3D00270A7C
:101430000A0000272027002027002D006E6F746906
:101440006669636174696F6E200063616E63656CC9
:10145000005072696E742041626F7274656400445A
:1014600069736D6973730055492041626F727465C9
:101470006400726573756D65002A2A2A43506C6199
:101480007920546F6E652A2A2A005761726E696E40
:10149000673A20436C65616E20436972636C652016
:1014A00072657175697265732058590A00576172C7
:1014B0006E696E673A20526164697573204F757466
:1014C000206F662052616E67650A004E6F7A7A6CF3
:1014D0006520746F6F20636F6C64202D20536B69DF
:1014E0007070696E6720776970650A003D3D6F6EA8
:1014F0005072696E7454696D65725061757365647C
:101500003D3D00486F6D696E67204661696C65649A
:10151000006F70656E00545249474745524544007C
:101520003A20007A5F6D696E00795F6D696E0078B0
:101530005F6D696E005265706F7274696E672065C9
:101540006E6473746F70207374617475730A000035
:10155000809D4300009A430000C843000000000043
:101560000000000000000020746F6F206C6F6E6739
:1015700020657874727573696F6E20707265766518
:101580006E7465640A0020636F6C64206578747201
:101590007573696F6E2070726576656E7465640A26
:1015A0000000000000000000000000000057617211
:1015B0006E696E673A20486F6D696E672042756D7F
:1015C000702044697669736F72203C20310A0002F2
:1015D000020400809D4300009A430000C8430000BD
:1015E0000041000000410000004000000001000038
:1015F00000010000800055555500000040003333C5
:101600003300AAAA2A004992240000002000C771D2
:101610001C0099991900D1451700555515003BB18B
:1016200013002449120011111100000010000F0FC7
:101630000F00E3380E0043790D00CCCC0C00C33012
:101640000C00E8A20B0064210B00AAAA0A00703D5E
:101650000A009DD80900427B090092240900DCD3CE
:101660000800888808001042080000000800F0C147
:1016700007008787070075500700711C07003EEBC5
:101680000600A1BC06006990060066660600703E72
:1016900006006118060017F4050074D105005BB060
:1016A0000500B290050062720500555505007839B5
:1016B0000500B81E0500050505004EEC040087D4A2
:1016C0000400A1BD040090A7040049920400C17D5C
:1016D0000400EE690400C7560400444404005C3270
:1016E00004000821040041100400000004003FF041
:1016F0000300F8E0030026D20300C3C30300CCB507
:1017000003003AA803000A9B0300388E0300C0813F
:1017100003009F750300D0690300505E03001D5352
:10172000030034480300913D0300333303001629BE
:101730000300381F030097150300300C0300030358
:1017400003000BFA020049F10200BAE802005CE073
:1017500002002DD802002DD0020059C80200B0C0EE
:10176000020031B90200DAB10200AAAA0200A0A365
:101770000200BC9C0200FA9502005C8F0200DF8828
:10178000020082820200457C020027760200277058
:101790000200436A02007C640200D05E02003F59EE
:1017A0000200C8530200FFFDFCFAF8F6F4F2F0EE76
:1017B000ECEAE9E7E5E3E1E0DEDCDAD9D7D5D4D23B
:1017C000D0CFCDCBCAC8C7C5C3C2C0BFBDBCBAB9D4
:1017D000B7B6B4B3B2B0AFADACAAA9A8A6A5A4A23F
:1017E000A1A09E9D9C9A99989795949392908F8E84
:1017F0008D8B8A8988878684838281807F7E7D7BAA
:101800007A797877767574737271706F6E6D6C6BB0
:101810006A696867666564636261605F5E5D5C5BA0
:101820005A5958585756555453525150504F4E4D7F
:101830004C4B4A4A49484746464544434242414048
:101840003F3E3E3D3C3B3B3A393838373635353400
:101850003332323130302F2E2E2D2C2B2B2A2929AA
:1018600028272726252524232322212120201F1E47
:101870001E1D1C1C1B1B1A191918181716161515D6
:1018800014131312121111100F0F0E0E0D0D0C0C5C
:101890000B0A0A09090808070706060505040403D8
:1018A00003020201000020746F6F206C6F6E6720CE
:1018B000657874727573696F6E2070726576656E87
:1018C0007465640A0020636F6C64206578747275B7
:1018D00073696F6E2070726576656E7465640A0058
:1018E0003D3D6F6E5072696E7454696D65725374CC
:1018F00061727465643D3D003D3D6F6E53746F725F
:101900006553657474696E67733D3D003D3D6F6E50
:10191000436F6E66696775726174696F6E53746F39
:1019200072655772697474656E3D3D0053657474D9
:10193000696E67732053746F726564000A20696E64
:101940006974207A70726F62655F7A6F666673651C
:1019500074203D20003D3D6F6E436F6E6669677574
:10196000726174696F6E53746F7265526561643D24
:101970003D00454550524F4D20496E697469616C78
:10198000697A65640A003B200020204D3630332000
:1019900000546F6F6C2D6368616E67696E673A0003
:1019A0002055005431204C002055005430204C006C
:1019B00046696C616D656E74206C6F61642F756E25
:1019C0006C6F6164206C656E677468733A00204BBD
:1019D0000020204D3930302054004C696E65617212
:1019E00020416476616E63653A0020204D343133C6
:1019F000205300506F7765722D4C6F7373205265C2
:101A0000636F766572793A002044002049002020F7
:101A10004D33303420500020440020490020204D18
:101A20003330312050005049442073657474696E1E
:101A300067733A002020473239205334205A00205F
:101A40004A00202047323920533320490020204DBE
:101A50003432302053004D65736820426564204C59
:101A60006576656C696E673A0020204D323036200D
:101A70005800486F6D65206F66667365743A002084
:101A8000580020530020204D323035204200416460
:101A900076616E6365643A20423C6D696E5F736582
:101AA000676D656E745F74696D655F75733E205315
:101AB0003C6D696E5F66656564726174653E205455
:101AC0003C6D696E5F74726176656C5F66656564B6
:101AD000726174653E20583C6D61785F785F6A651D
:101AE000726B3E20593C6D61785F795F6A65726BFD
:101AF0003E205A3C6D61785F7A5F6A65726B3E206A
:101B0000453C6D61785F655F6A65726B3E0020548D
:101B10000020520020204D323034205000416363B9
:101B2000656C65726174696F6E2028756E69747377
:101B30002F7332293A20503C7072696E745F616372
:101B400063656C3E20523C726574726163745F61C0
:101B50006363656C3E20543C74726176656C5F61B2
:101B60006363656C3E0020204D3230312058004DBB
:101B70006178696D756D20416363656C6572617430
:101B8000696F6E2028756E6974732F7332293A005D
:101B900020204D3230332058004D6178696D756DCD
:101BA000206665656472617465732028756E69745A
:101BB000732F73293A005374657073207065722017
:101BC000756E69743A0020204D3230302053002069
:101BD000440020204D32303020540020446973618D
:101BE000626C65640A0046696C616D656E74207391
:101BF000657474696E67733A0020286D6D29002042
:101C000020473231202020203B20556E69747320FC
:101C1000696E206D6D003D3D6F6E4C6F6164536564
:101C20007474696E67733D3D000000FA430000FA6A
:101C30004300002041000096420000A0420000A0A6
:101C4000420000C8430000BE42DC050000DC050085
:101C500000640000004B00000024F4D43050C38E18
:101C600020C2A24017828B7011127A910D816CD91B
:101C70000AA861E108C7586607615143061E4B5D1B
:101C800005C145A7041A411104093D980371393172
:101C9000034036DB0265339102D4305402802E1D9E
:101CA00002632CEE01752AC501B028A0011027811E
:101CB000018F2564012B244B01E0223401AC211F4C
:101CC000018D200D01801FFC00841EED00971DDF9B
:101CD00000B81CD200E61BC600201BBC00641AB270
:101CE00000B219A8000A19A0006A189900D117912A
:101CF0000040178B00B516840031167E00B31579AD
:101D0000003A157300C7146F0058146A00EE13668A
:101D1000008813630025135E00C7125B006C125726
:101D20000015125400C111510070114F0021114BC8
:101D300000D61049008D10470046104400021042A2
:101D400000C00F4000800F3E00420F3C00060F3BDA
:101D500000CB0E3800930E37005C0E3500270E3492
:101D600000F30D3200C10D3100900D3000600D2EDA
:101D700000320D2D00050D2C00D90C2B00AE0C29C6
:101D800000850C29005C0C2700350C27000E0C2662
:101D900000E80B2400C40B2400A00B23007D0B23C0
:101DA000005A0B2100390B2100180B2000F80A1FE4
:101DB00000D90A1E00BB0A1E009D0A1D00800A1DD4
:101DC00000630A1C00470A1B002C0A1B00110A1A98
:101DD00000F7091A00DD091900C4091900AB091937
:101DE00000920917007B091800630917004C0916B7
:101DF0000036091600200916000A091500F5081515
:101E000000E0081400CC081400B8081400A408145A
:101E100000900813007D0812006B08130058081288
:101E2000004608120034081100230811001208119E
:101E30000001081100F0071000E0071000D00710A3
:101E400000C0071000B0070F00A107100091070E97
:101E50000083070F0074070F0065070E0057070E79
:101E60000049070E003B070D002E070E0020070D4E
:101E70000013070D0006070D00F9060C00ED060D16
:101E800000E0060C00D4060C00C8060C00BC060CD2
:101E900000B0060C00A4060B0099060C008D060B82
:101EA0000082060B0077060B006C060B0061060A29
:101EB0000057060B004C060A0042060A0038060AC4
:101EC000002E060A0024060A001A060A0010060957
:101ED0000007060A00FD050900F4050900EB0509E5
:101EE00000E2050900D9050900D0050900C7050968
:101EF00000BE050900B5050800AD050800A50509E7
:101F0000009C050800940508008C0508008405085D
:101F1000007C050800740508006C050700650508CD
:101F2000005D050700560508004E05070047050738
:101F3000004005080038050700310507002A05079D
:101F400000230507001C050600160507000F0507FE
:101F5000000805060002050700FB040600F504075B
:101F600000EE040600E8040600E2040700DB0406B5
:101F700000D5040600CF040600C9040600C3040609
:101F800000BD040600B7040600B1040500AC040659
:101F900000A6040600A00405009B040600950405A5
:101FA00000900406008A04050085040500800406EC
:101FB000007A04050075040500700405006B040533
:101FC0000066040500610405005C04050057040573
:101FD00000520405004D04050048040500430405B3
:101FE000003E0404003A04050035040500300404F2
:101FF000002C04050027040400230405001E04042B
:10200000001A04040016040500110404000D040461
:1020100000090405000404040000040400FC030497
:1020200000F8030400F4030400F0030400EC0304CC
:1020300000E8030400E4030400E0030400DC0304FC
:1020400000D8030400D4030400D0030400CC03042C
:1020500000C8030300C503030024F404D9201BC4F3
:102060000C5C0E9804C4095F0265077101F405F960
:1020700000FB04B30048048700C1036900580355FE
:102080000003034500BE023A008402310053022AD5
:10209000002902250004022000E4011C00C80119E7
:1020A00000AF0117009801140084011300710110A2
:1020B000006101100051010E0043010D0036010BBB
:1020C000002B010B0020010B00150109000C010978
:1020D0000003010800FB000800F3000800EB000704
:1020E00000E4000600DE000600D8000600D200066C
:1020F00000CC000500C7000500C2000500BD0004BB
:1021000000B9000400B5000400B1000400AD0004F3
:1021100000A9000400A5000300A20003009F000422
:10212000009B000300980003009500020093000349
:1021300000900003008D0002008B00030088000265
:10214000008600020084000300810002007F00027C
:10215000007D0002007B0002007900020077000190
:10216000007600020074000200720001007100029B
:10217000006F0002006D0001006C0002006A0001A7
:1021800000690002006700010066000100650001AF
:1021900000640002006200010061000100600001B3
:1021A000005F0002005D0001005C0001005B0001B7
:1021B000005A0001005900010058000100570001B9
:1021C00000560001005500010054000100530000BA
:1021D00000530001005200010051000100500001B5
:1021E000004F0001004E0000004E0001004D0001B4
:1021F000004C0001004B0000004B0001004A0001B0
:1022000000490001004800000048000100470001AB
:1022100000460000004600010045000000450001A6
:1022200000440001004300000043000100420000A0
:102230000042000100410000004100010040000197
:10224000003F0000003F0001003E0000003E000192
:10225000003D0000003D0001003C0000003C00008B
:10226000003C0001003B0000003B0001003A000080
:10227000003A000100390000003900010038000078
:10228000003800000038000100370000003700016E
:102290000036000000360000003600010035000066
:1022A000003500000035000100340000003400005B
:1022B000003400010033000000330000003300014F
:1022C0000032000000320000003200010031000046
:1022D000003100000031000100300000003000003B
:1022E00000300001002F0000002F0000002F000030
:1022F000002F0001002E0000002E0000002E000123
:10230000002D0000002D0000002D0000002D000118
:10231000002C0000002C0000002C0000002C00010C
:10232000002B0000002B0000002B0000002B000100
:10233000002A0000002A0000002A0000002A0001F4
:1023400000290000002900000029000000290000E9
:1023500000290001002800000028000000280000DB
:1023600000280000002800010027000000270000CE
:1023700000270000002700000027000100260000C1
:1023800000260000002600000026000000260001B4
:1023900000250000002500000025000000250000A9
:1023A000002500000025000100240000002400009A
:1023B000002400000024000000240001002300008D
:1023C0000023000000230000002300000023000081
:1023D0000023000000230001002200000022000072
:1023E0000022000000220000002200000022000164
:1023F0000021000000210000002100000021000059
:102400000021000000210000002100010020000048
:10241000002000000020000000200000002000003C
:10242000002000000020000000200001001F00002C
:10243000001F0000001F0000001F0000001F000020
:10244000001F0000001F0001001E0000001E000011
:10245000001E0000001E000000232C0000B8220017
:1024600000561800003A0F0000B8080000B1040040
:1024700000710200003E01000020436F756E742061
:10248000583A0023646566696E65204445464155A7
:102490004C545F0000626564004B6420004B69206F
:1024A000004B702000504944204175746F74756E64
:1024B000652066696E6973686564212050757420B3
:1024C000746865206C617374204B702C204B6920FC
:1024D000616E64204B6420636F6E7374616E7473FD
:1024E0002066726F6D2062656C6F7720696E746F05
:1024F00020436F6E66696775726174696F6E2E68CE
:102500000A00504944204175746F74756E652066E9
:1025100061696C6564212074696D656F75740A006A
:10252000504944204175746F74756E652066616909
:102530006C6564212054656D706572617475726597
:1025400020746F6F20686967680A00204B643A2026
:1025500000204B693A2000204B703A200020436C49
:10256000617373696320504944200A00204E6F2034
:102570006F76657273686F6F740A002054753A2025
:1025800000204B753A2000206D61783A2000206DC4
:10259000696E3A200020643A200020626961733A33
:1025A0002000504944204175746F74756E65207326
:1025B000746172740A00504944204175746F7475D7
:1025C0006E65206661696C6564212054656D706577
:1025D00072617475726520746F6F20686967680A2C
:1025E0000042656400453100626564002C20737907
:1025F0007374656D2073746F707065642120486515
:10260000617465725F49443A200048656174696E7F
:1026100067204661696C65640048656174696E672E
:10262000206661696C6564004D31313220536875F4
:1026300074646F776E001000C90210012C01400114
:10264000220170011801B0010E01F00104015002D5
:10265000FA00B002F0003003E600D003DC00900482
:10266000D2007005C800A006BE000008B400B00982
:10267000AA00D00BA000600E960060118C0000151F
:10268000820020197800C01D6E00A0226400B027CF
:102690005A00902C500000314600E0343C001038C5
:1026A0003200903A2800603C1E00A03D1400803E9D
:1026B0000A00203F0000544845524D414C205255DD
:1026C0004E4157415900546865726D616C205275D6
:1026D0006E61776179004572723A204D41585445D8
:1026E0004D50004D415854454D50207472696767F4
:1026F00065726564004572723A204D494E54454DED
:1027000050004D494E54454D5020747269676765BD
:1027100072656400202F002042403A0020403A00B9
:1027200020573A0020573A00496E76616C69642060
:1027300065787472756465720A00416374697665C0
:102740002045787472756465723A2000486F74652C
:102750006E6420746F6F20636F6C640A007C3C3E73
:102760005E2B3D3F2F5B5D3B2C2A225C0043616E5C
:102770006E6F74206F70656E20737562646972206D
:1027800000534420496E6974204661696C005344CB
:102790002063617264206F6B0A006F70656E526F08
:1027A0006F74206661696C65640A00766F6C756D84
:1027B000652E696E6974206661696C65640A004EF5
:1027C0006F20534420636172640A000A4D32340062
:1027D0004D3233202573002E0A006F70656E20661F
:1027E00061696C65642C2046696C653A2000466915
:1027F0006C652073656C65637465640A00205369B9
:102800007A653A200046696C65206F70656E656474
:102810003A2000454E4420535542524F5554494E9C
:10282000450A002220706F73002220706172656E6D
:10283000743A2200535542524F5554494E45204355
:10284000414C4C207461726765743A220053756282
:1028500063616C6C204F766572666C6F77004578AB
:10286000636565646564206D617820535542524FFD
:102870005554494E452064657074683A002E0A002C
:1028800044656C6574696F6E206661696C65642C63
:102890002046696C653A200046696C652064656C69
:1028A000657465643A005344207072696E74696E91
:1028B00067206279746520004E6F74205344207045
:1028C00072696E74696E670A0057726974696E671F
:1028D00020746F2066696C653A20006672657368C3
:1028E00000646F696E67002066696C653A20004E6F
:1028F0006F7720002F6175746F25632E670060016C
:10290000F4017001EA019001E001B001D601D001AB
:10291000CC010002C2013002B8016002AE01900297
:10292000A401D0029A012003900170038601C00324
:102930007C0130047201A004680120055E01B0052D
:10294000540160064A0120074001F0073601F008F3
:102950002C01100A2201500B1801C00C0E01500E60
:1029600004013010FA002012F0005014E600C016E6
:10297000DC007019D200501CC800501FBE0070222D
:10298000B400B025AA00F028A000202C9600302F1B
:102990008C0010328200A0347800F0366E00E038EF
:1029A0006400803A5A00403B5500E03B5000F03C48
:1029B0004600C03D3C00603E3200E03E2800303F13
:1029C0001E00503F1900703F1400A03F0A00C03F96
:1029D0000000D03FF6FFE03FECFF2020506C616E1E
:1029E0006E657242756666657242797465733A20E7
:1029F000002046726565204D656D6F72793A200042
:102A0000436F6D70696C65643A2041707220323496
:102A100020323032310A00204C61737420557064CA
:102A2000617465643A20323032312D30342D3138C2
:102A3000207C20417574686F723A2054696E794D1C
:102A4000616368696E657333440A00322E302E3735
:102A50005F4457372E330A004D61726C696E002057
:102A6000536F6674776172652052657365740A00EE
:102A7000205761746368646F672052657365740AD8
:102A8000002042726F776E206F75742052657365F7
:102A9000740A002045787465726E616C205265730B
:102AA00065740A00506F77657255700A007374611F
:102AB00072740A004732385859004D3130303100B5
:102AC0006572726F722077726974696E6720746FB5
:102AD0002066696C650A00446F6E652073617669D3
:102AE0006E672066696C652E0A004D323900456EAE
:102AF0006473746F70730025532025632025632051
:102B0000256320256300205A3A0020593A002058B6
:102B10003A00656E6473746F7073206869743A204C
:102B20000000000A0B02090C0D0E08070304010047
:102B30000000000000000000000000000000000095
:102B40000000000000000000000000000012111052
:102B50000000000000000000000000000000000075
:102B600000000000000000FFFFFF486F6D6520259A
:102B70007325732573204669727374003D3D6F6E33
:102B800055736572436F6E6669726D5265717569D2
:102B90007265643D3D00220A00556E6B6E6F776E64
:102BA00020636F6D6D616E643A2022002042002028
:102BB00050006F6B00204500205A00205900204D26
:102BC000393220580020453A00205A3A0020593A1C
:102BD00000583A0043616E6E6F7420656E746572C2
:102BE000207375626469723A20004D323520500AB4
:102BF0004D323400526573756D6500554920506142
:102C0000757365004E6F204D61746368203A005003
:102C1000675570005067446F776E004973204669AE
:102C20006C6520004973204469722000476F55701D
:102C300044697200486173204D65646961004669AA
:102C40006C656E616D652053656C656374656400C9
:102C50004D3130303043004D313030300046696CFA
:102C6000616D656E7420537461742030202D2033A3
:102C70000046696C616D656E742053746174203018
:102C8000202D20320046696C616D656E742053748E
:102C900061742030202D2031002046696C616D6503
:102CA0006E7420526573706F6E7365204E6F0052A4
:102CB0006573756D652059657320647572696E67FB
:102CC000207072696E74000A204E6F2046696C6134
:102CD0006D656E7400496E76616C6964204F707426
:102CE000696F6E004D3530300053746F726520533C
:102CF000657474696E6773004265642050494420AE
:102D000053746172746564004D3939390A4D323833
:102D10003050305331363000424C546F7563682068
:102D20005265736574004D3530320A4D35303000D0
:102D3000496E697420454550524F4D00486F746587
:102D40006E64205049442053746172746564004578
:102D50006E676C69736820416C7265616479205399
:102D60006574004368696E657365204E6F74205307
:102D70007570706F7274656400496E4C616E674364
:102D8000686F696365000A202A2A2A726563646194
:102D9000742E646174615B305D203D004732380AF7
:102DA0004731204631303030205A313000556E7373
:102DB0007570706F72746564204F7074696F6E20E7
:102DC00053656C656374656400473236523235353D
:102DD00000473238004731204631303030205A30F9
:102DE0002E30004732380A4731204631303030200B
:102DF0005A302E30004D353030005A204F66667301
:102E00006574203A202573004D353030005A204F2C
:102E10006666736574203A202573004732380A4786
:102E20003146313530305A302E30004732385A0A68
:102E3000473146313530305A302E30004D3834006D
:102E4000473146313030305A302E30004732380A60
:102E5000473146313030305A302E30004D616E757A
:102E6000616C53657454656D70005A204F666673CB
:102E70006574203A2025730053746F702054726972
:102E80006767657265640053746F70204E6F0053FE
:102E9000746F705072696E740048616E646C652066
:102EA000446174612041646A7573742032205365F3
:102EB0007474696E672053637265656E20004861A3
:102EC0006E646C652044617461205072696E744652
:102ED000696C6520332053657474696E6720536391
:102EE0007265656E200048616E646C652044617493
:102EF00061205072696E7446696C6520322053659A
:102F00007474696E672053637265656E20004D3876
:102F1000340048616E646C652044617461205072B5
:102F2000696E7446696C6520506F73740048616EF9
:102F3000646C652044617461205072696E744669E6
:102F40006C652050726500426567696E53776974DD
:102F50006368003D3D20436865636B6B65793D3D6B
:102F6000007265636461742E61646472203D3D008B
:102F70007265636461742E646174615B305D203DD1
:102F80003D0077616974776179203D3D0020202AFA
:102F90002A2A2A2A2A2A5254535F48616E646C6591
:102FA000446174612A2A2A2A2A2A2A2A2000526580
:102FB00073656E643A200000002200250028002B73
:102FC000002E003100340002010000050108010B51
:102FD0000100002100240027002A002D00300033CA
:102FE0000001010000040107010A010505050507AC
:102FF0000508080808020202020A0A080804040474
:10300000040101010101010101030303030303039F
:1030100003040707070C0C0C0C0C0C0C0C0202022E
:103020000206060606060606060B0B0B0B0B0B0B21
:103030000B010210202008081020401020408002C0
:1030400001020108040201010204081020408080EE
:103050004020100804020180040201804020100872
:10306000040201080402010102040810204080014A
:1030700002040810204080436F6F6C696E672E2E2B
:103080002E0048656174696E672E2E2E004520253E
:103090005300544D33442043522D582052656164EF
:1030A000792E005072696E74696E672E2E2E005054
:1030B00072696E7420506175736564006E6F746917
:1030C0006669636174696F6E2000504944205475CD
:1030D0006E652046696E6973686564004D32340020
:1030E0009800CC0011241FBECFEFD1E2DEBFCDBFD0
:1030F00000E00CBF13E0A0E0B2E0E8E5F0E502E09C
:103100000BBF02C007900D92AE3FB107D9F726E181
:10311000AEEFB3E001C01D92AD37B207E1F718E1A1
:10312000C1E7D8E100E006C021970109802FFE0128
:103130000F944D24C037D10780E00807A9F70F94FA
:1031400041130D941A280C94000080919A129091CA
:103150009B12891B877089F48091070E81110DC025
:103160008091631290916412892B39F481E09091DF
:10317000A30A911103C080E0089581E00895CF93E0
:10318000DF93DB01F9019C919130C1F0943080F024
:1031900094509C938830D1F480819181009771F094
:1031A000019791838083480F591FEA01188206C056
:1031B0008C3539F49C5F9C93943041F4DF91CF912E
:1031C00008958B3339F781E08C93F8CF20813181DA
:1031D000B9016F5F7F4F71836083420F531FEA0114
:1031E0008883808191818F3591056CF7E7CF0F93AC
:1031F0001F9381E000918A1410918B1420918C14FC
:1032000030918D14409186145091871460918814E8
:1032100070918914041715072607370708F480E012
:103220001F910F91089590E080E00895282F9091CC
:10323000640B833021F495FD0FC094FD0FC0892FDE
:1032400090E0B0E0A0E004C0B695A795979587956B
:103250002A95D2F78170089581E0089580E008955D
:10326000129A479A0895269A2E9A08958F929F92BD
:10327000AF92BF92CF92DF92EF92FF920F931F9384
:10328000CF93DF93CDB7DEB72C970FB6F894DEBFA0
:103290000FBECDBF8B0140E050E068E472E44D8387
:1032A0005E836F83788740E050E060EA70E449878E
:1032B0005A876B877C878130B9F1823009F459C015
:1032C00020E030E040E050E46091020D7091030D89
:1032D0008091040D9091050D0F9462244B017C01A7
:1032E00020E030E048EC53E40F94C226181634F482
:1032F000812C912C88ECE82E93E4F92EF801A0841F
:10330000B184C284D3849401A701B501C6010F948E
:10331000C226181614F054016701C501D60189832D
:103320009A83AB83BC8348C0BE01675F7F4FC801EF
:1033300008960E9454C7B8016C5F7F4FAE014B5F87
:103340005F4FC8010E9432C70E9481D32C960FB6EE
:10335000F894DEBF0FBECDBFDF91CF911F910F91CB
:10336000FF90EF90DF90CF90BF90AF909F908F90A5
:103370000895F80120853185428553856091020DBD
:103380007091030D8091040D9091050D0F946224AE
:103390006B017C0120E030E048EC53E40F94841D85
:1033A00087FD06C0C12CD12C28ECE22E23E4F22E9E
:1033B000C982DA82EB82FC82BE01675F7F4FCE0159
:1033C0000196B7CFEFEFF8E01082118212821382DC
:1033D00014820C94D0F3EF92FF920F931F93CF932C
:1033E000DF93CDB7DEB78C01EDB6FEB60F94D11CDE
:1033F00001962DB73EB7281B390B0FB6F8943EBF88
:103400000FBE2DBF8DB79EB70196B8010F94CA1C91
:103410000E94A1F00FB6F894FEBE0FBEEDBEDF9184
:10342000CF911F910F91FF90EF9008958C389105E7
:1034300014F08CE890E09093EB118093EA110C94D7
:103440009F9C2F923F924F925F926F927F928F92AA
:103450009F92AF92BF92CF92DF92EF92FF920F9323
:103460001F93CF93DF93D62FC72FFC0180809180CD
:10347000A280B380C501B40120E831E541E050E00D
:103480000F94C823C9016DE671E00F9439246B01D4
:103490007C01C501B40120E13EE040E050E00F9422
:1034A000C823CA01B90128E130E040E050E00F94A0
:1034B000C823362E272E062F172F8CE3482E512C8B
:1034C000612C712CC501B401A30192010F94C82392
:1034D000B62EA72ECA01B901A30192010F94C823E9
:1034E000CB01C114D10479F1AF92BF927F936F9356
:1034F0002F923F92FF92EF92DF92CF9285E593E178
:103500009F938F93CF93DF930F941B1D8DB79EB71F
:103510000E960FB6F8949EBF0FBE8DBF8D2F9C2FB9
:10352000DF91CF911F910F91FF90EF90DF90CF909F
:10353000BF90AF909F908F907F906F905F904F90D3
:103540003F902F900895E114F104C9F0AF92BF921B
:103550007F936F932F923F92FF92EF9285E493E1D6
:103560009F938F93CF93DF930F941B1DEDB7FEB7FF
:103570003C960FB6F894FEBF0FBEEDBFCFCF012B28
:10358000B9F0AF92BF927F936F932F923F9289E3EE
:1035900093E19F938F93CF93DF930F941B1D8DB770
:1035A0009EB70A960FB6F8949EBF0FBE8DBFB6CFDA
:1035B000892BA9F0AF92BF927F936F9381E393E140
:1035C0009F938F93CF93DF930F941B1DEDB7FEB79F
:1035D00038960FB6F894FEBF0FBEEDBF9FCFAF92E7
:1035E000BF928DE293E19F938F93CF93DF930F94DC
:1035F0001B1D0F900F900F900F900F900F908ECF7C
:10360000AB01BC0140938A1450938B1460938C14CB
:1036100070938D1482EF95E10C94038E0F931F939A
:10362000CF93DF9300D01F92CDB7DEB79C0105EE9C
:103630001AE090E1EAEFFCE0D80101900D929A9532
:10364000E1F7F9012081318142815381F8016085E0
:103650007185828593850F946224F8016087718754
:103660008287938780E090E0A0EAB0E489839A8320
:10367000AB83BC83CE0101960E94C1D10F900F9005
:103680000F900F90DF91CF911F910F9108952F927E
:103690003F924F925F926F927F928F929F92AF92E2
:1036A000BF92CF92DF92EF92FF921F93CF93DF935F
:1036B000CDB7DEB72C970FB6F894DEBF0FBECDBFE7
:1036C0007A011901DC012D913D914D915C912D8381
:1036D0003E834F835887FB01408051806280738016
:1036E0008090FA0C9090FB0CA090FC0CB090FD0C1C
:1036F000A50194016D817E818F8198850F94841D31
:1037000081110EC011E0A30192016091FE0C709135
:10371000FF0C8091000D9091010D0F94841D81117B
:1037200010E0D1012D913D914D915C9129873A870F
:103730004B875C87F701C080D180E280F3802091C5
:103740000102309102024091030250910402C7012C
:10375000B6010F94841D882309F44EC0C092010263
:10376000D0920202E0920302F09204028091060DD0
:103770009091070DA091080DB091090D4091FE0C9C
:103780005091FF0C6091000D7091010D8092E50A3F
:103790009092E60AA092E70AB092E80A4093E90AFA
:1037A0005093EA0A6093EB0A7093EC0AC092ED0A18
:1037B000D092EE0AE092EF0AF092F00A8093F10ABA
:1037C0009093F20AA093F30AB093F40A20E030E059
:1037D00040E05FE36091C40C7091C50C8091C60C11
:1037E0009091C70C0F94EA1D69837A838B839C8325
:1037F000CE0101960E94C1D12D813E814F81588515
:103800002093E50A3093E60A4093E70A5093E80ACA
:103810004092E90A5092EA0A6092EB0A7092EC0A2E
:10382000D1012D913D914D915C916091F10A709182
:10383000F20A8091F30A9091F40A0F946224609343
:10384000F10A7093F20A8093F30A9093F40A11112B
:103850002FC020E030E0A90169857A858B859C85A1
:103860000F94841D811133C060E070E088EC92E415
:1038700069837A838B839C83CE0101960E94C1D198
:103880002C960FB6F894DEBF0FBECDBFDF91CF915F
:103890001F91FF90EF90DF90CF90BF90AF909F90DF
:1038A0008F907F906F905F904F903F902F900895F2
:1038B0002AEF3EE74AE25FE36091C80C7091C90CC1
:1038C0008091CA0C9091CB0C0F94EA1DD1CF60E08F
:1038D00070E080EA91E4CCCF8091D5049091D60439
:1038E000009731F04AE050E070E060E00D949F1BDB
:1038F00060E070E0CB0108950F931F93CF93DF93A7
:1039000000D000D01F921F92CDB7DEB78B01FC0113
:1039100023A5211102C00E94F2F11D821E821F8286
:10392000188620E030E040E05FE36091020D709186
:10393000030D8091040D9091050D0F94622469830D
:103940007A838B839C839E012B5F3F4FAE014F5F39
:103950005F4F6EEF7CE08AEF9CE00E94471B1D8268
:103960001E821F82188620E030E040E05FE3F8010D
:1039700060857185828593850F94622469837A833B
:103980008B839C83B8016C5F7F4F9E012B5F3F4F01
:10399000AE014F5F5F4FC8010E94471B28960FB6CC
:1039A000F894DEBF0FBECDBFDF91CF911F910F9175
:1039B00008958091D5049091D604009731F04AE0A3
:1039C00050E070E060E00D94711A60E070E0CB01AF
:1039D00008950E94D91C97FD0CC00E94D91C6F3F0E
:1039E00071058105910509F034F40E94D91C862FD8
:1039F000089580E008958FEF08958091D504909107
:103A0000D604892B41F00E94E91C91E0811101C08C
:103A100090E0892F089591E0FCCFCF92DF92EF9252
:103A2000FF92CF93C62FFC01C080D180E280F3804B
:103A300020E030E0A901C701B6010F94841D20E009
:103A400030E0A90187FD14C020E030E048EC52E4EA
:103A5000C701B6010F94C22624E630E040E050E0F2
:103A6000181634F0C701B6010F94CE259B01AC01A6
:103A7000AFEFB0E00F94092424E630E040E050E0DE
:103A80000F94EA23B9018C2FCF91FF90EF90DF9034
:103A9000CF900C94CEA08091090180FD06C080914A
:103AA0008E1483FB882780F9089580E00895CF92D3
:103AB000DF92EF92FF92FC01C080D180E280F38020
:103AC000663019F510920409109205091092060942
:103AD00010920709109208090E949F9C20E030E094
:103AE000A901C701B6010F94841D87FF1DC0C12C19
:103AF000D12C7601C701B6010F94CF26CB01FF90E0
:103B0000EF90DF90CF900C94161A0E94E21920E0FB
:103B100030E0A901C701B6010F94841D87FF15C0CD
:103B2000C12CD12C760122C020E030E04CE053E4DF
:103B3000C701B6010F94C2261816E4F6C12CD12C89
:103B40009CE0E92E93E4F92ED5CF20E030E849ED52
:103B500053E4C701B6010F94C22618163CF4C12CD9
:103B600080E8D82E89EDE82E83E4F82EC701B6014F
:103B70000F94CF26CB01FF90EF90DF90CF900C9465
:103B800085C19091970C977081E0973009F080E0A3
:103B9000089560919D1170919E11072E000C880B65
:103BA000990B0F948B1D20917F05309180054091DA
:103BB0008105509182050F94EA1D20E030E0A901B3
:103BC0000F9462240895E091F80CE150E73028F456
:103BD000F0E0E155FD4F8081089580E00895CF9396
:103BE000DF931092570C1092E20C1092E40C10929A
:103BF000E30C10925B0510925A05CFEFDFEF809136
:103C00008E1485FD07C00E945F89D093E512C09392
:103C1000E412F5CF8FEF9FEF9093E5128093E412BB
:103C2000DF91CF9108958F929F92AF92BF92CF92E2
:103C3000DF92EF92FF920F931F93CF93DF93109237
:103C40000F0510920E052FE320930D0510920C0521
:103C500010920B0510920A051092060510920705A6
:103C600010920805109209059C01F90190812F5FBF
:103C70003F4F9032D1F39E34C9F4818190ED980F7B
:103C80009A3020F08D3211F08B3281F432969F0100
:103C90002F5F3F4F808180538A3008F47BC09F01A3
:103CA0002F5F3F4F8081803209F476C0F093F90A8C
:103CB000E093F80A8F010F5F1F4FC0816AE270E046
:103CC000C8010F94B027009731F0FC013197808133
:103CD0008032E1F31182CD3429F0C43519F0C734B4
:103CE00009F04BC0F80180810F5F1F4F8032D1F384
:103CF00080538A3008F041C0C0930D0530E020E0C9
:103D00004AE0DF011196429FC001439F900D1124AC
:103D10009C01205331098081280F311D87FD3A9580
:103D2000818190ED980F9A30C8F130930C05209363
:103D30000B058E3261F4329690E04AE0DF01319655
:103D40008C9150ED580F5A3058F190930A05CD01DF
:103D5000DC0101964C914032D9F3CD3489F52E31F6
:103D6000310539F018F52731310519F02C313105BD
:103D700039F5B0930F05A0930E05DF91CF911F91F8
:103D80000F91FF90EF90DF90CF90BF90AF909F90FA
:103D90008F900895F9017BCFF90181CFFD01B1CF5B
:103DA000949F800D112490ED980FC8CF25373105D1
:103DB00038F027373105E8F2203A83E03807C9F2B6
:103DC000D091F80A40E050E0BA0110E000E0C12CC8
:103DD000D12C7601C394FD0131968C91882309F48E
:103DE0007FC08132E1F4CD34D1F420323105B9F411
:103DF00040930605509307056093080570930905E5
:103E0000F0930F05E0930E0563E270E0CF010F948D
:103E1000B027009709F4B1CFFC011082AECF8154D6
:103E20008A3108F058C0DF019D91903291F0A0EDE9
:103E3000A90FAA30E8F09E3271F4918190539A3024
:103E4000B8F00115110519F48F010150110990E026
:103E500013C0FD01E8CF9D3211F09B3291F79181A3
:103E6000A0EDA90FAA3020F09E3259F79281E6CF3B
:103E70009E2F9D1B309759F3A82FB0E046015701A4
:103E800004C0880C991CAA1CBB1C8A95D2F748292F
:103E900059296A297B29A451BB4F9C938081815465
:103EA000DF018A3108F497CFDF018191882309F47B
:103EB00092CF90ED980F9A30B8F393ED980F92301F
:103EC00098F38B3289F3CD010196EC91E03209F041
:103ED00082CFDC01F8CF0115110501F78D01DECF8E
:103EE00010930F0500930E054093060550930705A8
:103EF000609308057093090540CF0F931F93CF93EC
:103F0000DF93C82FD0E0FE01EE0FFF1FEA5CFD4FEC
:103F100071836083CC0FDD1FCC0FDD1F8E010A5E25
:103F20001D4F072E000C880B990B0F948B1D2AE058
:103F300037ED43E25CE30F94EA1DC25ADA4F288161
:103F400039814A815B810F94EA1DF8016083718396
:103F500082839383DF91CF911F910F9108959B01ED
:103F6000AC01485F5F4FBC016C5F7F4F0C94471BF7
:103F70002F923F924F925F926F927F928F929F9279
:103F8000AF92BF92CF92DF92EF92FF920F931F9367
:103F9000CF93DF93CDB7DEB7A6970FB6F894DEBF09
:103FA0000FBECDBF8C011B015A8749874090FA0C88
:103FB0005090FB0C6090FC0C7090FD0C8090FE0CFF
:103FC0009090FF0CA090000DB090010DDB018D9141
:103FD0009D910D90BC91A02D8B8B9C8BAD8BBE8B3E
:103FE0009C01AD01C301B2010F9461246B017C01FE
:103FF000D10114968D919D910D90BC91A02D8F8B28
:10400000988FA98FBA8F9C01AD01C501B4010F949F
:1040100061246B8F7C8F8D8F9E8FA985BA858D9142
:104020009D910D90BC91A02D8B879C87AD87BE87FD
:104030009C01AD01C301B2010F9461246F8F78A37D
:1040400089A39AA3A985BA8514968D919D910D9007
:10405000BC91A02D8F87988BA98BBA8B9C01AD0149
:10406000C501B4010F9461246BA37CA38DA39EA30F
:10407000A7019601C701B6010F94EA1D6B017C01EF
:104080002B8D3C8D4D8D5E8DCA01B9010F94EA1DBB
:104090009B01AC01C701B6010F9462244B015C0186
:1040A0002B893C894D895E896B857C858D859E85B4
:1040B0000F9461242B013C012F89388D498D5A8D35
:1040C0006F85788989899A890F9461246B017C01B5
:1040D000A3019201C301B2010F94EA1D2B013C011F
:1040E000A7019601C701B6010F94EA1D9B01AC011F
:1040F000C301B2010F9462240F9410276B017C015D
:104100002F8D38A149A15AA1CA01B9010F94EA1D06
:104110002B013C012BA13CA14DA15EA1CA01B9011B
:104120000F94EA1D9B01AC01C301B2010F946224FC
:104130009B01AC01C501B4010F94C2261816B4F559
:1041400020E030E0A901C701B6010F94C22687FF25
:104150002AC0C701B601905820E030E040EA50E4A0
:104160000F94C226181614F5A10169857A85C80135
:104170000E94B81FA6960FB6F894DEBF0FBECDBF43
:10418000DF91CF911F910F91FF90EF90DF90CF9033
:10419000BF90AF909F908F907F906F905F904F9067
:1041A0003F902F900895C701B601D6CF20E030E0B0
:1041B00040E050E4C501B4010F94C226181624F45F
:1041C000B101C8010E947C1C19821A821B821C82C8
:1041D000BE016F5F7F4FC1010E94AF1F2DEC3CEC11
:1041E0004CEC5CE3C701B6010F94EA1D9B01AC01E6
:1041F000F80160817181828193810F94EA1D6D8342
:104200007E838F839887D8019B968C919B97882378
:10421000C9F02AE939E949E95FE314966D917D9186
:104220008D919C9117970F94EA1D69837A838B83F4
:104230009C83BE016F5F7F4F85EE9AE00E94AF1FA7
:10424000F80113A6BE016B5F7F4F89859A850E9496
:10425000AF1F90CF4F925F926F927F929F92AF92DB
:10426000BF92CF92DF92EF92FF920F931F93CF9363
:10427000DF93CDB7DEB768970FB6F894DEBF0FBEF9
:10428000CDBFFB019080342F390D353008F026C1A9
:10429000E180022F0E0D053008F020C1EE2DF0E078
:1042A000E453FB4F4080512C712C612C092C04C02D
:1042B00076946794579447940A94D2F740FE0EC1BF
:1042C00010E0F801E453FB4F4080512C712C612C1D
:1042D000C32ED12C04C076946794579447943A9592
:1042E000D2F740FEFBC0F22E642F5C01660F770B05
:1042F000072E000C880B990B0F948B1D2B013C0192
:10430000892D94E08902F0011124E159FB4EA301AB
:10431000920160817181828193810F9462246D8703
:104320007E878F87988BF601EE0FFF1FEE0FFF1F22
:10433000E159FB4EA30192016081718182819381D9
:104340000F94612469837A838B839C836F2D660F1E
:10435000770B072E000C880B990B0F948B1D2B01EC
:104360003C018E2D94E08902F0011124E55AFB4EA8
:10437000A301920160817181828193810F946224F3
:10438000698B7A8B8B8B9C8B000F111F000F111F79
:10439000F801E55AFB4EA30192016081718182818F
:1043A00093810F9461246D837E838F839887F501B9
:1043B00080859185A285B38589879A87AB87BC87DD
:1043C0008D8B9E8BAF8BB88F43E351E061E070E043
:1043D000CE0141960E948CA043E351E061E070E081
:1043E000CE0105960E948CA04AE351E061E070E0A6
:1043F000CE010D960E948CA04AE351E061E070E08E
:10440000CE0101960E948CA0C988DA88EB88FC88CE
:1044100027E137EB41ED58EBC701B6010F94C226F7
:1044200087FD5CC023E030E04AE953E4C701B601F0
:104430000F94841D18160CF451C0CD84DE84EF84D3
:10444000F88827E137EB41ED58EBC701B6010F942F
:10445000C22687FD43C023E030E84DE953E4C7019D
:10446000B6010F94841D1816CCF1CD80DE80EF804C
:10447000F88427E137EB41ED58EBC701B6010F9403
:10448000C22687FD2BC023E030E04AE953E4C70190
:10449000B6010F94841D18160CF1C980DA80EB80E8
:1044A000FC8027E137EB41ED58EBC701B6010F94D3
:1044B000C22687FD13C023E030E84DE953E4C7016D
:1044C000B6010F94841D18164CF0AE014F5F5F4F7C
:1044D000BE01635F7F4FC5010E94B81F68960FB68B
:1044E000F894DEBF0FBECDBFDF91CF911F910F912A
:1044F000FF90EF90DF90CF90BF90AF909F907F9014
:104500006F905F904F9008950E94D91CCB01089541
:104510000F931F93CF938091D5049091D604009769
:10452000E9F0FC018F01C1912C2F2F7D81F0C53462
:1045300011F0C536B9F7F801108270E060E00F9411
:104540001319F801C083CF911F910F91089570E066
:1045500060E0CF911F910F910D94131960E070E00E
:10456000CB01F1CF2FEB280F2A3108F047C0E22F03
:10457000F0E08091060590910705A0910805B091A3
:10458000090504C0B695A795979587952A95D2F702
:1045900080FD02C081700895E451FB4FE081EE235D
:1045A00041F18091F80A9091F90AE80FF92FF11D75
:1045B000808190ED980F9A3030F08E3251F48181E5
:1045C00080538A3098F4F093D604E093D50481E0C8
:1045D00008958D3211F08B3249F4818190ED980F5E
:1045E0009A3088F38E3211F48281EACFF0E0E0E075
:1045F000EACF1092D6041092D504E9CF80E0089556
:104600000E94B222882341F081E02091D5043091AC
:10461000D604232B09F480E00895CF93DF93EB01B8
:104620000E940023882319F00E94D91CEB01CE01BF
:10463000DF91CF910895CF93DF93EB010E94002388
:10464000882321F0DF91CF910C948422CE01DF9159
:10465000CF910895CF93C62F0E940023882319F08D
:10466000CF910C94E91C8C2FCF910895CF92DF92BB
:10467000EF92FF926A017B010E940023882331F0B0
:10468000FF90EF90DF90CF900C948822C701B60185
:10469000FF90EF90DF90CF9008954F925F926F92CE
:1046A0007F928F929F92AF92BF92CF92DF92EF92C2
:1046B000FF921F93CF93DF9300D01F92CDB7DEB749
:1046C00019821A821B821C82CE0101964C0185EE52
:1046D000C82E8AE0D82E9AEFE92E9CE0F92E2BE422
:1046E000A22E2CE0B22E10E088E5810F0E9400235C
:1046F000F40181934F01882309F4E0C00E948822CD
:104700002B013C01812F0E941619882309F4CCC08B
:10471000F7012081318142815381C301B2010F949D
:104720006224F60160837183828393831F5FF4E0C8
:10473000CF0ED11C84E0E80EF11C94E0A90EB11C50
:10474000133091F685E40E9400238C83882309F4BA
:10475000C0C00E9488226B017C0183E00E94161970
:10476000882371F02091060D3091070D4091080DBE
:104770005091090DC701B6010F9462246B017C01B1
:10478000C092F10AD092F20AE092F30AF092F40A8F
:104790008091DF08882359F180918E1482FF27C011
:1047A0008C81882321F18981811103C08A8188232A
:1047B000F1F02DEC3CEC4CE45DE36091910B7091D9
:1047C000920B8091930B9091940B0F9462249B0118
:1047D000AC016091020D7091030D8091040D9091D8
:1047E000050D0F94C226181614F40E9408EE40E03E
:1047F00050E0BA0186E40E94362320E030E0A901AF
:104800000F94C226181684F40E94882220E030E01B
:1048100040E752E40F945C2560934702709348028E
:104820008093490290934A028091630B83FD28C0D4
:1048300080918E0A882321F12091060D3091070D79
:104840004091080D5091090D6091F10A7091F20AA2
:104850008091F30A9091F40A0F94612420919B0AAD
:1048600030919C0A40919D0A50919E0A0F946224B7
:1048700060939B0A70939C0A80939D0A90939E0A72
:104880000F900F900F900F90DF91CF911F91FF909D
:10489000EF90DF90CF90BF90AF909F908F907F90E0
:1048A0006F905F904F900895F50120813181428192
:1048B0005381C301B2010F94612433CFF70180818A
:1048C0009181A281B381F60180839183A283B38316
:1048D0002DCF8091060D9091070DA091080DB091FC
:1048E000090D8093F10A9093F20AA093F30AB09312
:1048F000F40A4ECFCF93DF93C82FD62F0E94002308
:10490000882321F0DF91CF910C94FD1C8C2F0E9405
:10491000B222811101C08D2FDF91CF910895E8E877
:10492000FBE087EBDF011D928A95E9F708958091FE
:10493000DF08811104C00E948F240C943AF9809101
:104940008E1482FD0C9408EE08958091880B8823C4
:1049500061F090913E0C891308C080918E1483FF02
:1049600004C08BEC9BE00C9445F980E00895FC01B9
:10497000238121110C94C4910895CF93DF93109259
:10498000E0081092E1081092E2081092E308EEEFBE
:10499000FAE084E6DF011D928A95E9F7C0E0D0E0F5
:1049A0006D2F8C2F0E94D4EEDF5FD530C9F7CF5F1B
:1049B000C530A9F7DF91CF9108959091F90C981720
:1049C000B1F00E9403C28091F90C882341F08AEF74
:1049D0009CE00E9419C41092F90C0C94A0C781E0CD
:1049E0008093F90C8AEF9CE00E9458C1F6CF08959D
:1049F000EF92FF920F931F93CF93DF930EEF1AE086
:104A0000C5E07801D5E0F7016191719181919191B3
:104A10007F0120E030E0A9010F94841D81110EC0B8
:104A2000D15089F7C1500C5E1F4FC111EACFDF9101
:104A3000CF911F910F91FF90EF90089581E0F7CFF4
:104A4000EFE6F0E0808182608083089580919F117D
:104A50009091A011892B79F480919F119091A011D0
:104A6000892B49F420919F113091A01181E0232BD3
:104A700019F480E0089581E00895CF92DF92EF92DB
:104A8000FF926B017C0183E3C816D104E104F104B9
:104A900070F082E3C81AD108E108F10862E370E01F
:104AA00080E090E00E9491F30E94C1CAECCFC70160
:104AB000B6010E9491F3FF90EF90DF90CF900C949D
:104AC000C1CA20915C0520FF14C020E83EE3629F2C
:104AD000A001639F500D729F500D1124CA0196953D
:104AE000879596958795009731F08A950000E9F7AC
:104AF00008950C943D2508958091F80C882341F089
:104B0000813041F064E670E080E090E00C943D2557
:104B1000129AF8CF479AF6CF5F9A8091970C8E7FC2
:104B20008093970C8A9A8091970C8D7F8093970C35
:104B30008091080180958170809306018091970C87
:104B40008B7F8093970C0C94301990918E1493FB6B
:104B5000882780F993FF06C081E09091F5159111A7
:104B600001C080E00895CF93C0915D05CF7739F5FE
:104B70000E94A525882319F18091861490918714AD
:104B8000A0918814B09189140097A105B105B9F0DE
:104B9000BC01CD016D597F4F8F4F9F4F24E630E010
:104BA00040E050E00F94C82360918A1470918B14F8
:104BB00080918C1490918D140F94C823C22F8C2F48
:104BC000CF91089570E060E080E00E94CEA070E098
:104BD00060E081E00C94CEA081E008958F929F92D6
:104BE000AF92BF92CF92DF92EF92FF920F93CF934B
:104BF000DF931F92CDB7DEB75C017B0149016B01EA
:104C0000C40ED51EF501808191810F94A223898362
:104C1000002311F0F7018083BE016F5F7F4FC40155
:104C20000E949FE4F50180819181019691838083A8
:104C3000FFEFEF1AFF0AEC14FD0421F780E00F905C
:104C4000DF91CF910F91FF90EF90DF90CF90BF90C9
:104C5000AF909F908F9008959091D10095FD0CC0DA
:104C60009091D00095FF08C08093D6008091D0002D
:104C700080648093D0000895209114042F5F2F77D3
:104C80000FB607FC27C090911504921328C090918D
:104C9000D00095FF1EC09091150440911404941308
:104CA00006C09091D1009F7D9093D10012C0E92F52
:104CB000F0E0EC5EFB4F32819F5F9F773093D60030
:104CC000909315043091D00030643093D000491790
:104CD00041F3D9CF90911504921301C0FBCFE0911D
:104CE0001404F0E0EC5EFB4F828320931404809167
:104CF000D10080628093D10008958F929F92AF92ED
:104D0000BF92CF92DF92EF92FF920F931F93CF93B8
:104D1000DF937C0121E5E20EF11CD7014C914A356D
:104D200009F0A4C06C01B2E5CB0ED11CF6013081B4
:104D3000353A09F09BC0EC01C05BDF4F288123307E
:104D400008F494C08C0100561F4FD8014C93E15BCE
:104D5000FF4F308331962083EF54F1093081E05BBF
:104D6000FF4F30833038B1F43196AC54B1093C91E7
:104D70003083E854F109AF5ABF4F50E040E0225071
:104D8000330B42175307CCF4808132968D934F5FDB
:104D90005F4FF7CF233031F5313809F074C0FC0193
:104DA000EC55FF4FDC01AC5ABF4F2C91208331965C
:104DB000885A9F4FDC018C9180834801B12CA12C33
:104DC000888190E002968A159B050CF43FC0F4019F
:104DD00081914F010E942C260E94B5E4FFEFAF1A8B
:104DE000BF0AEECF323821F5FC01EC5AFF4F30817B
:104DF0004181E05BFF4F408331963083DC01AA554F
:104E0000BF4F50E040E02350330B42175307ACF63E
:104E1000FA01EE7FE45AFF4FE80FF91F60817181BC
:104E20007C9311966C9311974E5F5F4F1296EDCF66
:104E3000243019F6333809F6FC01EC5AFF4F208173
:104E40003181E05BFF4F30833196B0CF80E5DE01EA
:104E50001D928A95E9F78AE1F80111928A95E9F79E
:104E60008AE5D7018C9385EAF6018083DF91CF91A3
:104E70001F910F91FF90EF90DF90CF90BF90AF9078
:104E80009F908F900895323809F097CFADCFAF92B1
:104E9000BF92CF92DF92EF92FF920F931F93CF9327
:104EA000DF93EC0184E6C82E80E2D82EE12CF12CB1
:104EB00002E8A12C90E2B92E15E00093F313C09202
:104EC000F413D092F513E092F613F092F713B09228
:104ED000FD13A092FC131093F01380EA93E10E945B
:104EE0007D268FEFC81AD80AE80AF80A88E7C8169C
:104EF00080E2D806E104F10401F724E630E240E064
:104F000050E0BE0180EA93E1DF91CF911F910F91B4
:104F1000FF90EF90DF90CF90BF90AF900C94BAE4E9
:104F2000CF92DF92EF92FF920F931F93CF93DF9375
:104F3000CDB7DEB77C01CDB6DEB60F94D11C01969D
:104F40002DB73EB7281B390B0FB6F8943EBF0FBEE6
:104F50002DBF0DB71EB70F5F1F4FB701C8010F94CC
:104F6000CA1CF80101900020E9F73197E01BF10B12
:104F7000759720F089E792E0F801848BC8010E94C0
:104F800047270FB6F894DEBE0FBECDBEDF91CF919E
:104F90001F910F91FF90EF90DF90CF9008958F9227
:104FA0009F92AF92BF92CF92DF92EF92FF920F93B8
:104FB0001F93CF93DF930E94EF1D3AE0C32E30E2A0
:104FC000D32EE12CF12C15E002E846015701CAE08E
:104FD000D0E01092FD131092FC131093F013009385
:104FE000F3138092F4139092F513A092F613B092FB
:104FF000F71380EA93E10E947D2621978FEF881AAC
:10500000980AA80AB80A209721F78AE0C80ED11C8E
:10501000E11CF11C82EDC81680E2D806E104F1041F
:10502000A1F6C12C20E2D22EE12CF12CD5E0C2E871
:105030001092FD131092FC13D093F013C093F3134E
:10504000C092F413D092F513E092F613F092F71396
:1050500080EA93E10E947D261092FD131092FC13CA
:10506000D093F013C093F313D701C6018C529F4F16
:10507000AF4FBF4F8093F4139093F513A093F613A3
:10508000B093F71380EA93E10E947D268FEFC81A50
:10509000D80AE80AF80A8AE0C81680E2D806E104CD
:1050A000F10431F69EEDC92E90E2D92EE12CF12CBF
:1050B000D5E0C2E81092FD131092FC13D093F013C8
:1050C000C093F313C092F413D092F513E092F61349
:1050D000F092F71380EA93E10E947D268FEFC81AC1
:1050E000D80AE80AF80A86EEC81680E2D806E10473
:1050F000F10401F7CC24C39482E1D82EE12CF12CE9
:105100000AE010E0D5E0C2E81093FD130093FC1311
:10511000D093F013C093F313C092F413D092F5130D
:10512000E092F613F092F71380EA93E10E947D2655
:105130001093FD130093FC13D093F013C093F3135B
:10514000D701C6018096A11DB11D8093F4139093E1
:10515000F513A093F613B093F71380EA93E10E943E
:105160007D268FEFC81AD80AE80AF80A85E1C81622
:1051700082E1D806E104F10439F682E190E09093EF
:10518000FD138093FC13D093F013C093F31384E1C9
:1051900090E1A0E0B0E08093F4139093F513A09316
:1051A000F613B093F71380EA93E1DF91CF911F914B
:1051B0000F91FF90EF90DF90CF90BF90AF909F90B6
:1051C0008F900C947D261F920F920FB60F92112490
:1051D0000BB60F922F938F939F93EF93FF93809132
:1051E000150420911404821306C08091D1008F7D94
:1051F0008093D10012C0E82FF0E0EC5EFB4F92816B
:105200008F5F8F779093D600809315049091D00094
:1052100090649093D000281741F3FF91EF919F91F4
:105220008F912F910F900BBE0F900FBE0F901F907C
:1052300018951F920F920FB60F9211240BB60F9272
:105240000F931F932F933F934F935F936F937F938E
:105250008F939F93AF93BF93CF93DF93EF93FF937E
:10526000C091D60000911105D091100511E01D0FDD
:105270001F7390911304913108F09FC0E92FF0E063
:105280008827EA5BF64D8F4F0D944D2457298629C8
:105290009529A429AB29DD29AF29DD29B329B7290F
:1052A000DD29BB29BF29C329CA29DD29D529C03257
:1052B00029F028F5CA3011F0CD3031F5011731F061
:1052C000ED2FF0E0E05FFA4FC283D12FD0931005AD
:1052D000FF91EF91DF91CF91BF91AF919F918F910E
:1052E0007F916F915F914F913F912F911F910F91FE
:1052F0000F900BBE0F900FBE0F901F901895CD34DE
:1053000081F081E0CE3471F080E10CC0CA3338F412
:10531000C033A0F6C03291F2CD32B1F7CFCFCD3449
:1053200099F782E080931304C9CFC13359F018F480
:10533000C03221F2E9CF88E0C433A1F38BE0C83357
:1053400089F3E2CF83E0EECF84E0C03359F386E007
:10535000C13341F3D9CF85E0C833B1F6E3CF87E05D
:10536000C23391F6DFCF89E0C13371F6DBCF8AE03B
:10537000C03351F6D7CF8CE0C73331F6D3CF8DE0B1
:10538000C63311F6CFCFC03209F498CF8EE0C335C3
:1053900049F2BACF80ED8C0F8A3008F08FCF9FE0B2
:1053A000909313048093120489CFCA3019F0CD3042
:1053B00009F084CF1092130481CFCA3019F0CD3098
:1053C00009F07CCF80915A148823A1F3973079F0AB
:1053D00038F4953079F71092460210926512EACFB0
:1053E0009A3049F09F3031F70E948CE4E3CF81E09E
:1053F0008093FE08DFCF81E08093FD08DBCF9091A2
:10540000C00095FFFCCF8093C6000895CF93DF9333
:10541000EC018991882319F00E94FF29FACF8DE0D1
:105420000E94FF298AE0DF91CF910C94FF29CF924F
:10543000DF92EF92FF92CF936B017C01C42F4A3031
:1054400069F4F7FE0BC0F094E094D094C094C11CB2
:10545000D11CE11CF11C8DE20E94FF294C2FC701D9
:10546000B601CF91FF90EF90DF90CF900C94D0F9E0
:10547000CF93DF93EC01FE0184912196882319F0EC
:105480000E94FF29F8CFDF91CF9108952F923F928C
:105490004F925F926F927F928F929F92AF92BF9244
:1054A000CF92DF92EF92FF920F931F93CF93DF93F0
:1054B000CDB7DEB7CD54D1090FB6F894DEBF0FBE1D
:1054C000CDBF2A969FAF8EAF2A9727967FAF6EAF3C
:1054D00027972C965FAF4EAF2C972E963FAF2EAFEF
:1054E0002E9728960FAF28978CE0EBE7F2E0DE01CD
:1054F0001D9601900D928A95E1F78CE0E7E8F2E0C5
:10550000DE01599601900D928A95E1F7809154122F
:10551000909155128A3A9105F4F48BEC94E10E9433
:10552000382AC35BDF4F0FB6F894DEBF0FBECDBF86
:10553000DF91CF911F910F91FF90EF90DF90CF906F
:10554000BF90AF909F908F907F906F905F904F90A3
:105550003F902F90089580914B02882309F464C1F5
:1055600080914C0281117BC1A0905902B0905A02E7
:10557000C0905B02D0905C02E0904D02F0904E0231
:1055800000914F029090500220E030E84DE953E442
:10559000B701802F992D0F94C22618160CF07CC0ED
:1055A000C701A02FB92D8D879E87AF87B88BEDAA35
:1055B000F9AE0AAF9CAE20E030E848E953E4B70109
:1055C000802F992D0F94C22618160CF082C0C701A7
:1055D000A02FB92D898F9A8FAB8FBC8F30905D0231
:1055E00020905E0290915F0221969FAF2197A0913B
:1055F00060022296AFAF2297B09151022396BFAFBF
:105600002397E09152022496EFAF2497F091530232
:105610002596FFAF25978090540220E030E040E2CD
:1056200052E46B2F7E2F8F2F982D0F94C2261816C1
:105630000CF05CC023968FAD239724969FAD2497E2
:105640002596AFAD2597B82D898B9A8BAB8BBC8BEC
:105650008D8F9E8FAF8FB8A38DAF9EAFAFAF182D3C
:105660004090550250905602609057027090580238
:1056700020E030E040E85FE3C301B2010F94C226AE
:1056800018160CF05EC04D8A5E8A6F8A788E49A229
:105690005AA26BA27CA267C020E030E84DE953E437
:1056A000B501C6010F94841D87FF0BC0C501D6014B
:1056B0008D879E87AF87B88BADAAB9AECAAEDCAE78
:1056C0007ACF1DAA20E829AF3DE93AAF83E48CAF39
:1056D00072CF20E030E848E953E4B501C6010F94E9
:1056E000841D87FF7BCFC501D60174CF20E030E059
:1056F00040E252E4632D722D21968FAD21972296C0
:105700009FAD22970F94841D87FF15C0832D922D86
:105710002196AFAD21972296BFAD2297898B9A8BA8
:10572000AB8BBC8B8D8F9E8FAF8FB8A33DAE2EAE53
:10573000AFAF1B2F95CF1DAE1EAEA0E2AFAF12E4F0
:105740008FCF40906102509062026090630270902F
:10575000640220E030E040E85FE3C301B2010F944F
:10576000841D87FD90CF2C96EEADFFAD2C97408029
:105770005180628073802DA939AD4AAD5CADC30103
:10578000B2010F9462249B01AC01B501C6010F94D4
:10579000841D87FD3FC0A30192016DA979AD8AAD3B
:1057A0009CAD0F9461249B01AC01B701802F992D12
:1057B0000F94C226181674F12DAD3EAD4FAD512F8A
:1057C000C301B2010F9462249B01AC01632D722DC1
:1057D00021968FAD219722969FAD22970F94841D1D
:1057E00087FD18C0A30192016DAD7EAD8FAD912FE5
:1057F0000F9461249B01AC0123966FAD23972496EF
:105800007FAD249725968FAD2597982D0F94C226AE
:105810001816B4F42A96AEADBFAD2A978C9182309B
:1058200079F48DEA94E17BCE1DAE1EAEB0E2BFAF3F
:1058300012E41DAAE0E8E9AFFDE9FAAF23E42CAFDA
:105840002A96EEADFFAD2A9780818230A9F4289682
:105850009FAD28979370D1F58AE894E160CE1DAE94
:105860001EAE30E23FAF12E41DAA80E889AF9DE989
:105870009AAFA3E4ACAFE4CF2896FFAD2897F0FD34
:1058800010C04091FA0C5091FB0C6091FC0C70918F
:10589000FD0C498F5A8F6B8F7C8F4D875E876F878A
:1058A000788B28962FAD289721FD10C04091FE0CD3
:1058B0005091FF0C6091000D7091010D4D8F5E8F26
:1058C0006F8F78A3498B5A8B6B8B7C8B28963FAD5F
:1058D000289732FD10C04091020D5091030D609148
:1058E000040D7091050D49A35AA36BA37CA34D8BA6
:1058F0005E8B6F8B788F813009F461C0823009F440
:10590000A6C18CE0EAEFFCE0DE01119601900D9259
:105910008A95E1F71DA61EA61FA618AA88E0FE011B
:105920003D96DE01959601900D928A95E1F78E01E4
:105930000B5D1F4FAE01435D5F4FBE01675D7F4F43
:10594000C8010E9432C7F12CD02EE12E2796AEADB1
:10595000BFAD27978C9190E095958795F81619061D
:105960000CF026C21DA61EA61FA618AA88E0FE01DE
:105970007996AD2DBE2D01900D928A95E1F7AE017D
:10598000435D5F4FBE01675D7F4FC8010E9432C714
:105990001DA61EA61FA618AA88E0FE013D96D801E6
:1059A00001900D928A95E1F7AE01435D5F4FBE0114
:1059B000675D7F4FC8010E9432C7F394C7CF2D8522
:1059C0003E854F855889698D7A8D8B8D9C8D0F947E
:1059D00061244B015C0120E030E0A9010F94841D9B
:1059E000882309F49ECD29893A894B895C896D8D7C
:1059F0007E8D8F8D98A10F9461246B017C0120E036
:105A000030E0A9010F94841D882309F48ACD8CE02D
:105A1000EAEFFCE0DE01119601900D928A95E1F724
:105A20001DA61EA61FA618AA88E0FE013D96DE014F
:105A3000959601900D928A95E1F7AE01435D5F4F17
:105A4000BE01675D7F4FCE0185960E9432C72E96BC
:105A5000AEADBFAD2E978C91880F89AF20E030E0BE
:105A6000A901C501B4010F94C2262401350187FFA5
:105A700004C077FA709477F8709420E030E0A901C0
:105A8000C701B6010F94C22687FF76C0D701C601B1
:105A9000B0588DAB9EABAFABB8AFA30192016DA96F
:105AA0007EA98FA998AD0F94841D181614F0750166
:105AB0006401B9ADAB2FB0E0BBAFAAAFBD01BB0F66
:105AC000880B990B0F948B1D9B01AC01C701B6018C
:105AD0000F945C256B017C0100E02796EEADFFADD5
:105AE00027978081081708F057C110E0812F012EF9
:105AF000000C990B2AAD3BAD821793070CF053C0F5
:105B0000CE0149961C0110FD03C0DE011D961D014A
:105B1000612F012E000C770B880B990B0F948B1DB6
:105B2000A70196010F94EA1D4B015C01A3019201AC
:105B30006DA97EA98FA998AD0F94841D1DA21EA2E8
:105B40001FA218A6A50194011816DCF06D857E85AC
:105B50008F8598890F9462246DA77EA78FA798AB35
:105B6000B1016C5F7F4FAE014B5D5F4FCE018D96F3
:105B70000E9432C71F5FBACFCDAADEAAEFAAF8AE45
:105B80008CCF69897A898B899C890F9462246DA74F
:105B90007EA78FA798ABAE014B5D5F4FBE01635DE3
:105BA0007F4FC101E5CF19AD17FD4FC0FE017996BA
:105BB0001F0110FD04C09E01235F3F4F1901612F9B
:105BC000012E000C770B880B990B0F948B1DA701EE
:105BD00096010F94EA1D4B015C01A30192016DA98E
:105BE0007EA98FA998AD0F94841D1DA21EA21FA28D
:105BF00018A6A50194011816B4F06D857E858F85D1
:105C000098890F9462246DA77EA78FA798ABB101E6
:105C10006C5F7F4FAE014B5D5F4FCE018D960E9452
:105C200032C71150C1CF69897A898B899C890F94B9
:105C300062246DA77EA78FA798ABAE014B5D5F4F27
:105C4000BE01635D7F4FC101EACF0F5F46CF27964C
:105C5000AEADBFAD27978C91882309F462CC8CE060
:105C6000EAEFFCE0DE01119601900D928A95E1F7D2
:105C70001DA61EA61FA618AA88E0FE013D96DE01FD
:105C8000959601900D928A95E1F75E01BDE2AB0E0B
:105C9000B11C7E01E5E2EE0EF11CA501BE01675DBF
:105CA0007F4FC7010E9432C700E0DA2CCB2C3E2C7C
:105CB0002F2C2796AEADBFAD27978C91081708F013
:105CC00054C0F12CE12C19AA1AAA1BAA1CAAB701CC
:105CD0000F2C000C880B990B0F948B1D2CE739EDC2
:105CE00040E25FE30F94EA1D2B013C010F9457251E
:105CF0002C96EEADFFAD2C9780809180A280B38072
:105D0000A50194010F94EA1D2DAD3EAD4FAD512F6D
:105D10000F9462246DA77EA78FA798ABC301B20131
:105D20000F9402279B01AC01C501B4010F94EA1D39
:105D30002DA939AD4AAD5CAD0F9462246DA37EA34D
:105D40008FA398A7AE014F5C5F4F6D2D7C2D832DE7
:105D5000922D0E9432C7FFEFEF1AFF0A2AE0E216E7
:105D6000F10409F0B0CF0F5FA4CF1DA61EA61FA699
:105D700018AA88E0FE013D96DE01959601900D92ED
:105D80008A95E1F7AE01435D5F4FBE01675D7F4FCE
:105D9000CE0185960E9432C71DA21EA21FA218A680
:105DA000BE016B5D7F4FCE0101960E9412F2B9CB0E
:105DB0001DA21EA21FA218A6B801F5CF0F931F9314
:105DC0000E94C4F30091880A1091890A20918A0ADE
:105DD00030918B0A011511052105310509F067C0C5
:105DE0002091D212222309F45FC0E091D0122150F9
:105DF0002093D21221E02E0F2093D0123091D31293
:105E0000231302C01092D01224E0E29FF00111246B
:105E1000EC52FD4E00811181228133810093840A6E
:105E20001093850A2093860A3093870A600F711FAA
:105E3000811D911D6093880A7093890A80938A0A54
:105E400090938B0A8091860A9091870A892B61F141
:105E50001FB7F89489E794E10E94382A8AE00E94EB
:105E6000FF2984E096E09093FD138093FC1380EA71
:105E700090E89093FF138093FE1387E08093F013D4
:105E800082E88093F31380EA90E0A0E0B0E0809392
:105E9000F4139093F513A093F613B093F71380EADD
:105EA00093E10E947D261FBF1F910F910895601BF3
:105EB000710B820B930B97FDF7CF40981092880AD5
:105EC0001092890A10928A0A10928B0AEDCF0F93D2
:105ED0001F93CF93DF938C01EB019091D21220910D
:105EE000D312921305C00E94DE2E0E94C1CAF5CFC4
:105EF0008091D11234E0839FF0011124EC52FD4EC9
:105F000011830083D383C2839F5F9093D2128F5FEC
:105F1000281739F08093D112DF91CF911F910F9103
:105F200008951092D112F8CFCF92DF92EF92FF92A4
:105F30001F93CF93DF93182F662351F01092B8046C
:105F40001092B4041092B5041092B6041092B704E3
:105F50000E94C4F36B017C018091B4049091B5045C
:105F6000A091B604B091B704A7019601281B390B84
:105F70004A0B5B0BDA01C901B7FD3DC02091B804A3
:105F800017FD13C0412F012E000C550B4C5F5F4FC6
:105F9000822F022E000C990B4817590764F184EFE9
:105FA00091E0A0E0B0E0211724F488EE93E0A0E0B7
:105FB000B0E08C0D9D1DAE1DBF1D8093B404909369
:105FC000B504A093B604B093B7042170C22F30E09B
:105FD000D32F84E28C9FB0018D9F700D7C1B112408
:105FE00060597C4F82E390E00E94672F8091B80453
:105FF0008F5F8093B804DF91CF911F91FF90EF9056
:10600000DF90CF900895CF93DF9300D01F92CDB74C
:10601000DEB783E094E10E94382A8AE00E94FF29DB
:106020008091F70C8330D9F119821A821B821C826D
:1060300060E0CE0101960E940D1D19821A821B821A
:106040001C8261E0CE0101960E940D1D81E08093CB
:106050006B021092F40C80936C0281E09AE59093AD
:10606000FD138093FC1383E390E09093FF138093E0
:10607000FE1387E08093F01382E88093F31384E8A3
:1060800090E0A0E0B0E08093F4139093F513A09318
:10609000F613B093F71380EA93E10E947D260F90E8
:1060A0000F900F900F90DF91CF9108956F927F9294
:1060B0008F929F92AF92BF92CF92DF92EF92FF9218
:1060C0000F931F93CF93DF93CDB7DEB764970FB6CF
:1060D000F894DEBF0FBECDBF1092D0008091D000EB
:1060E00082608093D0001092D50080E18093D4002C
:1060F0008091D10080618093D1008091D10088602F
:106100008093D1008091D10080688093D1008091EC
:10611000D1008F7D8093D1008AE58093F113809325
:10612000A11385EA8093F2138093A213E0E4F4E1D3
:106130008AE1DF011D928A95E9F78091F30C8823AB
:1061400009F473C283E090E09093FD138093FC13F5
:1061500085E08093F01382E88093F3138FE190E160
:10616000A0E0B0E08093F4139093F513A093F6139E
:10617000B093F71380EA93E10E947D2684E690E0D5
:106180009093FD138093FC1305E00093F01312E845
:106190001093F31386E090E1A0E0B0E08093F41355
:1061A0009093F513A093F613B093F71380EA93E15D
:1061B0000E947D268BE090E09093FD138093FC136A
:1061C0000093F0131093F31380E092E1A0E0B0E0AD
:1061D0008093F4139093F513A093F613B093F713F1
:1061E00080EA93E10E947D261092FD131092FC1329
:1061F0000093F0131093F31384E390E1A0E0B0E078
:106200008093F4139093F513A093F613B093F713C0
:1062100080EA93E10E947D261092FD131092FC13F8
:106220000093F0131093F3138AE390E1A0E0B0E041
:106230008093F4139093F513A093F613B093F71390
:1062400080EA93E10E947D26809152129091531230
:106250009093FD138093FC130093F0131093F313AA
:1062600086E390E1A0E0B0E08093F4139093F513FF
:10627000A093F613B093F71380EA93E10E947D2672
:106280008091E8119091E9119093FD138093FC1394
:106290000093F0131093F3138CE390E1A0E0B0E0CF
:1062A0008093F4139093F513A093F613B093F71320
:1062B00080EA93E10E947D2682E090E09093FD13B6
:1062C0008093FC130093F0131093F3138EE190E18D
:1062D000A0E0B0E08093F4139093F513A093F6132D
:1062E000B093F71380EA93E10E947D2681E08093CA
:1062F0006B0270E6C72E70E1D72EE12CF12C1092C4
:10630000FD131092FC130093F0131093F313C0923B
:10631000F413D092F513E092F613F092F71380EA9B
:1063200093E10E947D26BFEFCB1ADB0AEB0AFB0A42
:10633000E4E7CE16E0E1DE06E104F10401F7CE0168
:1063400001967C0184E1D7011D928A95E9F781E0ED
:106350008F9390E99F938F939CE29F938F939F934A
:1063600084E993E09F938F93FF92EF920F94EA2733
:1063700020E630E140E050E061EA73E080EA93E13A
:106380000E94BAE42AE630E140E050E06BEA73E0B4
:1063900080EA93E10E94BAE424E730E140E050E073
:1063A000B70180EA93E10E94BAE42EE730E140E0D1
:1063B00050E067EB73E080EA93E10E94BAE4109248
:1063C000FD131092FC130093F0131093F3138EE05F
:1063D00090E1A0E0B0E08093F4139093F513A093C4
:1063E000F613B093F71380EA93E10E947D26109292
:1063F000FD131092FC130093F0131093F3138FE02E
:1064000090E1A0E0B0E08093F4139093F513A09393
:10641000F613B093F71380EA93E10E947D260FB63E
:10642000F894DEBF0FBECDBF4AE0C42E40E2D42EAA
:10643000E12CF12C55E0752E62E8662E46015701DD
:106440000AE010E01092FD131092FC137092F0130A
:106450006092F3138092F4139092F513A092F613C6
:10646000B092F71380EA93E10E947D260150110952
:10647000FFEF8F1A9F0AAF0ABF0A0115110511F726
:106480008AE0C80ED11CE11CF11C92EDC91690E205
:10649000D906E104F10491F6C12C30E2D32EE12CAF
:1064A000F12C05E012E81092FD131092FC130093FA
:1064B000F0131093F313C092F413D092F513E092FB
:1064C000F613F092F71380EA93E10E947D26109272
:1064D000FD131092FC130093F0131093F313D701E4
:1064E000C6018C529F4FAF4FBF4F8093F4139093D0
:1064F000F513A093F613B093F71380EA93E10E948B
:106500007D26AFEFCA1ADA0AEA0AFA0ABAE0CB160F
:10651000B0E2DB06E104F10431F62EEDC22E20E2FA
:10652000D22EE12CF12C05E012E81092FD1310920E
:10653000FC130093F0131093F313C092F413D09252
:10654000F513E092F613F092F71380EA93E10E94BC
:106550007D26EFEFCE1ADE0AEE0AFE0AF6EECF1621
:10656000F0E2DF06E104F10401F7CC24C39482E1F8
:10657000D82EE12CF12C9AE0A92EB12C05E012E8DE
:10658000B092FD13A092FC130093F0131093F31339
:10659000C092F413D092F513E092F613F092F71331
:1065A00080EA93E10E947D26B092FD13A092FC1335
:1065B0000093F0131093F313D701C6018096A11D29
:1065C000B11D8093F4139093F513A093F613B09339
:1065D000F71380EA93E10E947D268FEFC81AD80A4C
:1065E000E80AF80A95E1C91692E1D906E104F10436
:1065F00039F689E693E10E94382A8AE00E94FF2951
:1066000064960FB6F894DEBF0FBECDBFDF91CF9179
:106610001F910F91FF90EF90DF90CF90BF90AF90C0
:106620009F908F907F906F90089582E090E08CCD46
:106630000E9456301092590581E080936C028BE1E4
:1066400094E10E94382A8AE00C94FF290F931F934B
:10665000CF938C01C62F87E990E10E94382AC801A8
:106660000E94382A8AE30E94FF2980E38C0F0E944F
:10667000FF298AE0CF911F910F910C94FF298AE1A5
:1066800092E10E94382A60E08AE092E10E9426337B
:1066900060E085EF91E10E94263361E08EEE91E1AA
:1066A0000E94263361E083EE91E10E94263361E08F
:1066B00083ED91E10E94263360E08AEC91E10E9433
:1066C000263361E080EC91E10E94263360E086EBA6
:1066D00091E10E94263360E08FEA91E10E94263327
:1066E00060E087EA91E10E94263361E089E991E167
:1066F0000E94263361E08BE891E10E94263360E03E
:106700008CE791E10E94263360E08EE691E10E94E1
:10671000263360E088E591E10E94263361E087E45A
:1067200091E10E94263361E088E391E10E942633E3
:1067300061E081E391E10E94263360E08AE291E129
:106740000E94263361E081E291E10E94263361E0FC
:106750008CE091E10E94263361E08EEF90E10E948F
:10676000263361E08BEE90E10E94263360E08EEDEF
:1067700090E10E94263361E089ED90E10E9426338A
:1067800061E08CEC90E10E94263360E088EB90E1C0
:106790000E94263360E085EA90E10E94263360E0A3
:1067A00081E994E10E941319682F61708CE990E1EE
:1067B0000C9426330E94FF2986E09BE00C94382A33
:1067C0000F931F93CF938C01C62F88E097E00E9410
:1067D000382AC8010E94382ACC2331F08AE0CF91B0
:1067E0001F910F910C94FF29CF911F910F91089544
:1067F0000F94571010926512109246020E94A52520
:10680000882351F080918E1482FD06C08CED90E3B8
:10681000909364128093631261E082E794E10E9496
:10682000E0330C94F3D60F931F93CF93DF938C0137
:106830006F3F19F41092E31160E02091E311862F6D
:10684000062E000C990B2817190609F08CF5609399
:10685000E31160E08CE394E10E94E033C8010E9400
:10686000382A8AE00E94FF29C8010F94D11C800FAA
:10687000911FEC01C01BD10BC034D1053CF0019736
:10688000FC012491207C2038D1F3F3CFDD27AE0129
:10689000B80183EA91E10F94F21CCD55DE4E1882C7
:1068A00083EA91E1DF91CF911F910F910C944727DB
:1068B000DF91CF911F910F91089510926512109260
:1068C000460280918E14806480938E1461E08AE485
:1068D00094E10E94E0334FE554E167E674E185E01E
:1068E0000E94C7E660E081E594E10C941334CF92F6
:1068F000DF92EF92FF920F931F93CF93DF9300D01D
:106900001F92CDB7DEB77C016B018A0161E083EC99
:1069100097E00E94E0334FE554E16AEC77E085E0D0
:106920000E94C7E69091A11181E0890F8093A11187
:1069300080918E1482FF06C08B7F80938E149E5FA1
:106940009093A1110E9485D780E1EAEFFCE0ACEBC7
:10695000B4E001900D928A95E1F70E9403C2809104
:10696000BB0481110FC081E08093BB048091650B53
:106970008093B9041092650B8091660B8093BA04E2
:106980001092660B20E030E0A901F701608171816F
:10699000828193810F94841D8823F1F08091620B92
:1069A00081110CC080913A0290913B020197209195
:1069B0005212309153122817390774F080E090E09A
:1069C000A0E7B2E489839A83AB83BC83BE016F5F87
:1069D0007F4FC7010E9473C787E00E948DC5811158
:1069E00003C0B6010E94361920E030E0A901F80189
:1069F00060817181828193810F94841D882319F0B5
:106A0000C8010E9409F00E947C2581E00F900F9040
:106A10000F900F90DF91CF911F910F91FF90EF900A
:106A2000DF90CF90089560E081EE97E00E94E03320
:106A300082E197E00E94382A8AE00C94FF29EF92C5
:106A4000FF920F931F93CF937C018B01C42F60E0C3
:106A500081EE97E00E94E033C7010E94382A80E26D
:106A60000E94FF29C8010E94382ACC2319F08C2FDC
:106A70000E94FF298AE0CF911F910F91FF90EF9024
:106A80000C94FF29DF92EF92FF920F931F93CF9305
:106A9000DF93D82E7B018A01E9010E941335D09241
:106AA000661240E0B70185EF97E00E941F3501159F
:106AB000110531F040E0B8018EEE97E00E941F35DD
:106AC000209731F040E0BE018EEE97E00E941F3526
:106AD00060E081EE97E00E94E03389EE97E00E944B
:106AE000382A8AE0DF91CF911F910F91FF90EF90AC
:106AF000DF900C94FF29AF92BF92CF92DF92EF927A
:106B0000FF920F931F93CF93DF9383EF96E00E9442
:106B1000382A6091E0087091E1088091E208909134
:106B2000E30845E00E94589880EE96E00E94382ADB
:106B3000C0E0D9E0D15021F080E20E94FF29FACFD5
:106B40008C2F0E9437FACF5FC53099F78AE00E94F8
:106B5000FF290EEF1AE0C0E080E20E94FF298C2F8F
:106B60000E9437FA5801D5E080E20E94FF29F50122
:106B7000C080D180E280F380A7019601C701B601F1
:106B80000F94542781112CC020E030E0A901C701E7
:106B9000B6010F94C22687FD03C08BE20E94FF2935
:106BA00045E0C701B6010E945898D15084E1A80E73
:106BB000B11CD111D9CF8AE00E94FF29CF5F0C5FB1
:106BC0001F4FC53049F68AE0DF91CF911F910F9199
:106BD000FF90EF90DF90CF90BF90AF900C94FF2983
:106BE000F12C80E20E94FF29F3948DE3F8E0FF127C
:106BF000F9CFDBCF811107C08BE19FE00E94382ADB
:106C00008AE00C94FF298FE19FE0F8CFCF93DF93C8
:106C1000EB010E94382ACE01DF91CF910C943EFA0D
:106C2000CF93C62F0E94382A8C2FCF910C9437FA1D
:106C3000CF92DF92EF92FF926A017B010E94382A85
:106C400042E0C701B601FF90EF90DF90CF900C9427
:106C50005898CF92DF92EF92FF926A017B010E94D7
:106C6000382A4AE0C701B601FF90EF90DF90CF903D
:106C70000C94172ACF93DF93EB010E94382ACE01A0
:106C8000DF91CF910C940DE54F925F926F927F92BE
:106C90008F929F92AF92BF92CF92DF92EF92FF922C
:106CA0000F931F93CF93DF9300D000D01F921F92BA
:106CB000CDB7DEB78091580581110AC48091560581
:106CC000909157059C012F5F3F4F309357052093BC
:106CD00056058E3E924008F4FBC38091521290916B
:106CE00053129093FD138093FC1305E00093F0136F
:106CF00012E81093F31386E390E1A0E0B0E08093F4
:106D0000F4139093F513A093F613B093F71380EA5E
:106D100093E10E947D268091E8119091E911909372
:106D2000FD138093FC130093F0131093F3138CE383
:106D300090E1A0E0B0E08093F4139093F513A0935A
:106D4000F613B093F71380EA93E10E947D268091B9
:106D50005412909155129093FD138093FC1300935D
:106D6000F0131093F31384E390E1A0E0B0E080937C
:106D7000F4139093F513A093F613B093F71380EAEE
:106D800093E10E947D268091EA119091EB119093FE
:106D9000FD138093FC130093F0131093F3138AE315
:106DA00090E1A0E0B0E08093F4139093F513A093EA
:106DB000F613B093F71380EA93E10E947D2681E0F9
:106DC0008093580510925705109256058091F70C44
:106DD000882339F10E94A518811123C0809155059F
:106DE0008F5F8093550580915505853620F0109270
:106DF00055051092F70CE091F70CE150E73008F0E0
:106E00006AC00E2E000CFF0B8827E65FF84C8F4FF0
:106E10000D944D24143763372F395B399C39D4399D
:106E2000673710925505DFCF0E94C11D882309F4F2
:106E300052C081E080936C0285EF93E10E94382A72
:106E40008AE00E94FF2980E190E09093FD138093F7
:106E5000FC1385E08093F01312E81093F31384E1A0
:106E600090E1A0E0B0E08093F4139093F513A09329
:106E7000F613B093F71380EA93E10E947D2681E038
:106E80009AE59093FD138093FC1386E390E0909332
:106E9000FF138093FE1387E08093F0131093F31396
:106EA00084E890E0A0E0B0E08093F4139093F513B1
:106EB000A093F613B093F71380EA93E10E947D2626
:106EC0001092F70C08C00E94C11D882321F00E9477
:106ED000A5188823A9F380916C02882309F4D8C6E9
:106EE000809159058111C0C284E096E09093FD1312
:106EF0008093FC1380EA90E89093FF138093FE1335
:106F000017E01093F01302E80093F31380EA90E087
:106F1000A0E0B0E08093F4139093F513A093F613E0
:106F2000B093F71380EA93E10E947D268091670277
:106F300090916802A0916902B0916A020097A10540
:106F4000B10509F03FC21092FD131092FC1315E039
:106F50001093F0130093F3138AE890E1A0E0B0E0FF
:106F60008093F4139093F513A093F613B093F71353
:106F700080EA93E10E947D2689E090E09093FD13E2
:106F80008093FC131093F0130093F3138CE890E1BB
:106F9000A0E0B0E08093F4139093F513A093F61360
:106FA000B093F71380EA93E10E947D2680916702F7
:106FB00090916802A0916902B0916A020097F1E095
:106FC000AF07B10508F441C2B093FD13A093FC13C1
:106FD0009093FF138093FE1387E08093F01382E871
:106FE0008093F31388E890E1A0E0B0E08093F4137D
:106FF0009093F513A093F613B093F71380EA93E1FF
:107000000E947D268091670290916802A09169029A
:10701000B0916A02BA2FA92F982F8827009721E0F4
:10702000A207B10508F417C2B093FD13A093FC1397
:107030009093FF138093FE1387E08093F01312E880
:107040001093F31381EA90E0A0E0B0E08093F41392
:107050009093F513A093F613B093F71380EA93E19E
:107060000E947D268091F90C882309F4FAC183E0FF
:1070700090E09093FD138093FC1385E08093F013D0
:107080001093F31385E490E1A0E0B0E08093F41353
:107090009093F513A093F613B093F71380EA93E15E
:1070A0000E947D2680915905875E80935905209125
:1070B0005905822F90E0253608F021C29093FD13E8
:1070C0008093FC1385E08093F01382E88093F313A0
:1070D00080E090E1A0E0B0E08093F4139093F5138A
:1070E000A093F613B093F71380EA93E10E947D26F4
:1070F0000E94A518811114C20E94A525811105C006
:1071000090915C0591FD0E94A51890915C0580FB13
:1071100091F990935C0591FD03C280918E1482FDDC
:10712000FFC18091A2118150823008F4F9C16091B1
:10713000EA117091EB11072E000C880B990B0F943C
:107140008B1D6B017C0120E030E0A9010F94841DB0
:10715000882309F460C66091E8117091E911072E47
:10716000000C880B990B0F948B1D2B013C0120E028
:1071700030E040E050E4C701B6010F946124A30160
:1071800092010F94C22618160CF467C66091521231
:1071900070915312072E000C880B990B0F948B1DC6
:1071A0006D837E838F8398876091541270915512FE
:1071B000072E000C880B990B0F948B1D4B015C0163
:1071C00020E030E040E251E40F9461242D813E81C3
:1071D0004F8158850F94C22618160CF43EC620E045
:1071E00030E040E050E4C701B6010F946224A301EF
:1071F00092010F94841D87FD10C020E030E040E232
:1072000051E4C501B4010F9462242D813E814F8168
:1072100058850F94841D87FF0FC684E190E09093FA
:10722000FD138093FC1385E08093F01382E8809334
:10723000F31384E190E1A0E0B0E08093F413909325
:10724000F513A093F613B093F71380EA93E10E942D
:107250007D268091F50C811121C682E01FC687EE44
:1072600093E10E94382A8AE00E94FF2981E09AE592
:107270009093FD138093FC1380E490E09093FF13B0
:107280008093FE1317E01093F01382E88093F313BA
:1072900084E890E0A0E0B0E08093F4139093F513BD
:1072A000A093F613B093F71380EA93E10E947D2632
:1072B0001093F70C10CE8091E60C882309F40BCEC6
:1072C0000E94C11D882309F406CE0E94A5188111D1
:1072D00002CE89ED93E10E94382A8AE00E94FF29BC
:1072E0008091E70C90E0B0E0A0E0895B9F4FAE4F4B
:1072F000B54A21E03AE53093FD132093FC139093B7
:10730000FF138093FE1387E08093F01382E880934D
:10731000F31384E890E0A0E0B0E08093F41390933E
:10732000F513A093F613B093F71380EA93E10E944C
:107330007D261092E60CC4CD0E94C11D882309F45D
:10734000CACD0E94A5188111C6CD81E080936C0240
:107350001092F70C8BEC93E10E94382A8AE00E948D
:10736000FF2981E09AE59093FD138093FC138EE44E
:1073700090E09093FF138093FE1387E08093F013C7
:1073800082E88093F31384E890E0A0E0B0E080937B
:10739000F4139093F513A093F613B093F71380EAC8
:1073A00093E10E947D2697CD0E94A518811193CD6F
:1073B00019821A821B821C8262E0CE0101960E9411
:1073C000A5EB7ECD0196A11DB11D35E0B695A79523
:1073D000979587953A95D1F70197A109B10900973B
:1073E000E1E0AE07B10548F1B093FD13A093FC13A3
:1073F0009093FF138093FE131093F01312E81093F1
:10740000F3138AE890E1A0E0B0E08093F413909346
:10741000F513A093F613B093F71380EA93E10E945B
:107420007D2688E090E09093FD138093FC1385E027
:107430008093F0131093F313A9CD9093FD138093D1
:10744000FC1385E08093F013D9CF9093FD138093C4
:10745000FC1385E0C2CD9093FD138093FC1385E06F
:10746000ECCD82E090E005CE8A3F08F020CE8EEF92
:10747000809359058AEB93E10E94382A8AE00E94A2
:10748000FF2981E080936C0281E09AE59093FD13DF
:107490008093FC138DE290E09093FF138093FE1392
:1074A00087E08093F01382E88093F31384E890E000
:1074B000A0E0B0E08093F4139093F513A093F6133B
:1074C000B093F71380EA93E10E947D26109258054D
:1074D00028960FB6F894DEBF0FBECDBFDF91CF91D7
:1074E0001F910F91FF90EF90DF90CF90BF90AF90E2
:1074F0009F908F907F906F905F904F9008958456EB
:1075000091099093FD138093FC1385E08093F01311
:1075100082E88093F31381E090E1A0E0B0E0DCCD5D
:107520008CE090E09093FD138093FC1315E0109392
:10753000F01382E88093F31384E190E1A0E0B0E0DF
:107540008093F4139093F513A093F613B093F7136D
:1075500080EA93E10E947D260E942FD620E13EE042
:1075600040E050E00F94C8232115310581E0480721
:10757000510508F470C05093FD134093FC133093F1
:10758000FF132093FE1387E08093F01312E810930B
:10759000F31380E190E1A0E0B0E08093F4139093C6
:1075A000F513A093F613B093F71380EA93E10E94CA
:1075B0007D260E942FD620E13EE040E050E00F946F
:1075C000C8232CE330E040E050E00F94C823309310
:1075D000FD132093FC1305E00093F0131093F313B5
:1075E00082E190E1A0E0B0E08093F4139093F51372
:1075F000A093F613B093F71380EA93E10E947D26DF
:107600000E94B325882309F401C48F5F8093540539
:10761000E82EF12C833330F5EE0CFF1CF092FD13B5
:10762000E092FC130093F0131093F3138EE090E1BB
:10763000A0E0B0E08093F4139093F513A093F613B9
:10764000B093F71380EA93E10E947D261092FD1318
:107650001092FC132BC03093FD132093FC13109356
:10766000F01394CF84E690E09093FD138093FC1385
:107670000093F0131093F3138EE090E1A0E0B0E0DC
:107680008093F4139093F513A093F613B093F7132C
:1076900080EA93E10E947D26A2E3EA1AA0E8FA0AB2
:1076A000EE0CFF1CF092FD13E092FC130093F0131C
:1076B0001093F3138FE090E1A0E0B0E08093F41317
:1076C0009093F513A093F613B093F71380EA93E128
:1076D0000E947D260E94B32590E09093FD13809335
:1076E000FC1385E08093F01382E88093F31386E126
:1076F00090E1A0E0B0E08093F4139093F513A09391
:10770000F613B093F71380EA93E10E947D260E945E
:10771000C91D20E030E048EC52E40F94EA1D0F94BC
:10772000CE257093FD136093FC1305E00093F013D6
:1077300012E81093F31386E290E1A0E0B0E08093AA
:10774000F4139093F513A093F613B093F71380EA14
:1077500093E10E947D2680913602909137029093AA
:10776000FD138093FC130093F0131093F31380E048
:1077700093E1A0E0B0E08093F4139093F513A0930D
:10778000F613B093F71380EA93E10E947D2620E080
:1077900030E040E251E46091AC0C7091AD0C80910E
:1077A000AE0C9091AF0C0F94EA1D0F94D5257093F9
:1077B000FD136093FC130093F0131093F31382E412
:1077C00092E1A0E0B0E08093F4139093F513A093BE
:1077D000F613B093F71380EA93E10E947D2620E030
:1077E00030E040E251E46091B00C7091B10C8091B6
:1077F000B20C9091B30C0F94EA1D0F94D5257093A1
:10780000FD136093FC130093F0131093F31386E4BD
:1078100092E1A0E0B0E08093F4139093F513A0936D
:10782000F613B093F71380EA93E10E947D2620E0DF
:1078300030E040E251E46091B40C7091B50C80915D
:10784000B60C9091B70C0F94EA1D0F94D525709348
:10785000FD136093FC130093F0131093F3138AE469
:1078600092E1A0E0B0E08093F4139093F513A0931D
:10787000F613B093F71380EA93E10E947D2620E08F
:1078800030E040E251E46091B80C7091B90C809105
:10789000BA0C9091BB0C0F94EA1D0F94D5257093F0
:1078A000FD136093FC130093F0131093F3138EE415
:1078B00092E1A0E0B0E08093F4139093F513A093CD
:1078C000F613B093F71380EA93E10E947D2680912E
:1078D0007302909174029093FD138093FC130093B4
:1078E000F0131093F31382E592E1A0E0B0E08093EF
:1078F000F4139093F513A093F613B093F71380EA63
:1079000093E10E947D268091710290917202909382
:10791000FD138093FC130093F0131093F31384E58D
:1079200092E1A0E0B0E08093F4139093F513A0935C
:10793000F613B093F71380EA93E10E947D2620E0CE
:1079400030E040E251E460915712709158128091FA
:10795000591290915A120F94EA1D0F94D5257093E5
:10796000FD136093FC130093F0131093F31386E55B
:1079700092E1A0E0B0E08093F4139093F513A0930C
:10798000F613B093F71380EA93E10E947D262CEA68
:1079900035EC47E25EE360915B1270915C1280917E
:1079A0005D1290915E120F945C2520E030E040E281
:1079B00051E40F94EA1D0F94D5257093FD13609345
:1079C000FC130093F0131093F3138AE592E1A0E007
:1079D000B0E08093F4139093F513A093F613B09353
:1079E000F71380EA93E10E947D262CEA35EC47E20A
:1079F0005EE360915F1270916012809161129091CC
:107A000062120F94EA1D20E030E040E251E40F944E
:107A1000EA1D0F94D5257093FD136093FC1300931A
:107A2000F0131093F3138EE592E1A0E0B0E08093A1
:107A3000F4139093F513A093F613B093F71380EA21
:107A400093E10E947D2620E030E040E251E4609125
:107A5000ED117091EE118091EF119091F0110F9452
:107A6000EA1D0F94D5257093FD136093FC130093CA
:107A7000F0131093F31382E692E1A0E0B0E080935C
:107A8000F4139093F513A093F613B093F71380EAD1
:107A900093E10E947D262CEA35EC47E25EE360919B
:107AA000F1117091F2118091F3119091F4110F94F2
:107AB0005C2520E030E040E251E40F94EA1D0F9491
:107AC000D5257093FD136093FC130093F01310936E
:107AD000F31386E692E1A0E0B0E08093F413909374
:107AE000F513A093F613B093F71380EA93E10E9485
:107AF0007D262CEA35EC47E25EE36091F51170914A
:107B0000F6118091F7119091F8110F94EA1D20E081
:107B100030E040E251E40F94EA1D0F94D5257093B4
:107B2000FD136093FC130093F0131093F3138AE694
:107B300092E1A0E0B0E08093F4139093F513A0934A
:107B4000F613B093F71380EA93E10E947D268091AB
:107B5000F00C811105C08091F20C882309F46DC0EE
:107B60006091521270915312072E000C880B990BE2
:107B70000F948B1D20E030E048EC52E40F94EA1D96
:107B80006B017C016091541270915512072E000C0C
:107B9000880B990B0F948B1D9B01AC01C701B6019B
:107BA0000F945C250F94D5256536710510F064E6B9
:107BB00070E07093FD136093FC1305E00093F013E5
:107BC00012E81093F31384E290E1A0E0B0E0809318
:107BD000F4139093F513A093F613B093F71380EA80
:107BE00093E10E947D266091521270915312072EEC
:107BF000000C880B990B0F948B1D6B017C0120E00E
:107C000030E04AE253E40F94C226181624F480911F
:107C1000F00C811146C16091541270915512072EDB
:107C2000000C880B990B0F948B1D9B01AC01C701B5
:107C3000B6010F94C22687FFAFC18091E60C88235E
:107C400039F18091E50C91E0980F9093E50C90E06C
:107C50009093FD138093FC1385E08093F01382E8EA
:107C60008093F31382E490E1A0E0B0E08093F413FA
:107C70009093F513A093F613B093F71380EA93E172
:107C80000E947D268091E50C8A3010F01092E50C60
:107C90000E944B1D882309F4B5C16091E00C7091DE
:107CA000E10CEE24E394F12C61157105A9F090E04C
:107CB00080E00F94891D20E030E040E85EE30F94FF
:107CC000EA1D0F94402520E030E040E85FE30F9488
:107CD00062240F94D5257B0101E010E08091E20C35
:107CE000811102C010E000E08091E4129091E51251
:107CF0008F3F980711F40E945A929093E512809357
:107D0000E412080F191FB80190E080E00F94891D5C
:107D100020E030E040E85EE30F94EA1D0F94402538
:107D20004B015C01F092FD13E092FC1305E000931F
:107D3000F01312E81093F31380E193E1A0E0B0E0B8
:107D40008093F4139093F513A093F613B093F71365
:107D500080EA93E10E947D26C501B4010F94D525E8
:107D60007093FD136093FC130093F0131093F313BF
:107D700082E193E1A0E0B0E08093F4139093F513D7
:107D8000A093F613B093F71380EA93E10E947D2647
:107D900000E414E1AAE1FA2E8091100590911105FA
:107DA0002091520530915305891B8F7309F449C105
:107DB0002A3131050CF0DBC190911005809111053D
:107DC0004FEF5FEF981749F0E82FF0E0E05FFA4FD0
:107DD00042818F5F8F7380931105F901E05CFB4E48
:107DE0004083809140148A3509F0B3C162E070E0AD
:107DF00080E090E00E9461258091520590915305AA
:107E000001969093530580935205C6CF1092FD13AF
:107E10001092FC1307CC6091541270915512072EEA
:107E2000000C880B990B0F948B1D20E030E0A9010A
:107E30000F94841D81118FC98CE090E09093FD1305
:107E40008093FC1385E08093F01382E88093F31312
:107E500084E190E1A0E0B0E04ECC8DE090E0909322
:107E6000FD138093FC1385E08093F01382E88093E8
:107E7000F31384E190E1A0E0B0E08093F4139093D9
:107E8000F513A093F613B093F71380EA93E10E94E1
:107E90007D268091F50C811101C081E08093F50C65
:107EA00036CC1092F00C20E030E040E251E46091DA
:107EB000E80C7091E90C8091EA0C9091EB0C0F9416
:107EC000EA1D0F94CE257093FD136093FC1300936D
:107ED000F0131093F31384E590E1A0E0B0E08093F9
:107EE000F4139093F513A093F613B093F71380EA6D
:107EF00093E10E947D2620E030E040E251E4609171
:107F0000EC0C7091ED0C8091EE0C9091EF0C0F94B5
:107F1000EA1D0F94CE257093FD136093FC1300931C
:107F2000F0131093F31388E590E1A0E0B0E08093A4
:107F3000F4139093F513A093F613B093F71380EA1C
:107F400093E10E947D2689E993E10E94382A8AE024
:107F50000E94FF2981E09AE59093FD138093FC1322
:107F600081E490E09093FF138093FE1387E0809369
:107F7000F0131093F31384E890E0A0E0B0E0809356
:107F8000F4139093F513A093F613B093F71380EACC
:107F900093E10E947D2651CE6091F20C662309F494
:107FA0004CCE062E000C770B80E893E10E943A3607
:107FB0008AE00E94FF291092F20C84E090E09093F6
:107FC000FD138093FC1385E08093F01312E8109367
:107FD000F3138EE890E1A0E0B0E08093F413909367
:107FE000F513A093F613B093F71380EA93E10E9480
:107FF0007D2681E09AE59093FD138093FC1383E541
:1080000090E0B0CF1092FD131092FC1305E00093A6
:10801000F01312E81093F31380E193E1A0E0B0E0D5
:108020008093F4139093F513A093F613B093F71382
:1080300080EA93E10E947D261092FD131092FC13BA
:1080400093CE121613060CF492C08091A413909153
:10805000A513A091A613B091A7138C34E0E19E075D
:10806000A105B10509F432CA8A349041A105B105D0
:1080700009F42CCA20E030E040E251E46091FA0CAF
:108080007091FB0C8091FC0C9091FD0C0F94EA1DFB
:108090000F94CE257093FD136093FC1305E00093BD
:1080A000F01312E81093F31388E490E1A0E0B0E03D
:1080B0008093F4139093F513A093F613B093F713F2
:1080C00080EA93E10E947D2620E030E040E251E426
:1080D0006091FE0C7091FF0C8091000D9091010D4C
:1080E0000F94EA1D0F94CE257093FD136093FC133B
:1080F0000093F0131093F3138AE490E1A0E0B0E052
:108100008093F4139093F513A093F613B093F713A1
:1081100080EA93E10E947D2620E030E040E251E4D5
:108120006091020D7091030D8091040D9091050DE9
:108130000F94EA1D0F94CE257093FD136093FC13EA
:108140000093F0131093F3138CE490E1A0E0B0E0FF
:10815000B1C9121613060CF01FCEF8012F2D119283
:108160002A95E9F7109253051092520515CE909179
:10817000A11380914014981321C09091A213809173
:10818000411498131BC023303105C4F09091421460
:108190009093A013809143148093A3139330D1F450
:1081A000982F9D7F9038B1F4909144149F3409F03A
:1081B00059C0909145149B3409F054C0E0E4F4E1B7
:1081C0008AE1DF011D928A95E9F71092530510921A
:1081D00052053BCF833809F045C0809144149091FB
:1081E0004514982789279827B0E0A0E08093A4132E
:1081F0009093A513A093A613B093A713C090461411
:10820000D12CF12CE12CC092A813D092A913E092AA
:10821000AA13F092AB1327E434E140E050E0BA0136
:108220004C155D056E057F0508F04AC0DB01CA01EB
:10823000B695A795979587950696880F991FFC0187
:10824000E056FC4ED9018C9111969C918927982774
:108250008927918380834E5F5F4F6F4F7F4F2E5FE3
:108260003F4FDECF813861F58091441490E0B0E05B
:10827000A0E08093A4139093A513A093A613B093AA
:10828000A71380914514482F50E070E060E04093C0
:10829000A8135093A9136093AA137093AB13A6E489
:1082A000B4E1ECEAF3E190E030E020E082179307DC
:1082B00039F04D9150E0419351932F5F3F4FF6CFEE
:1082C000E0E4F4E18AE1DF011D928A95E9F710927A
:1082D0005305109252050E9444FAB7CE8111B0C0E6
:1082E00084E49CE00E94382A40910E0950910F09C5
:1082F00060911009709111098CE69CE00E9418367B
:108300004091160950911709609118097091190947
:108310008CEA9BE20E941836409112095091130991
:10832000609114097091150985EB9BE20E94183643
:1083300060911A0970911B09072E000C880B990B8C
:108340000F948B1DAB01BC018FEA9BE20E94183693
:1083500060911C0970911D09072E000C880B990B68
:108360000F948B1DAB01BC0189E69CE00E9418367E
:1083700060911E0970911F09072E000C880B990B44
:108380000F948B1DAB01BC0186E69CE00E94183661
:10839000609122097091230983E69CE00E943A369D
:1083A000609124097091250980E69CE00E943A368C
:1083B00060913E0970E08DE59CE00E943A36609144
:1083C0003D0970E090E080E00F94891DAB01BC0195
:1083D0008AE59CE00E9418366091260970E090E0E2
:1083E00080E00F94891DAB01BC0187E59CE00E94F1
:1083F00018364091270950912809609129097091F8
:108400002A098FE79AE10E94183640912B09509172
:108410002C0960912D0970912E098BEB9BE20E9433
:10842000183640912F0950913009609131097091AF
:10843000320988EB9BE20E9418368AE00C94FF29EF
:1084400080E59CE04FCF8F929F92AF92BF92CF92E8
:10845000DF92EF92FF920F931F93CF93DF9300D0A1
:1084600000D01F921F92CDB7DEB781E50E94B222E5
:10847000882309F464C120E030E0A9016091120969
:108480007091130980911409909115090F94C226D7
:1084900018160CF041C18091620B81110DC08091C2
:1084A0003A0290913B02019720915412309155125B
:1084B000281739070CF430C180E1EAEFFCE0A5EEA3
:1084C000BAE001900D928A95E1F7809133098770A7
:1084D000F12C873009F089C0F0902609FF2009F4BB
:1084E00084C020912F093091300940913109509179
:1084F00032096091020D7091030D8091040D9091ED
:10850000050D0F9462246093020D7093030D809308
:10851000040D9093050D8090610290906202A090EE
:108520006302B0906402A50194010F94C22618164C
:1085300044F48092020D9092030DA092040DB0922B
:10854000050D20E030E040E05FE36091C40C7091E5
:10855000C50C8091C60C9091C70C0F94EA1D6983DD
:108560007A838B839C83CE0101960E945BC60E9416
:1085700003C28091270990912809A0912909B091FF
:108580002A098093FA0C9093FB0CA093FC0CB093F7
:10859000FD0C80912B0990912C09A0912D09B0918F
:1085A0002E098093FE0C9093FF0CA093000DB093C6
:1085B000010DE090F80C80E090E0A8ECB2E4898333
:1085C0009A83AB83BC83A12CB12C65018E010F5F14
:1085D0001F4F26E03DE042E05DE06EEF7CE08AEF79
:1085E0009CE00E944AC40E9403C260911A097091E3
:1085F0001B09072E000C880B990B0F948B1D20E094
:1086000030E040E752E40F945C256D837E838F83D6
:1086100098872091120930911309409114095091C3
:10862000150960910E0970910F09809110099091C0
:1086300011090F94622469837A838B839C83BE0122
:108640006B5F7F4FCE0101960E9473C7FF2021F11F
:108650008091FE0C9091FF0CA091000DB091010D46
:108660004091FA0C5091FB0C6091FC0C7091FD0C48
:108670004093E50A5093E60A6093E70A7093E80A8C
:108680008093E90A9093EA0AA093EB0AB093EC0A6C
:1086900084EC9CE00E94C1D160911E0970911F0979
:1086A000072E000C880B990B0F948B1D20E030E0F7
:1086B00040E752E40F945C256D837E838F83988717
:1086C00020E030E0A90160911609709117098091AE
:1086D0001809909119090F94622469837A838B8316
:1086E0009C83BE016B5F7F4FCE0101960E9473C7D2
:1086F0008091F10A9091F20AA091F30AB091F40AE4
:108700008093060D9093070DA093080DB093090D6B
:1087100086E09DE00E9414C228960FB6F894DEBF52
:108720000FBECDBFDF91CF911F910F91FF90EF90C2
:10873000DF90CF90BF90AF909F908F90089583E58A
:108740000E9400238823F1F00E9488226B017C01A3
:1087500020E030E0A9010F94841D87FD3FC120E097
:1087600030E84BE354E4C701B6010F94C226181653
:108770000CF438C1C0920E09D0920F09E092100992
:10878000F092110982E40E9400238823F9F00E94EC
:1087900088226B017C0120E030E040E251EC0F9434
:1087A000841D87FD27C120E030E040E251E4C7018D
:1087B000B6010F94C22618160CF423C1C0921609F4
:1087C000D0921709E0921809F092190985E40E94E5
:1087D00000238823F1F00E9488226B017C0120E0B5
:1087E00030E0A9010F94841D87FD12C120E030E81C
:1087F0004BE354E4C701B6010F94C22618160CF4DB
:108800000BC1C0921209D0921309E0921409F092A0
:10881000150980E50E940023882399F00E94882290
:108820000F94CE25693185E1780714F068E175E190
:108830006A30710514F46AE070E070931B0960936C
:108840001A0982E50E940023882399F00E94882259
:108850000F94CE25693185E1780714F068E175E160
:108860006A30710514F46AE070E070931D0960933A
:108870001C0985E50E940023882399F00E94882224
:108880000F94CE25693185E1780714F068E175E130
:108890006A30710514F46AE070E070931F09609308
:1088A0001E0987E50E940023882369F00E94882220
:1088B00011E020E030E0A9010F94841D811101C076
:1088C00010E01093260988E50E9400238823D1F048
:1088D0000E9488220F94CE2577FDA6C06C3381E0DC
:1088E000780714F06BE371E0072E000C880B990BEE
:1088F0000F948B1D60932709709328098093290991
:1089000090932A0989E50E9400238823D1F00E94D0
:1089100088220F94CE2577FD8BC0653381E07807E0
:1089200014F064E371E0072E000C880B990B0F9490
:108930008B1D60932B0970932C0980932D099093C4
:108940002E098AE50E940023882351F00E94882284
:1089500060932F0970933009809331099093320905
:1089600010923C098CE40E940023882379F00E9435
:1089700084228230910550F480933D0991E020914A
:10898000F80C281708F090E090933E0981E40E94CB
:10899000B222882321F00E94FD1C80933E0984E5C9
:1089A0000E94B222882309F449C08091D504909195
:1089B000D604892B09F446C00E9484228230910596
:1089C000D8F52091F80C28171906B1F18F5F809324
:1089D0003C090E943ECA10923C099ECEC12CD12C6B
:1089E0007601C8CEC12C30E8D32E3BE3E32E34E42D
:1089F000F32EC0CEC12CD12C20E2E22E21ECF22E9F
:108A0000DDCEC12CD12C90E2E92E91E4F92ED6CE08
:108A1000C12CD12C7601F5CEC12C80E8D82E8BE369
:108A2000E82E84E4F82EEDCE60E070E0CB0162CF5A
:108A300060E070E0CB017DCF10923C0980E00E94A5
:108A40006E416ACE0E943ECA67CE2F923F924F92ED
:108A50005F926F927F928F929F92AF92BF92CF92CE
:108A6000DF92EF92FF920F931F93CF93DF93CDB7D7
:108A7000DEB7C058D1090FB6F894DEBF0FBECDBF28
:108A800081E99AE00E94382A0F94861081116EC005
:108A900084E50E940023882329F00E94842260E05C
:108AA0000E94A2C780E090E0A0E8BFE389839A8398
:108AB000AB83BC838D839E83AF83B8878DEC9CECA6
:108AC000ACE4BEE389879A87AB87BC8780E090E0FF
:108AD000A0E2B1E48D879E87AF87B88B8CE390E0EE
:108AE0009A8B898B8DEC90E09C8B8B8B8DEC9CEC26
:108AF000ACECBEE38D8B9E8BAF8BB88F80E090E0AB
:108B0000A0EEBFE3898F9A8FAB8FBC8F1BA61CA6EC
:108B10004AE959E969E97EE38FE40E9436236D8FC3
:108B20007E8F8F8F98A360E083E40E947A2489A3CC
:108B300060E08BE40E947A248AA382E40E940023EE
:108B4000882381F10E948422009761F19C012852C0
:108B500031092536310520F16CE870E083E69AE0B2
:108B60000E943A368EE59AE00E94382AC058DF4FBC
:108B70000FB6F894DEBF0FBECDBFDF91CF911F912E
:108B80000F91FF90EF90DF90CF90BF90AF909F90AC
:108B90008F907F906F905F904F903F902F900895AF
:108BA0009A8B898B8CE40E9400238823E1F00E9439
:108BB00088226B017C01C986DA86EB86FC8620E080
:108BC00030E0A9010F94C22687FD0AC020E030E002
:108BD00040E050E4C701B6010F94841D18161CF440
:108BE00086E39AE0C1CF81E50E94B222882331F169
:108BF0008091D5049091D604892BE9F00E948822B7
:108C00006B017C01CD82DE82EF82F8862DEC3CEC9C
:108C10004CE45DE30F94C22687FD0AC020E030E0FB
:108C200040E751E4C701B6010F94841D181634F4CF
:108C300085E09AE099CF8AED99E096CF83E50E948E
:108C400000238823E9F00E9488226B017C01CD8AF1
:108C5000DE8AEF8AF88E2DEC3CEC4CEC5DE30F9451
:108C6000C22687FD0AC020E030E040E050E4C701A2
:108C7000B6010F94841D18161CF483EB99E074CF91
:108C800080E50E94B222882341F18091D504909121
:108C9000D604892B19F48BE799E066CF8BA58F5FFB
:108CA0008BA70E9488226B017C01CD86DE86EF8631
:108CB000F88A20E030E0A9010F94C22687FD0AC09F
:108CC00020E030E048EC51E4C701B6010F94841D68
:108CD00018161CF483E599E047CF86E40E94002330
:108CE0008823E9F00E9488226B017C01C98EDA8E0C
:108CF000EB8EFC8E20E030E040E85FE30F94C2266C
:108D000087FD0AC020E030E040E850E4C701B6012A
:108D10000F94841D18161CF48AE299E025CFC98CA3
:108D2000DA8CEB8CFC8C8D889E88AF88B88CA70180
:108D30009601C701B6010F94EA1D9B01AC0160E0EA
:108D400070E084E490E40F945C2529813A814B81A2
:108D50005C810F94EA1D2B013C01A5019401C50122
:108D6000B4010F94EA1DA70196010F94EA1D2CEEA1
:108D700031E548EB5DE30F945C259B01AC01C30139
:108D8000B2010F94EA1D69837A838B839C8388E404
:108D90000E940023882379F00E948422009759F0D2
:108DA0009C01255A31092F30314018F08CEF98E0A2
:108DB000DBCE9C8B8B8B85E50E94B2228823C9F089
:108DC0000E94C4F3611571058105910511F00F949E
:108DD0000A198091D5049091D604892B91F00E94B4
:108DE00088226093D1047093D2048093D30490932B
:108DF000D40482E50E94B222811108C088EC98E078
:108E0000B3CE60E070E088E492E4EBCF8091D504CB
:108E10009091D604892B61F00E948422E5969FAF41
:108E20008EAFE597181619064CF084E998E09CCEB1
:108E30008AE190E0E5969FAF8EAFE59789E50E94C5
:108E40000023882309F4BEC00E94882220914F0C81
:108E50003091500C4091510C5091520C0F94612460
:108E60004B015C0188E50E940023882309F4B3C00C
:108E70000E94882220914B0C30914C0C40914D0C5B
:108E800050914E0C0F9461246B017C01CBA2DCA2AB
:108E9000EDA2FEA28FA298A6A9A6BAA627E137EB5B
:108EA00041ED58EBC501B4010F94C22687FD9CC06B
:108EB00023E030E04AE953E4C501B4010F94841D76
:108EC00018160CF491C027E137EB41ED58EBC701C0
:108ED000B6010F94C22687FD87C023E030E84DE934
:108EE00053E4C701B6010F94841D18160CF47CC01E
:108EF00084E40E94B22291E089270E94DD2480E070
:108F000090E0A0EAB0E48DA79EA7AFA7B8ABCE01D2
:108F10008D960E9497F190916F0BEC969FAFEC9716
:108F200010926F0B0E94AEC489E498E00E94382A28
:108F300089899A898A3191050CF059C08B899C895D
:108F40000E9485C161E08091F80C0E94E79A81112E
:108F500056C06FEF8EE598E00E9413348CA5811106
:108F600004C0CE0101960E94F2F180E090E0A0EAF8
:108F7000B0E48093ED0A9093EE0AA093EF0AB093C9
:108F8000F00A1DA61EA61FA618AABE01635D7F4F8C
:108F900085EE9AE00E94AF1FEC965FADEC97509380
:108FA0006F0B0E94AEC48AA18111E0CD1092EB112B
:108FB0001092EA110E949F9C8091F80C90E00E9410
:108FC00085C1D4CD8090FE0C9090FF0CA090000D38
:108FD000B090010D47CFC090FA0CD090FB0CE09000
:108FE000FC0CF090FD0C52CF8AE698E0BDCD0E94BB
:108FF000161A81E00E946F998111A0CFAACF10921A
:10900000060D1092070D1092080D1092090D86E0C2
:109010009DE00E9414C28BA5882309F452C020E071
:1090200030E040E751E46091C80C7091C90C809128
:10903000CA0C9091CB0C0F945C256DA77EA78FA7CF
:1090400098AB80E1EAEFFCE0A5EEBAE001900D926A
:109050008A95E1F72D853E854F8558896091F10A03
:109060007091F20A8091F30A9091F40A0F946224AD
:109070006093F10A7093F20A8093F30A9093F40AD2
:10908000CE018D960E94C1D12D853E854F85588990
:109090006091F10A7091F20A8091F30A9091F40ABA
:1090A0000F9461246093F10A7093F20A8093F30A9B
:1090B0009093F40A8CA5811104C0CE0101960E9400
:1090C000F2F1ECECF4E085E0DF011D928A95E9F71E
:1090D00080E1EAEFFCE0A5EEBAE001900D928A95FE
:1090E000E1F789859A85AB85BC858093ED0A9093DD
:1090F000EE0AA093EF0AB093F00A1DA61EA61FA6C3
:1091000018AABE01635D7F4F85EE9AE00E94AF1FF3
:10911000BE01635E7F4F85EE9AE00E94AF1F89A17A
:10912000882309F4F5C32091FA0C3091FB0C40918F
:10913000FC0C5091FD0CE0962CAF3DAF4EAF5FAFF5
:10914000E0978091FE0C9091FF0CA091000DB091E2
:10915000010DAC968CAF9DAFAEAFBFAFAC97AFE695
:10916000B4E1A196BFAFAEAFA197312C212CBFEFD8
:109170006C96BFAF6C97EFEFA496EFAFA497FFEF9D
:10918000E396FFAFE3972FE4E6962FAFE69733EC35
:10919000E7963FAFE79707E481E090E0A0E0B0E01A
:1091A000022C04C0880F991FAA1FBB1F0A94D2F774
:1091B000C458DF4F88839983AA83BB83CC57D040A0
:1091C000ACECB4E0E296BFAFAEAFE297EBE5F4E112
:1091D000A396FFAFEEAFA39710E0C058DF4F2882F1
:1091E000C058D040E296AEADBFADE2978D91E29609
:1091F000BFAFAEAFE29790E0B0E0A0E0C458DF4F61
:10920000288139814A815B81CC57D04082239323C6
:10921000A423B523892B8A2B8B2B09F0E5C0A196BB
:10922000AEADBFADA197CD90DD90ED90FC90A39633
:10923000AEADBFADA3972D913D914D915C91A89698
:109240002CAF3DAF4EAF5FAFA897A7019601E09658
:109250006CAD7DAD8EAD9FADE0970F9461242B0179
:109260003C01A8962CAD3DAD4EAD5FADA897AC9638
:109270006CAD7DAD8EAD9FADAC970F9461244B016D
:109280005C01A3019201C301B2010F94EA1D2B01FD
:109290003C01A5019401C501B4010F94EA1D9B0195
:1092A000AC01C301B2010F9462240F9410274B014B
:1092B0005C01A70196016BA17CA18DA19EA10F94D9
:1092C00061246B017C01A8962CAD3DAD4EAD5FAD28
:1092D000A8976FA178A589A59AA50F9461242B0161
:1092E0003C01A7019601C701B6010F94EA1D6B016D
:1092F0007C01A3019201C301B2010F94EA1D9B01FD
:10930000AC01C701B6010F9462240F94102720E02E
:1093100030E040E751E40F945C25A50194010F94DF
:1093200062246B017C018090D1049090D204A090C3
:10933000D304B090D40420E030E040E85FE3C501FE
:10934000B4010F94C2261816F4F4C501B4010F94A9
:10935000CE254B015C0160E070E0CB0118141904CC
:109360001A041B0434F40F94BB18A50194010F9444
:10937000EA230F948B1D9B01AC01B601C7010F942A
:1093800062246B017C019601A701E3966FADE39720
:10939000E6967FADE697E7968FADE797902F0F940F
:1093A000C22618160CF56C961FAF6C97C058DF4F8D
:1093B000B881C058D040A496BFAFA497E896CFAE6E
:1093C000E897E996DFAEE997EA96EFAEEA97EB9673
:1093D000FFAEEB97E396CFAEE397E696DFAEE69768
:1093E000E796EFAEE7970F2D1F5FA396EEADFFADAB
:1093F000A3973496A396FFAFEEAFA397153009F06D
:10940000F1CEFFEF2F1A3F0AA1962EAD3FADA197E7
:109410002C5F3F4FA1963FAF2EAFA19735E02316AB
:10942000310409F0B9CE6C964FAD6C97E42FF0E0A3
:10943000E453FB4F208181E090E0A0E0B0E0A496EF
:109440000FACA49704C0880F991FAA1FBB1F0A94D2
:10945000D2F7822B8083A4965FADA49762965FAF0C
:10946000629763964FAF6397E8968FADE897E9965A
:109470009FADE997EA96AFADEA97EB96BFADEB9754
:1094800067968CAF9DAFAEAFBFAF67975F3F09F4F4
:1094900023C24F3F09F420C284E04802F0011124A6
:1094A000E55AFB4E108101813280238027E137EBA2
:1094B00041ED58EB612F702F832D922D0F94C22612
:1094C00087FD0EC223E030E04AE953E4612F702F9C
:1094D000832D922D0F94841D18160CF401C2A496AE
:1094E0009FADA497A4E09A02F0011124E159FB4E2C
:1094F000C080D180E280F38027E137EB41ED58EB6B
:10950000B601C7010F94C22687FDEAC123E030E807
:109510004DE953E4B601C7010F94841D18160CF4ED
:10952000DFC120E030E040EA50E4B601C7010F940B
:109530006224A0966FAFA097A2967FAFA297A59640
:109540008FAFA597A9969FAFA997CB01A596AFAD71
:10955000A597A996BFADA99721968CAF9DAFAEAF49
:10956000BFAF2197812F902FA32DB22D25968CAFC1
:109570009DAFAEAFBFAF2597A496BFADA497B11175
:1095800009C26C96EFAD6C97E111D1C120E030E0DB
:1095900040EA50E4612F702F832D922D0F946224A6
:1095A000A4966FAFA497AD967FAFAD97E1968FAFBE
:1095B000E197E3969FAFE3976C96FFAD6C97FF231F
:1095C00009F4AAC26C963FAD6C97A096CFAEA09757
:1095D000A296DFAEA297A596EFAEA597A996FFAE8D
:1095E000A99734300CF0CDC122ED822E23E5922EC6
:1095F0002BE7A22E21E4B22E21964CAC5DAC6EACD2
:109600007FAC219725962CAD3DAD4EAD5FAD259736
:109610006F962CAF3DAF4EAF5FAF6F97A301920136
:10962000B601C7010F9461242D966CAF7DAF8EAF4C
:109630009FAF2D976F962CAD3DAD4EAD5FAD6F9743
:10964000612F702F832D922D0F94612461966CAF42
:109650007DAF8EAF9FAF6197A30192016091FA0C2D
:109660007091FB0C8091FC0C9091FD0C0F94612487
:109670002B013C016F962CAD3DAD4EAD5FAD6F97AC
:109680006091FE0C7091FF0C8091000D9091010D86
:109690000F9461246F966CAF7DAF8EAF9FAF6F97C5
:1096A000A0968FADA097A2969FADA297A596AFADBD
:1096B000A597A996BFADA9978DA79EA7AFA7B8AB51
:1096C000A4968FADA497AD969FADAD97E196AFAD43
:1096D000E197E396BFADE39789AB9AABABABBCAB7D
:1096E000C984DA84EB84FC84CDAADEAAEFAAF8AEA2
:1096F0002DEC3CEC4CEC5CE3C501B4010F94EA1D8D
:1097000029813A814B815C810F94EA1D2091060DDD
:109710003091070D4091080D5091090D0F9462246E
:1097200069AF7AAF8BAF9CAFA3019201C301B201C5
:109730000F94EA1D2B013C016F962CAD3DAD4EAD53
:109740005FAD6F97CA01B9010F94EA1D9B01AC018F
:10975000C301B2010F94622420E030E040E050E405
:109760000F94C2261816ACF420E030E040E05FE32E
:10977000C701B6010F94622429966CAF7DAF8EAFFE
:109780009FAF2997BE01635C7F4FCE0101960E9477
:109790007C1C89859A85AB85BC8529968CAF9DAF4D
:1097A000AEAFBFAF29976B961CAE1DAE1EAE1FAEFF
:1097B0006B97BE01695A7F4FCE01CD960E94AF1FB5
:1097C0008CA58823C1F02AE939E949E95FE36D8175
:1097D0007E818F8198850F94EA1D6B966CAF7DAF6B
:1097E0008EAF9FAF6B97BE01695A7F4F85EE9AE0AF
:1097F0000E94AF1F1CA6A090C00CB090C10CC090DE
:10980000C20CD090C30CE090BC0CF090BD0C009149
:10981000BE0C1091BF0C9701A801B501C6010F94B1
:10982000C226181614F075018601809047029090A8
:109830004802A0904902B0904A022DEC3CEC4CEC5E
:109840005DE3B701C8010F94EA1D6093470270936E
:1098500048028093490290934A0240E0BE01675B50
:109860007F4FCE018D960E94A0F480E1EAEFFCE0EC
:10987000A5EEBAE001900D928A95E1F78092470239
:1098800090924802A0924902B0924A0220E04FEF23
:10989000BE016F5A7F4FCE0101960E942A2120E01F
:1098A00041E0BE016F5A7F4FCE0101960E942A21EE
:1098B0002FEF40E0BE016F5A7F4FCE0101960E940C
:1098C0002A2121E040E0BE016F5A7F4FCE01019670
:1098D0000E942A210E9403C280910A0D80930B0DE1
:1098E000E5964EAD5FADE59741505109E5965FAF06
:1098F0004EAFE597452B09F42CCB62968FAD62975E
:1099000087FD27CB63968FAD639787FF08CC21CB6C
:109910002BA13CA14DA15EA1E0962CAF3DAF4EAF77
:109920005FAFE0978FA198A5A9A5BAA512CCC601F3
:10993000D70121968CAF9DAFAEAFBFAF219720E08E
:1099400030E040EA50E4612F702F832D922D0F9468
:10995000612425966CAF7DAF8EAF9FAF25976C9637
:109960002FAD6C9724300CF411CEA4961FAFA497A2
:10997000AD960FAFAD97E1963FAEE197E3962FAE70
:10998000E39792ED892E93E5992E9BEFA92E90E413
:10999000B92E32CEA4964FADA49744300CF46EC0CD
:1099A0006C965FAD6C975430BCF120E030E040EA3B
:1099B00050E4B601C7010F94612421966CAF7DAFCE
:1099C0008EAF9FAF219720E030E040EA50E4612F56
:1099D000702F832D922D0F946124A4966FAFA497BE
:1099E000AD967FAFAD97E1968FAFE197E3969FAFCE
:1099F000E3976C969FAD6C97A096CFAEA097A2967A
:109A0000DFAEA297A596EFAEA597A996FFAEA99750
:109A100094300CF0B6CFE8CDC601D70121968CAFBB
:109A20009DAFAEAFBFAF219720E030E040EA50E4F9
:109A3000612F702F832D922D0F94622425966CAF89
:109A40007DAF8EAF9FAF25976C968FAD6C978111D0
:109A5000BACF20E030E040EA50E4B601C7010F94ED
:109A60006124A0966FAFA097A2967FAFA297A5960C
:109A70008FAFA597A9969FAFA99777CF6C96AFADFB
:109A80006C97A1112BC020E030E040E251E4A09699
:109A90006FADA097A2967FADA297A5968FADA59723
:109AA000A9969FADA9970F946124A0966FAFA09738
:109AB000A2967FAFA297A5968FAFA597A9969FAFC5
:109AC000A997A4961FAFA497AD960FAFAD97E19657
:109AD0003FAEE197E3962FAEE39786CD6C96BFAD90
:109AE0006C97B43034F120E030E040E251E4A096CD
:109AF0006FADA097A2967FADA297A5968FADA597C3
:109B0000A9969FADA9970F94612421966CAF7DAF64
:109B10008EAF9FAF2197D5CFA096CFAEA097A2963C
:109B2000DFAEA297A596EFAEA597A996FFAEA9972F
:109B300028CFA4961FAFA497AD960FAFAD97E1962F
:109B40003FAEE197E3962FAEE39782ED882E83E553
:109B5000982E8BEFA82E81E4B82E4ECD89ED96E09D
:109B60000C94382ACF92DF92EF92FF920F931F93BB
:109B7000CF93DF9388E50E94B222D82E89E40E9419
:109B8000B222C82E8823D1F10E948422D82F89E5E1
:109B90000E94B222182F8AE40E94B222082F882342
:109BA00009F455C00E948422C82F8AE50E94B2227F
:109BB000E82EF12C811104C081E50E94B222F82E1A
:109BC000C11001C000E0802F90E0D11001C010E072
:109BD000810F911D019721F4E11062C0F11060C066
:109BE0000E94AE4D84E29CE0DF91CF911F910F91D6
:109BF000FF90EF90DF90CF900C94382AD11002C0E4
:109C0000DFEFC5CF0E94882220914B0C30914C0C85
:109C100040914D0C50914E0C0F94612420E030E0A7
:109C200040EA51E40F94612420E030E042E052E445
:109C30000F94622421EC3FE04CE75CE30F94EA1DB3
:109C40000F94CE25D62F653008F4A1CFD9CF1111AE
:109C500002C0CFEFAACF0E94882220914F0C3091F2
:109C6000500C4091510C5091520C0F94612420E003
:109C700030E040EA51E40F94612420E030E042E01B
:109C800052E40F94622421EC3FE04CE75CE30F9434
:109C9000EA1D0F94CE25C62F653008F486CFD9CFA4
:109CA000D7FD02C0C7FF05C00E94AE4D8BE09CE00F
:109CB0009BCF0E9488229B01AC010D2FDD0F110B61
:109CC000AC2FCC0FBB0B60E070E0CB01FF2091F01C
:109CD00065E0609FF001619FF00D1124EA0FFB1F0A
:109CE000EE0FFF1FEE0FFF1FE250F54F60817181F5
:109CF00082819381E5E0E09FE001E19FD00D112496
:109D0000CA0FDB1FCC0FDD1FCC0FDD1FC250D54F9C
:109D10000F946224688379838A839B83DF91CF9138
:109D20001F910F91FF90EF90DF90CF90089583EDFA
:109D300096E00C94382ACF9384E50E940023C091CA
:109D4000F80C8823D9F00E94E91CC82F8230B4F0A7
:109D50000E94974E8DE40E94FF2980910B059091FF
:109D60000C050E943EFA6C2FCC0F770B8EE39DE022
:109D70000E943A368AE00E94FF29CFEF8C2FCF91C4
:109D800008954F925F926F927F928F929F92AF92BF
:109D9000BF92CF92DF92EF92FF921F93CF93DF9308
:109DA00000D000D01F921F92CDB7DEB70E949B4E0D
:109DB000D82E87FDB2C08AE50E940023812C912C09
:109DC00020E2A22E21E4B22E882341F040E050E0B0
:109DD000BA018AE50E9436234B015C011091F80C10
:109DE000ED2C0D2C000CFF081E151F0421F060E067
:109DF0008D2D0E94A2C720E030E0A901C501B40169
:109E00000F94C22618167CF580E090E0A0EAB0E43A
:109E10008D839E83AF83B8872091020D3091030D0F
:109E20004091040D5091050DC501B4010F946224B9
:109E30002B013C0120E030E048EC53E40F94841DFA
:109E400087FD06C0412C512C98EC692E93E4792EA5
:109E500049825A826B827C82BE016B5F7F4FCE014A
:109E600001960E9454C784E50E94002381116BC0B3
:109E70008091F80C882321F060E080E00E94A2C766
:109E80008091CF089091D008A091D108B091D208CC
:109E9000B05889839A83AB83BC83CE0101960E941C
:109EA00009F020E030E0A901C501B4010F94C226F9
:109EB00018165CF580E090E0A0EAB0E48D839E8304
:109EC000AF83B887A50194016091020D7091030DD5
:109ED0008091040D9091050D0F9461246B017C011C
:109EE00020E030E0A9010F94C22618161CF0C12C06
:109EF000D12C7601C982DA82EB82FC82BE016B5FD3
:109F00007F4FCE0101960E9454C78091F80C8117B3
:109F100021F060E0812F0E94A2C728960FB6F89426
:109F2000DEBF0FBECDBFDF91CF911F91FF90EF90AD
:109F3000DF90CF90BF90AF909F908F907F906F9069
:109F40005F904F90089585E50E94B2228823D1F05A
:109F50000E9488226B017C0120E030E0A901C7014A
:109F6000B6010F94C22687FF04C0F7FAF094F7F801
:109F7000F094F7FAF094F7F8F094C982DA82EB8261
:109F8000FC828BCFF70183E0EE0FFF1F8A95E1F78C
:109F9000E153F74FC080D180E280F380DDCF2F9274
:109FA0003F924F925F926F927F928F929F92AF9269
:109FB000BF92CF92DF92EF92FF920F931F93CF93B6
:109FC000DF93CDB7DEB76A970FB6F894DEBF0FBE4A
:109FD000CDBF83E50E94B222182F3090F90C882360
:109FE00019F00E94FD1C382E4090FA0C5090FB0C8A
:109FF0006090FC0C7090FD0C8091FE0C9091FF0C19
:10A00000A091000DB091010D8B8B9C8BAD8BBE8B05
:10A010008091020D9091030DA091040DB091050D5A
:10A020008F8B988FA98FBA8F112329F0311003C01D
:10A0300080E00E94DD2486E50E94B2228A8B0E9485
:10A04000F824882309F4C3C083E40E94B222882341
:10A0500009F49DC00E9488226B017C01AEEFBAE03A
:10A06000BF83AE83B987A887F5E0FD831D861E8672
:10A0700028EC2F8702EC1A86212C88EC8B8792E43F
:10A080009C87A885B985B98BA88B15E0E889F989E3
:10A0900081909190A190B190F98BE88B2A85322D17
:10A0A0004B855C85C501B4010F94841D87FF04C0F6
:10A0B0008A86292CAB86BC862D853E854F85502F00
:10A0C000C501B4010F94C226181624F48D869E860D
:10A0D000AF860B2D1150D1F6FD81F150FD8388859F
:10A0E0009985449699878887F111CBCF2D853E8538
:10A0F0004F85502F6A85722D8B859C850F94622425
:10A1000020E030E040E05FE30F94EA1DA7019601F4
:10A110000F9462244B015C012DEB37E346E855EBCD
:10A120000F94C22687FD0AC02DEB37E346E855E3BE
:10A13000C501B4010F94841D18164CF580E00E94EF
:10A14000DD2410E0EE80FF8000E0D7016D917D916D
:10A150008D919D917D016D01B4E0CB1AD108A501CF
:10A1600094010F946124F601608371838283938349
:10A17000602F812F0E94D4EE0F5F053031F71F5FF3
:10A180008E819F8144969F838E831530D9F6AA894C
:10A19000AA2351F00E94F824882331F081EE9AE03E
:10A1A0000E94382A0E947B358AE50E94B2228823C9
:10A1B00051F00E94882269837A838B839C83CE012D
:10A1C00001960E948AED832D0E94DD240BC0311080
:10A1D00003C09A89992341F30E94974E87EF9AE032
:10A1E0000E94382A332051F08091F90C811106C069
:10A1F0000E94AE4D82EC9AE00E94382A0E94974E4F
:10A2000084EB9AE00E94382A8091F90C0E94FA357A
:10A210000E94974E87EA9AE00E94382AC090470C25
:10A22000D090480CE090490CF0904A0C20E030E0CF
:10A23000A901C701B6010F94C22618160CF053C02D
:10A2400042E0C701B6010E9458988DE00E94FF29A4
:10A250008AE00E94FF29A30192016091FA0C70919B
:10A26000FB0C8091FC0C9091FD0C0F94841D8111CE
:10A270001FC02B893C894D895E896091FE0C7091CD
:10A28000FF0C8091000D9091010D0F94841D8111A0
:10A290000FC02F89388D498D5A8D6091020D7091B4
:10A2A000030D8091040D9091050D0F94841D811173
:10A2B0000E9481D36A960FB6F894DEBF0FBECDBF61
:10A2C000DF91CF911F910F91FF90EF90DF90CF9092
:10A2D000BF90AF909F908F907F906F905F904F90C6
:10A2E0003F902F90089582EA9AE00E94382AB3CFD7
:10A2F0005F926F927F928F929F92AF92BF92CF9216
:10A30000DF92EF92FF920F931F93CF93DF931F92F1
:10A31000CDB7DEB77C0139018B015B01A40EB51E00
:10A32000D12CC12CA016B10609F450C0F7018080D1
:10A330009180F80151908F015982C4010F94A2239A
:10A340005816B9F1652DC4010F94AA23FFEFCF1A57
:10A35000DF0AC6018F779927892B21F162E070E02F
:10A3600080E090E00E9491F3C4010F94A2239981B0
:10A370008917F9F00E94974E8FE394E00E94382AE3
:10A3800081E00F90DF91CF911F910F91FF90EF909F
:10A39000DF90CF90BF90AF909F908F907F906F9005
:10A3A0005F90089562E070E080E090E00E943D25BB
:10A3B000DBCFBE016F5F7F4FC3010E949FE4F701B7
:10A3C00080819181019691838083ACCF80E0D9CF49
:10A3D000CF93DF93CDB7DEB7A8970FB6F894DEBF63
:10A3E0000FBECDBF8C01F42E0E94CC9C0E94AE4DBE
:10A3F00083EB96E00E94382A0115110511F40AEA50
:10A4000016E080915C0580FD79C0816080935C05D9
:10A4100086E996E00E94382A8AE00E94FF29CC242F
:10A42000C3948AE5D82ED092FD13C092FC138FE01E
:10A4300090E09093FF138093FE1397E0792E709233
:10A44000F01322E8E22EE092F31334E8832E912CED
:10A45000A12CB12C8092F4139092F513A092F613D4
:10A46000B092F71380EA93E10E947D26D092FD130B
:10A47000C092FC1388E590E09093FF138093FE1345
:10A480007092F013E092F3138092F4139092F5130C
:10A49000A092F613B092F71380EA93E10E947D2612
:10A4A0008AE289838A838B838C83F801DE01159687
:10A4B000BE016F5F7F4FCD01861B970B24913196B4
:10A4C00021110CC0FB01E80FF91F8AE29F01261B36
:10A4D000370B2832310524F48193F8CF2D93EBCF3D
:10A4E00020E630E140E050E080EA93E10E94BAE4E7
:10A4F0006AE070E080E090E00E94612561E081EA1E
:10A5000096E00E94E03389EE93E030E6019729F06F
:10A51000232F2A950000E9F7F9CFF89489EE93E00C
:10A5200038EE019729F0232F2A950000E9F7F9CF9B
:10A530000E94CC9CFF2031F00E948C250E94331990
:10A54000A895FECF0E943019F9CF80910A0D909105
:10A550000B0D2FEF3FEF981751F0E92FF0E0E65F7A
:10A56000F24F228130E09F5F9F7790930B0DC901DE
:10A5700008951F920F920FB60F9211240F900FBEE5
:10A580000F901F9018951F920F920FB60F921124E3
:10A590000BB60F920F931F932F933F934F935F939D
:10A5A0006F937F938F939F93AF93BF93CF93DF93DB
:10A5B000EF93FF93C091C60000910B0DD0910A0D4F
:10A5C00011E01D0F1F7790911104913108F09FC089
:10A5D000E92FF0E08827E051FD4A8F4F0D944D247C
:10A5E000015330533F534E53555387535953875359
:10A5F0005D5361538753655369536D537453875348
:10A600007F53C03229F028F5CA3011F0CD3031F532
:10A61000011731F0ED2FF0E0E65FF24FC283D12F4A
:10A62000D0930A0DFF91EF91DF91CF91BF91AF9140
:10A630009F918F917F916F915F914F913F912F915A
:10A640001F910F910F900BBE0F900FBE0F901F9098
:10A650001895CD3481F081E0CE3471F080E10CC0EA
:10A66000CA3338F4C033A0F6C03291F2CD32B1F71C
:10A67000CFCFCD3499F782E080931104C9CFC13395
:10A6800059F018F4C03221F2E9CF88E0C433A1F3C5
:10A690008BE0C83389F3E2CF83E0EECF84E0C033B0
:10A6A00059F386E0C13341F3D9CF85E0C833B1F621
:10A6B000E3CF87E0C23391F6DFCF89E0C13371F693
:10A6C000DBCF8AE0C03351F6D7CF8CE0C73331F609
:10A6D000D3CF8DE0C63311F6CFCFC03209F498CF77
:10A6E0008EE0C33549F2BACF80ED8C0F8A3008F086
:10A6F0008FCF9FE0909311048093120489CFCA30CA
:10A7000019F0CD3009F084CF1092110481CFCA30F6
:10A7100019F0CD3009F07CCF80915A148823A1F331
:10A72000973079F038F4953079F71092460210920C
:10A730006512EACF9A3049F09F3031F70E948CE4DD
:10A74000E3CF81E08093FE08DFCF81E08093FD08B6
:10A75000DBCF8EBD0DB407FEFDCF08958FEF8EBD0C
:10A760000DB407FEFDCF8EB50895909164009B7FD8
:10A7700090936400982F906A96959CBD80FD03C0CD
:10A7800091E0863009F490E09DBD0895CF93DF936A
:10A79000EB010E94382ACE01DF91CF910C94C28D3B
:10A7A0002F923F924F925F926F927F928F929F92E1
:10A7B000AF92BF92CF92DF92EF92FF920F931F93CF
:10A7C000CF93DF93009709F0AAC11092E40C109286
:10A7D000E30C90935B0580935A05BAE0CB2EB0E270
:10A7E000DB2EE12CF12C15E002E846015701C4E113
:10A7F000D0E010924313109242131093361300933B
:10A80000391380923A1390923B13A0923C13B0926A
:10A810003D1386EE92E10E947D2621972FEF821A4A
:10A82000920AA20AB20A209721F744E1C40ED11C71
:10A83000E11CF11C8AE5C81680E2D806E104F104A7
:10A84000A1F6C12CA0E2DA2EE12CF12CD5E0C2E871
:10A850001092431310924213D0933613C0933913BE
:10A86000C0923A13D0923B13E0923C13F0923D1306
:10A8700086EE92E10E947D261092431310924213BD
:10A88000D0933613C0933913D701C6018C529F4F12
:10A89000AF4FBF4F80933A1390933B13A0933C1359
:10A8A000B0933D1386EE92E10E947D26EFEFCE1A23
:10A8B000DE0AEE0AFE0AFAE0CF16F0E2DF06E10455
:10A8C000F10431F6FEEDCF2EF0E2DF2EE12CF12C7B
:10A8D000D5E0C2E81092431310924213D09336137E
:10A8E000C0933913C0923A13D0923B13E0923C13B9
:10A8F000F0923D1386EE92E10E947D262FEFC21A60
:10A90000D20AE20AF20A46EEC41640E2D406E10494
:10A91000F10401F7CC24C394E2E1DE2EE12CF12C0A
:10A920000AE010E0D5E0C2E810934313009342130D
:10A93000D0933613C0933913C0923A13D0923B137D
:10A94000E0923C13F0923D1386EE92E10E947D2648
:10A950001093431300934213D0933613C0933913CB
:10A96000D701C6018096A11DB11D80933A13909323
:10A970003B13A0933C13B0933D1386EE92E10E94EB
:10A980007D268FEFC81AD80AE80AF80AE5E0CE1645
:10A99000E2E1DE06E104F10439F60091E30C1091E6
:10A9A000E40C0115110509F0D6C08091E20C882352
:10A9B00009F4E1C02AE030E240E050E06AEC73E0E4
:10A9C00086EE92E10E94BAE4C1E0D0E003E010E03C
:10A9D000E090E30CF090E40C35E0332E42E8242EB6
:10A9E00044244A94542C64E0662E712C7FE1C72ED7
:10A9F00074E0D72E8091E30C9091E40C800F911FAE
:10AA0000E816F90608F0D5C0C7010E94C4E58823FE
:10AA100009F481C08091061269EF71E1882311F079
:10AA200066E072E1FB0101900020E9F7CF01019798
:10AA3000861B970BF4E1FC9F9001FD9F300D1124C4
:10AA4000265F3F4D50E040E0459710F0FB01128A31
:10AA500086EE92E10E94BAE4CE018F5F9D4EB0E097
:10AA6000A0E021964E0124E0880C991C2A95E1F77C
:10AA7000FDEF8F1AFFE99F0AB12CA12C20918E14B3
:10AA800024FF7EC0709243136092421330923613BB
:10AA90002092391380933A1390933B13A0933C1365
:10AAA000B0933D1386EE92E10E947D26D09243132F
:10AAB000C0924213309236132092391380923A1387
:10AAC00090923B13A0923C13B0923D1386EE92E11C
:10AAD0000E947D26B7018AE394E10E9406368091A8
:10AAE000061266E072E1811102C069EF71E187E34D
:10AAF00094E10E94C65367E57CE083E394E10E9401
:10AB0000C65369EF71E182E394E10E94C6538EE27D
:10AB100094E10E94382A2FEFE21AF20A6BCF2091BB
:10AB2000E30C3091E40CA9014150510960915A05A0
:10AB300070915B056817790738F42C5F3F4F3093AD
:10AB4000E40C2093E30C45CE4430510508F43DCE8F
:10AB500024503109F4CF0430110569F48091E20CDE
:10AB6000882331F083E090E09093E40C8093E30C31
:10AB7000D0E0C0E02DCFD0E0C0E004E010E028CF6E
:10AB800010924313109242133092361320923913CD
:10AB900080933A1390933B13A0933C13B0933D13CF
:10ABA00086EE92E10E947D2650924313409242131A
:10ABB00081CFDF91CF911F910F91FF90EF90DF90A8
:10ABC000CF90BF90AF909F908F907F906F905F904D
:10ABD0004F903F902F900895AF92BF92CF92DF9207
:10ABE000EF92FF920F931F93CF93DF93CDB7DEB712
:10ABF000E6970FB6F894DEBF0FBECDBF00910E05ED
:10AC000010910F05F80101900020E9F731976F01CD
:10AC1000C01AD10AF801CF01801B910B8C159D053C
:10AC20003CF481918F32B9F7DF0111971C92F3CF79
:10AC30008BE1EEEAF4E1DE015C9601900D928A95DB
:10AC4000E1F7F12CE12CEC14FD040CF05DC0F801EF
:10AC5000EE0DFF1D8081811103C08FEFE81AF80A05
:10AC60005801AE0CBF1CF5018081882309F44CC04B
:10AC7000FFEFEF1AFF0AF801EE0DFF1D7F01E01A4A
:10AC8000F10A81918111FACFCE014C960E94559222
:10AC90008BE1FE017C96DE01119601900D928A9562
:10ACA000E1F7B501CE0101960E94638ACE010196BB
:10ACB0000E94B7248FE20E94FF2980910612811121
:10ACC0003BC087ED93E00E94C28D80918E1484FF7B
:10ACD0001BC019821C8221E0A501BE01645E7F4F6A
:10ACE000CE0101960E949794811129C08AE00E94AA
:10ACF000FF290E94974EB50189E193E10E94C65356
:10AD0000CE0101960E94B7248AE00E94FF29CE015D
:10AD10004C960E94B724E6960FB6F894DEBF0FBE9D
:10AD2000CDBFDF91CF911F910F91FF90EF90DF90FA
:10AD3000CF90BF90AF90089586E092E1C4CFCE014E
:10AD40004C960E94C4918BE1FE013196DE015C9627
:10AD500001900D928A95E1F7CE0101960E94B724E9
:10AD600072CF2F923F924F925F926F927F928F920B
:10AD70009F92AF92BF92CF92DF92EF92FF920F938A
:10AD80001F93CF93DF9300D000D000D01F921F926B
:10AD9000CDB7DEB7B82E8091070E843008F0D1C150
:10ADA0000E94C4F36B017C018091070E811108C0E1
:10ADB00080910A0D90910B0D891B8F7709F4FDC5C9
:10ADC00081E6A82E13C08A3019F08D3009F0F6C044
:10ADD0001092F20D8091900D9091910DFC01E4572D
:10ADE000F24F1682892BF1F40E94C1CA8091070E9E
:10ADF000843008F0ECC080910A0D90910B0D891BF6
:10AE00008F7709F4E4C00E94A55297FFDCCF0E941F
:10AE1000AE4D85E895E00E94382A80910A0D809316
:10AE20000B0DE4CF1092910D1092900D02E91DE0F0
:10AE3000F8018191803209F446C08E3409F0A9C02E
:10AE400060E875E0C8010F94011D4C01892B41F0A9
:10AE50006EE470E0C80104960F94B027009709F4DF
:10AE6000C8014AE050E070E060E001960F94711A6A
:10AE70002B013C0180918C0D90918D0DA0918E0D38
:10AE8000B0918F0D0196A11DB11D481659066A0695
:10AE90007B0629F060E08DE495E0892851F16AE2B3
:10AEA00070E0C8010F94DF279C01009729F1982FCB
:10AEB000901B912C992349F09150F801E90FF11D55
:10AEC00080819826F7CF8F01B3CF4AE050E070E041
:10AED00060E0C90101960F94711A292D30E050E00D
:10AEE00040E0621773078407950751F060E08EE237
:10AEF00095E00E9411EB7ACF60E084E095E0F9CF15
:10AF000040928C0D50928D0D60928E0D70928F0D2F
:10AF10008091E40A8130E1F067E470E0C8010F94A9
:10AF2000B0270097A9F04AE050E070E060E0019699
:10AF30000F94711A643071058105910548F483E618
:10AF400094E00E94382A60E089E594E00E9413347E
:10AF5000C092FA0AD092FB0AE092FC0AF092FD0A33
:10AF60008091920D8B3309F441CF8091070E84308C
:10AF700008F03CCF8091090E8A9DC001112462E93E
:10AF80007DE0865F914F0F94BB2780E00E94CBEA63
:10AF90002DCF80918E1480FFBBCF6AEE7AE2C8017C
:10AFA0000F94011D009731F0FC01838180538A309A
:10AFB00008F0AECF60E08AED94E09BCF20E93DE061
:10AFC00042E95DE062EF7DE00E94BF180FCF809103
:10AFD0008E1482FFB6C01A82198271E6F72EE0E164
:10AFE000EE2EF9E6DF2E8091070E843008F0A9C01E
:10AFF0000E94F7188111A5C041E050E0BE016B5FCF
:10B000007F4F82EF95E10E9417900D8110E001972C
:10B0100011F00FEF1FEF8091FA159091FB15A091A1
:10B02000FC15B091FD1580938A1490938B14A09316
:10B030008C14B0938D140E94F7180F3F100749F439
:10B04000811107C00E94AE4D83EA95E00E94382A24
:10B05000CACF4091090E242F30E00A3061F00D3044
:10B0600051F0882309F45FC089819A81009719F013
:10B0700001969A8389831092960489819A81F29E1F
:10B08000F001F39EF00D1124E95FF14FE80FF91F75
:10B090001382892B69F50E94C1CA0E94F718882380
:10B0A00009F4A1CF0E9403C282EF95E10E94C491EE
:10B0B00080918514882391F18150809385148D9D12
:10B0C000C001112462E08C5B964F0E947E96E09155
:10B0D000851424E0E29FF0011124E05CF64F6081CA
:10B0E0007181828193810E94001B0E94CC897BCF59
:10B0F0001A82198281E00E94CBEA80918A14909191
:10B100008B14A0918C14B0918D148093030E9093A6
:10B11000040EA093050EB093060EBFCF0E94CD91F2
:10B12000E092E40A60CF4F9DA0011124465F514F89
:10B130009E012F5F3F4F66E974E0802F0E94BF1889
:10B1400052CF0E94C4F36B017C01B11004C0809106
:10B15000A111882351F0C0929911D0929A11E092D6
:10B160009B11F0929C11BB24B3948091E7049091C1
:10B17000E804A091E904B091EA040097A105B105A3
:10B18000B1F04091991150919A1160919B11709179
:10B190009C11840F951FA61FB71FA7019601281B9E
:10B1A000390B4A0B5B0BDA01C901B7FF92C18091E1
:10B1B000080290910902A0910A02B0910B02892B1A
:10B1C0008A2B8B2B09F099C10E94C4F34B015C01BF
:10B1D00080916512811108C020919A1290919B1262
:10B1E00081E0291301C080E0209152123091531266
:10B1F00091E089272A3A31050CF480E091E04091F2
:10B200009B0450919C0460919D0470919E04452B79
:10B21000462B472B09F490E0981789F0882309F40E
:10B22000BDC1D501C40180569444A24FBF4F809345
:10B230009B0490939C04A0939D04B0939E04409023
:10B24000060D5090070D6090080D7090090D20912B
:10B250009704309198044091990450919A04C30145
:10B26000B2010F94841D882319F180919B04909161
:10B270009C04A0919D04B0919E044092970450922A
:10B2800098046092990470929A04892B8A2B8B2BD4
:10B2900009F449C0D501C40180569444A24FBF4F60
:10B2A00080939B0490939C04A0939D04B0939E0470
:10B2B00080919B0490919C04A0919D04B0919E0468
:10B2C0000097A105B10579F1881A990AAA0ABB0A63
:10B2D000B7FC29C010929B0410929C0410929D040C
:10B2E00010929E0483E096E00E94382A60E08FEE80
:10B2F00095E00E94133480915412909155121816C3
:10B30000190624F490E080E00E9485C18091EA1142
:10B310009091EB111816190634F41092EB1110925B
:10B32000EA110E949F9C8091A3049091A404A09193
:10B33000A504B091A60446015701881A990AAA0AE1
:10B34000BB0AD501C401B7FDB9C120919A129091F1
:10B350009B1280912C0240912D02291323C19091C0
:10B36000650B899FC0011124880F892F881F990BB5
:10B3700091958D838091660B489FC0011124880FA1
:10B38000892F881F990B91958E830E94C4F369833E
:10B390007A838B839C8340E0BE016F5F7F4FCE0139
:10B3A00005960E9431C56D8170E089E00E94BBF274
:10B3B00041E0BE016F5F7F4FCE0105960E9431C50F
:10B3C0006E8170E087E00E94BBF2809109098823BA
:10B3D00009F467C10091140210911502C801029787
:10B3E0002091541230915512281739070CF459C185
:10B3F00080909B128F82188619861A861B868091F0
:10B400009A129F80891509F4E7C0892D90E038E6EB
:10B41000A32EA89EF001A99EF00D1124E957FA4F22
:10B42000458956896789708D452B462B472B81F4BA
:10B43000418D528D638D748D452B462B472B41F4E6
:10B44000458D568D678D70A1452B462B472BE1F11D
:10B4500028E6B22EB89E9001B99E300D1124A901A4
:10B4600049575A4F1A01FA0161817281838194818F
:10B470000F9410274B015C01F10161A172A183A11E
:10B4800094A10F94891D2B013C01F10165A176A1C6
:10B4900087A190A50F94891D9B01AC01C301B20146
:10B4A0000F945C25A50194010F94EA1D4B015C01EA
:10B4B000288539854A855B850F94C226181624F4A1
:10B4C00088869986AA86BB868F818F5F87708F83D7
:10B4D00096CF0E94AE4D6091F80A7091F90A82EB06
:10B4E00095E00E94C6538AE00E94FF2940E070E088
:10B4F00060E090E080E00E94E85190919A12809183
:10B500009B12981749F0C0929911D0929A11E0922B
:10B510009B11F0929C1158CEBB2019F01092A704F9
:10B5200053CE0E94C4F30091991110919A11209169
:10B530009B1130919C118090080290900902A0907C
:10B540000A02B0900B02080D191D2A1D3B1D601B3D
:10B55000710B820B930B97FDE1CF8091A7048111B2
:10B5600033CE81E08093A7045F9A8091970C8E7F01
:10B570008093970C8A9A8091970C8D7F8093970C7B
:10B580008091080180958170809306018091970CCD
:10B590008B7F8093970C0E94301916CE80E090E04C
:10B5A000DC0145CE20919B1258E6259F9001112485
:10B5B00029573A4FF901EE59FF4F9081899FC001F9
:10B5C0001124880F892F881F990B91958D832D59F0
:10B5D0003F4FF9018081D0CE209132023091330269
:10B5E0004091340250913502688579858A859B8522
:10B5F0000F94EA1D4B015C01B801012E000C880B71
:10B60000990B0F948B1D9B01AC01C501B4010F94E4
:10B61000622469837A838B839C83409112025091C8
:10B620001302B801CE0101960E948CA089809A80F5
:10B63000AB80BC8040909F045090A0046090A10417
:10B640007090A204A3019201C501B4010F94841D5E
:10B6500087FF16C028E431EE4AE75FE3C301B20179
:10B660000F94EA1D20E037ED43EA5CE30F94622477
:10B67000A50194010F94EA1D69837A838B839C83CF
:10B6800069817A818B819C8160939F047093A0046F
:10B690008093A1049093A2040F94CE25CB010E9425
:10B6A00085C1F4E6CF0ED11CE11CF11CC092A304AD
:10B6B000D092A404E092A504F092A6040E94C1CA0C
:10B6C0008091E40A882309F439C190910901892FF6
:10B6D00080958170109100021817C9F020918E1486
:10B6E000206220938E148093000290FD40C164EF8D
:10B6F00071E080E090E00E943D250E94EF918091F2
:10B700008E1483FD7DC1111134C10E94CF270E9488
:10B71000C4F36B017C01109107021123F1F08091B9
:10B72000EB048823D1F04091A8045091A9046091C2
:10B73000AA047091AB0446015701841A950AA60A1F
:10B74000B70AB501A40177FD1AC0833009F430C1EE
:10B750000CF01FC181300CF024C1212F30E0A8EE85
:10B76000B3E00F941C24C60ED71EE81EF91EC0922B
:10B77000A804D092A904E092AA04F092AB048091AC
:10B78000A211813009F073C00E94C4F36B017C01E7
:10B790008091B0049091B104A091B204B091B3042F
:10B7A000A7019601281B390B4A0B5B0BDA01C90173
:10B7B000B7FD3AC0D701C601805F984DAF4FBF4F6C
:10B7C0008093B0049093B104A093B204B093B304F7
:10B7D0008090CB089090CC08A090CD08B090CE0877
:10B7E0000E942FD6AB01BC014093CB085093CC08EC
:10B7F0006093CD087093CE088091930A9091940A3B
:10B80000A091950AB091960A88199909AA09BB09CD
:10B81000840F951FA61FB71F8093930A9093940AD5
:10B82000A093950AB093960A8091AC049091AD04D0
:10B83000A091AE04B091AF0446015701881A990A4D
:10B84000AA0ABB0AD501C401B7FD11C020E8C20E87
:10B850002EEED21E26E3E21EF11CC092AC04D09262
:10B86000AD04E092AE04F092AF040E9435B10E94A4
:10B87000DE2E0E9444368091E604882381F10E94E6
:10B88000C4F36B017C018091E2049091E304A091E8
:10B89000E404B091E50446015701881A990AAA0AFE
:10B8A000BB0AD501C401B7FD1AC02091E60430E0FF
:10B8B000A8EEB3E00F941C24C60ED71EE81EF91E96
:10B8C000C092E204D092E304E092E404F092E50432
:10B8D0008091F80C0E94FC988AE00E94FF298091D8
:10B8E000E104882359F10E94C4F36B017C0180912B
:10B8F000DD049091DE04A091DF04B091E004A70183
:10B900009601281B390B4A0B5B0BDA01C901B7FD05
:10B9100015C02091E10430E0A8EEB3E00F941C24A0
:10B92000C60ED71EE81EF91EC092DD04D092DE04BA
:10B93000E092DF04F092E0040E948A892B960FB611
:10B94000F894DEBF0FBECDBFDF91CF911F910F9155
:10B95000FF90EF90DF90CF90BF90AF909F908F902F
:10B960007F906F905F904F903F902F9008950E942E
:10B97000DE91123008F0CBCE0E94CF2760E080E449
:10B9800096E050C08EE496E0909364128093631228
:10B99000BECE843009F0E1CE0E94974E85E596E058
:10B9A00004C00E94974E84E896E00E94382AD5CEC3
:10B9B0000E94974E8DE696E0F8CF8091FA0A90911A
:10B9C000FB0AA091FC0AB091FD0AA7019601281B71
:10B9D000390B4A0B5B0BDA01C901885E9340A10960
:10B9E000B109B7FDEDC98DE995E00E94382AC092F2
:10B9F000FA0AD092FB0AE092FC0AF092FD0AE0C932
:10BA0000123098F488E196E00E94382A8AE00E9479
:10BA1000FF290E94EF1D90E080E00E94D05360E07B
:10BA200081E396E00E94133472CE123009F06FCE9B
:10BA30000E94B995882379F081E00E948F9547EBA9
:10BA400050E068E87BE083E994E10E94179083E985
:10BA500094E10E94C4910E94A524811193CF0E9479
:10BA60008F240E943AF90E94858951CE8F929F922D
:10BA7000AF92BF92CF92DF92EF92FF920F931F93FC
:10BA8000CF93DF9300D01F92CDB7DEB75C016B017F
:10BA90007A01122F002309F443C00E94974E89E1D6
:10BAA00098E00E94382A61E0812F0E94942F9090A4
:10BAB000EB0483E08093EB0481E0809365120E94A5
:10BAC000133582E08093661240E369E078E085EF09
:10BAD00097E00E941F3540E069E97DE08EEE97E037
:10BAE0000E941F3560E081EE97E00E94E03389EE0E
:10BAF00097E00E94382A8AE00E94FF298BEF97E0A6
:10BB00000E94EB1980916512882341F060E0812F3B
:10BB10000E94942F81E00E94B156F4CF9092EB04E2
:10BB200020E030E0A901F50160817181828193817B
:10BB30000F94841D882371F080E090E0A0ECB0E4C5
:10BB400089839A83AB83BC83BE016F5F7F4FC5013E
:10BB50000E9473C720E030E0A901F6016081718185
:10BB6000828193810F94841D882351F18090D00CA1
:10BB70009090D10CA090D20CB090D30C80E090E0CB
:10BB8000A0E7B1E48093D00C9093D10CA093D20C99
:10BB9000B093D30C80E090E0A0EAB1E489839A836B
:10BBA000AB83BC83BE016F5F7F4FC6010E9473C72A
:10BBB0008092D00C9092D10CA092D20CB092D30C67
:10BBC00020E030E0A901F7016081718182819381D9
:10BBD0000F94C226181674F480E090E0A0E4B0E45C
:10BBE00089839A83AB83BC83BE016F5F7F4FC7019C
:10BBF0000E9473C729E93DE040ED57E06AED77E028
:10BC000081E00E9442350E94133581E00F900F9031
:10BC10000F900F90DF91CF911F910F91FF90EF90B8
:10BC2000DF90CF90BF90AF909F908F900895CF936B
:10BC3000C82F8091630B83FD14C08091620B81112A
:10BC400010C080913A0290913B029C012150310931
:10BC500040915412509155124217530714F40E9408
:10BC600085C1CC2331F061E08091F80CCF910C9428
:10BC7000E79A8091620B91E0892780934602809138
:10BC80004602882389F0809152129091531220919C
:10BC9000541230915512821B930B97FF03C091955C
:10BCA00081959109029744F4109246028091630BAA
:10BCB00083FF06C0C1E01AC080E00E94B156DFCF0A
:10BCC000C091620BC11112C080913A0290913B0267
:10BCD000019720915412309155122817390754F7C3
:10BCE0000E94974E82EB97E00E94382A8C2FCF91CA
:10BCF00008959F92AF92BF92CF92DF92EF92FF9200
:10BD00000F931F93CF93DF93CDB7DEB764970FB632
:10BD1000F894DEBF0FBECDBF0E949B4ED82E87FD8C
:10BD2000C6C08AE50E940023882309F4D2C040E0FF
:10BD300050E0BA018AE50E9436237B018C01B09065
:10BD4000F80C8D2D0D2C000C990BB816190621F04E
:10BD500060E08D2D0E94A2C72091020D3091030D4D
:10BD60004091040D5091050D60E070E088EC93E483
:10BD70000F946124962EA72E6C019701A8010F94B1
:10BD8000C22618161CF0E92CFA2C860120E030E0BF
:10BD9000A901B701C8010F94C226181624F4E12C9A
:10BDA000F12C00E010E0B701C8010F94CE25072E5A
:10BDB000000C880B990B0F948B1D6D837E838F83F2
:10BDC000988720E030E0A9010F94841D882321F09A
:10BDD000CE0105960E940E1B80E090E0A0EAB1E43F
:10BDE00089879A87AB87BC871D861E861F86188A1F
:10BDF0008CE40E94B222882309F470C00E94882239
:10BE00006B017C0120E030E0A901C701B6010F946D
:10BE1000C22687FF04C0F7FAF094F7F8F094C98AB5
:10BE2000DA8AEB8AFC8A2091541230915512243020
:10BE3000310574F08091521290915312821B930B32
:10BE400097FF03C091958195910901E004970CF447
:10BE500000E080E00E94175E882359F022E0AE01E6
:10BE6000475F5F4FBE016F5E7F4FCE010D960E9410
:10BE7000365D6D817E818F8198858B019C01305864
:10BE800009831A832B833C8320E030E0A9010F94BF
:10BE9000841D882321F0CE0101960E940E1B809103
:10BEA000F80C8B1521F060E08B2D0E94A2C76496E0
:10BEB0000FB6F894DEBF0FBECDBFDF91CF911F91BB
:10BEC0000F91FF90EF90DF90CF90BF90AF909F9039
:10BED0000895E12CF12C00E211E431CFE091F80C4F
:10BEE00088E0E89FF0011124E153F74FC480D5802A
:10BEF000E680F78087CF7F928F929F92AF92BF921A
:10BF0000CF92DF92EF92FF920F931F93CF93DF9325
:10BF100000D000D01F921F92CDB7DEB76C015B013D
:10BF20004A01722E7801009103090E94E219809162
:10BF30005412909155128E159F051CF4C7010E9452
:10BF400085C180E00E94175E882331F0272DA4016F
:10BF5000B501C6010E94365D1E141F0444F4C701DA
:10BF60000E9485C160E08091F80C0E94E79A81E010
:10BF70000E94175E80E090E0A0E7B2E489839A8394
:10BF8000AB83BC8380E090E0A0E8B0EC8D839E831F
:10BF9000AF83B887BE016F5F7F4FCE0105960E94C9
:10BFA00073C787E00E948DC5811158C08091020D32
:10BFB0009091030DA091040DB091050D4091C00426
:10BFC0005091C1046091C2047091C304C090BC043C
:10BFD000D090BD04E090BE04F090BF04C092E50A8A
:10BFE000D092E60AE092E70AF092E80A4093E90A62
:10BFF0005093EA0A6093EB0A7093EC0A8093ED0A7F
:10C000009093EE0AA093EF0AB093F00A80E090E0DC
:10C01000A8E4B2E489839A83AB83BC83CE01019602
:10C020000E94C1D18091C4049091C504A091C6041E
:10C03000B091C7048093ED0A9093EE0AA093EF0AA3
:10C04000B093F00A80E090E0A0EAB0E489839A839C
:10C05000AB83BC83CE0101960E94C1D1C12CD12CEF
:10C0600080E7E82E82E4F82EC982DA82EB82FC8235
:10C0700080E090E0A0E8B0E48D839E83AF83B88732
:10C08000BE016F5F7F4FCE0105960E9473C720E00F
:10C0900030E0A9016091C8047091C9048091CA047C
:10C0A0009091CB040F94841D87FF0BC0C982DA8264
:10C0B000EB82FC82BE016F5F7F4F88EC94E00E94B0
:10C0C00073C78091C8049091C904A091CA04B0912B
:10C0D000CB048093060D9093070DA093080DB093A9
:10C0E000090D8093F10A9093F20AA093F30AB0939A
:10C0F000F40A81EF9AE00E9414C28091DF08811156
:10C100000E9408EE61E088E398E00E94E0338091AD
:10C11000A11181508093A1114FE554E160E478E0D2
:10C1200085E00E94C7E68091A111882339F00E9422
:10C13000CC898091A11181508093A1118091BB0481
:10C14000882351F01092BB048091B9048093650B51
:10C150008091BA048093660B8091A211823011F411
:10C160000E94F3D60F94571028960FB6F894DEBFAE
:10C170000FBECDBFDF91CF911F910F91FF90EF9038
:10C18000DF90CF90BF90AF909F908F907F90089559
:10C19000CF92DF92EF92FF92CF93DF936B017C01FE
:10C1A000D42FC091EB0483E08093EB0481E0809373
:10C1B0006512C114D104E104F10431F00E94C4F30A
:10C1C000C60ED71EE81EF91E80916512882389F0DD
:10C1D000C114D104E104F10421F48D2F0E94B15661
:10C1E000F3CF0E94C4F36C197D098E099F0997FD56
:10C1F000F4CF10926512C093EB04DF91CF91FF90C2
:10C20000EF90DF90CF9008950F931F93CF93DF931C
:10C21000C82F162F0E94974EC11194C0C6E1D7E0D7
:10C22000CE010E94382A61E0812F0E94942F0E9443
:10C23000C4F3685370458F4F9F4F6093FF0870930E
:10C24000000980930109909302091092030900915B
:10C25000EB0483E08093EB0430E020E049E95DE00B
:10C2600064EA77E082E00E94423584EA97E00E9427
:10C27000EB1981E08093651280916512882309F49F
:10C2800064C060E0812F0E94942F8091030988236D
:10C2900009F454C00E94974E8AE897E00E94382A19
:10C2A00030E020E044E757E06BE777E082E00E946F
:10C2B00042358BE797E00E94EB1941E060E070E0C7
:10C2C000CB010E94C86030E020E050E040E067E62B
:10C2D00077E085E00E94423587E697E00E9490274C
:10C2E0000E94E21980E00E94175E0E94974ECE01E4
:10C2F0000E94382A0E94C4F3685370458F4F9F4FA5
:10C300006093FF08709300098093010990930209DC
:10C310001092030930E020E049E95DE06BE577E049
:10C3200082E00E9442358AE497E00E94EB1981E0A6
:10C330008093651261E0812F0E94942F81E00E941A
:10C34000B1569ACFCBE2D7E06BCF0093EB04DF91ED
:10C35000CF911F910F910895BF92CF92DF92EF92EC
:10C36000FF920F931F93CF93DF93CDB7DEB7A097C4
:10C370000FB6F894DEBF0FBECDBF0E949B4E87FD67
:10C38000E0C0B090F80C282F082E000C330BB2162A
:10C39000130619F060E00E94A2C785E40E94B22251
:10C3A000882309F4DEC00E9488226B017C0120E012
:10C3B00030E0A9010F94C22687FF04C0F7FAF09479
:10C3C000F7F8F094F7FAF094F7F8F094C98ADA8A5B
:10C3D000EB8AFC8A8CE0E3E9F2E0DE011196019041
:10C3E0000D928A95E1F78AE50E940023882351F097
:10C3F00040E050E0BA018AE50E94362369877A87D7
:10C400008B879C8788E50E940023882351F040E0B9
:10C4100050E0BA0188E50E94362369837A838B83D2
:10C420009C8389E50E940023882351F040E050E07E
:10C43000BA0189E50E9436236D837E838F839887B6
:10C4400085E50E94B222882309F492C00E948822C6
:10C450006B017C0120E030E0A901C701B6010F9417
:10C46000C22687FF04C0F7FAF094F7F8F094F7FAC1
:10C47000F094F7F8F094CD8ADE8AEF8AF88E198E60
:10C480001A8E1B8E1C8E8CE40E94B222882309F423
:10C490007CC00E9488226B017C0120E030E0A90171
:10C4A000C701B6010F94C22687FF04C0F7FAF094C3
:10C4B000F7F8F094CD8EDE8EEF8EF8A262E070E099
:10C4C00082E40E941B23F82E8091A111811131C0BA
:10C4D00021E0AE014B5E5F4FBE016F5F7F4FCE012B
:10C4E00041960E947734882321F16F2D81E00E94CC
:10C4F000046182E50E940023882309F453C00E944E
:10C50000842240E050E060EA71E44D875E876F87E7
:10C51000788B2091A111222361F08C012F2DAE0187
:10C52000435F5F4FBE01635E7F4FCE0149960E941D
:10C530007B5F8091F80C8B1521F060E08B2D0E94C1
:10C54000A2C7A0960FB6F894DEBF0FBECDBFDF9195
:10C55000CF911F910F91FF90EF90DF90CF90BF9000
:10C560000895C12CD12C80E8E82E80E4F82E2ACF43
:10C57000E091F80C88E0E89FF0011124E153F74FB7
:10C58000C080D180E280F38065CFE091F80C88E034
:10C59000E89FF0011124E153F74FC480D580E68075
:10C5A000F7807BCF90E080E0ACCFCF92DF92EF922C
:10C5B000FF920F931F93CF93DF93CDB7DEB76C97A6
:10C5C0000FB6F894DEBF0FBECDBF8CE40E94B2223E
:10C5D000882309F4B0C00E9488226B017C0120E00E
:10C5E00030E0A9010F94C22687FF04C0F7FAF09447
:10C5F000F7F8F094F7FAF094F7F8F094C98EDA8E21
:10C60000EB8EFC8E8CE0E3E9F2E0DE011196019006
:10C610000D928A95E1F788E50E9400238823A1F016
:10C6200040E050E0BA0188E50E94362320914B0C8F
:10C6300030914C0C40914D0C50914E0C0F94612454
:10C6400069837A838B839C8389E50E9400238823F6
:10C65000A1F040E050E0BA0189E50E943623209124
:10C660004B0C30914C0C40914D0C50914E0C0F9452
:10C6700061246D837E838F8398878AE50E940023DF
:10C68000882351F040E050E0BA018AE50E94362349
:10C6900069877A878B879C871D861E861F86188AE6
:10C6A0008091A111811138C020E0AE01435F5F4F3E
:10C6B000BE016F5F7F4FCE0149960E947734882379
:10C6C00059F18091DF0881110E9408EE60E080E05E
:10C6D0000E940461898D9A8DAB8DBC8DB0588D8B75
:10C6E0009E8BAF8BB88F198A1A8A1B8A1C8A1D866B
:10C6F0001E861F86188A8091A111882369F010E098
:10C7000000E020E0AE014B5E5F4FBE016F5E7F4FE9
:10C71000CE010D960E947B5F6C960FB6F894DEBF3B
:10C720000FBECDBFDF91CF911F910F91FF90EF9082
:10C73000DF90CF900895C12CD12C80E8E82E80E4C2
:10C74000F82E58CF2F923F924F925F926F927F9226
:10C750008F929F92AF92BF92CF92DF92EF92FF9211
:10C760000F931F93CF93DF93CDB7DEB7E5970FB647
:10C77000F894DEBF0FBECDBF8DAB2091EB042CAB88
:10C7800021E02093EB0480910D058D3409F4B8C4A9
:10C79000843511F40C942378873409F091C1809189
:10C7A0000B0590910C058A31910509F432C208F00D
:10C7B00079C18430910508F030C12091E40A8230BB
:10C7C000910508F48EC1213009F091C111E0029762
:10C7D00009F010E00E944D2319821A821B821C82EC
:10C7E0001D821E821F82188682E50E9400238823F4
:10C7F00009F490C10E9488226B017C0120E030E0A6
:10C80000A9010F94841D882309F4EAC04090FA0C12
:10C810005090FB0C6090FC0C7090FD0C8091FE0C15
:10C820009091FF0CA091000DB091010D8CA79DA7D8
:10C83000AEA7BFA78090E50A9090E60AA090E70A0D
:10C84000B090E80A8091E90A9091EA0AA091EB0A77
:10C85000B091EC0A88AB99ABAAABBBABA501940134
:10C86000C301B2010F94841D81110DC028A939A9FB
:10C870004AA95BA96CA57DA58EA59FA50F94841DD3
:10C88000882309F4ADC0A3019201C501B4010F943E
:10C89000612420E030E040E05FE30F94EA1D68A7E8
:10C8A00079A78AA79BA72CA53DA54EA55FA568A93A
:10C8B00079A98AA99BA90F94612420E030E040E087
:10C8C0005FE30F94EA1D2B013C0120E030E0A90159
:10C8D000C701B6010F94841D881F8827881F181769
:10C8E00009F40FC180E090E0A0E8BFEB8CA79DA702
:10C8F000AEA7BFA728A539A54AA55BA5CA01B9015E
:10C900000F94EA1D4B015C01A3019201C301B20126
:10C910000F94EA1D9B01AC01C501B4010F94622480
:10C920000F9410274B015C01AC019B01C701B601BC
:10C930000F94612468AB79AB8AAB9BABA5019401E2
:10C94000C701B6010F9462249B01AC0168A979A9C3
:10C950008AA99BA90F94EA1D6B017C0120E030E0BD
:10C96000A9010F94C22687FDD1C0C701B6010F945B
:10C9700010276B017C01C301B2019058A5019401FD
:10C980000F945C252CA53DA54EA55FA50F94EA1D2F
:10C99000A70196010F94EA1D28A539A54AA55BA514
:10C9A0000F94622469837A838B839C83A50194010D
:10C9B00068A579A58AA59BA50F945C252CA53DA506
:10C9C0004EA55FA50F94EA1DA70196010F94EA1DDD
:10C9D000A30192010F9462246D837E838F839887D5
:10C9E00020E030E0A90169817A818B819C810F94DC
:10C9F000841D8111A3C020E030E0A9016D817E81FA
:10CA00008F8198850F94841D811198C00E94AE4D2E
:10CA100081E59DE00E94382A6AC08C30910509F4B6
:10CA2000A0C08531910509F462C0049709F048C09F
:10CA300080E50E940023C12CD12C7601882321F0AF
:10CA40000E946C1C6B017C0183E50E9400238823FB
:10CA500061F00E94882220E030E04AE754E40F941D
:10CA6000EA1D0F94D5256B017C010E9403C28091C1
:10CA7000A311811105C060E087E69DE00E94133498
:10CA80000E94C4F3C60ED71EE81EF91E0E94C4F30E
:10CA90006C197D098E099F0997FF29C080E00E94CB
:10CAA000B156F4CF8A32910509F400C260F48C319A
:10CAB000910509F4C9C008F4AFC04D9709F4F3C15A
:10CAC0000E94FBEF14C08B35910509F470C28C35C0
:10CAD000910509F470C28A35910591F71092640BA3
:10CAE00006C0213021F40E944D230E9400CFFDA9F1
:10CAF000F11102C00E944DF42CA92093EB040C9478
:10CB0000657080E090E0A0E8BFE3F0CEC12CD12CAE
:10CB1000760131CF89E40E940023882331F00E94FE
:10CB2000882269837A838B839C838AE40E94002312
:10CB3000882309F455CF0E9488224ECF412FBE0191
:10CB40006F5F7F4F85EE9AE00E94A0F40E94C4F3CD
:10CB50006093991170939A1180939B1190939C11FB
:10CB6000C6CF0F9486108111C2CF70E060E080E5DF
:10CB70000E940D238CA365E070E083E50E940D23E5
:10CB800088A363E070E084E50E940D238C8F40E071
:10CB900050E060ED70E482E50E94362369837A8379
:10CBA0008B839C838091080587FD04C080910905D3
:10CBB000837069F160E088E50E947A24182F60E0B4
:10CBC00089E50E947A2400E0811102E0012B109196
:10CBD000F90C812F0E94DD2460E085E40E947A2414
:10CBE00091E0892780934C029E01245E3F4FAE0165
:10CBF0004F5F5F4FBE01605E7F4FCE0184960E9403
:10CC0000462A10924C02812F0E94DD2470CF11E041
:10CC1000DCCF0E9425456BCF0F948610811167CF22
:10CC20008CE0EFE9F2E0DE01119601900D928A9519
:10CC3000E1F770E060E080E50E940D23BE016F5FC8
:10CC40007F4F0E94361953CF87E00E948DC5811116
:10CC500006C060E08FE40E947A24811148CF0E94D0
:10CC600003C210924C026091F90C8CE40E947A2469
:10CC7000682E80E00E94DD240E94C4F36093991125
:10CC800070939A1180939B1190939C11809147020D
:10CC900090914802A0914902B0914A028093D90430
:10CCA0009093DA04A093DB04B093DC0480916502D6
:10CCB000909166029093D8048093D70484E690E024
:10CCC000909366028093650281E08093A00A0E949F
:10CCD00049D48AE50E94B222782E88E50E94B222C9
:10CCE000082F89E50E94B222182F081307C0102FC1
:10CCF000701204C001E011E07724739482E50E9471
:10CD00000023882309F4C5C00E9488226CA37DA358
:10CD10008EA39FA320E030E0A9010F94841D8823F7
:10CD200049F0011103C0112309F48AC0CE01849691
:10CD30000E9497F1002309F47EC0112309F478C002
:10CD40001092FA0C1092FB0C1092FC0C1092FD0C3D
:10CD50001092FE0C1092FF0C1092000D1092010D1B
:10CD60000E94A0C7E2EDF5E1C590D590E590F49062
:10CD7000E6EDF5E185909590A590B490A701960118
:10CD8000C501B4010F94841D87FF88C0A7019601D7
:10CD9000C501B4010F945C259B01AC010F94EA1D01
:10CDA00020E030E040E85FE30F9462240F94102706
:10CDB00020E030E048E452E40F94EA1D68A379A330
:10CDC0008AA39BA320E030E040EC5FE3C501B401FF
:10CDD0000F94EA1D905869837A838B839C8320E0AB
:10CDE00030E040EC5FE3C701B6010F94EA1D9058B4
:10CDF0006C8F7D8F8E8F9F8FAE01405E5F4FBE0127
:10CE00006F5F7F4FCE014C960E9432C70E9421D6A1
:10CE10001092FA0C1092FB0C1092FC0C1092FD0C6C
:10CE20001092FE0C1092FF0C1092000D1092010D4A
:10CE300080E00E942CD2112319F081E00E942CD2B4
:10CE4000772019F082E00E942CD20E94A0C7809126
:10CE50009F0A8093A00A862D0E94DD248091D90428
:10CE60009091DA04A091DB04B091DC048093470236
:10CE700090934802A0934902B0934A028091D7044C
:10CE80009091D80490936602809365020E9481D3AA
:10CE90002ECE60E070E080E890E438CFA5019401E8
:10CEA000C701B60177CF0E94727B21CE8091E40A40
:10CEB000813009F01CCE89E40E940023082F10E085
:10CEC000882319F00E948422182F8AE40E940023EC
:10CED000F82E882369F00E948422002309F45FC0A1
:10CEE000153008F459C080E79DE00E94382AFFCD34
:10CEF00080E00111F5CF90E1EAEFFCE0A5EEBAE0A9
:10CF000001900D929A95E1F7002391F094E01902B7
:10CF1000F0011124E159FB4E4081518162817381FE
:10CF20004093E50A5093E60A6093E70A7093E80A93
:10CF3000FF2091F0A4E08A02F0011124E55AFB4E93
:10CF400080819181A281B3818093E90A9093EA0A5A
:10CF5000A093EB0AB093EC0A40E050E0BA0186E4FB
:10CF60000E9436236B017C0120E030E0A9010F9480
:10CF7000C2261816C4F420E030E040E752E4C701AE
:10CF8000B6010F945C2569837A838B839C83CE01E1
:10CF900001960E94C1D1ABCDFF2009F4ACCF853002
:10CFA00008F4A9CFA0CF60E070E0CB01ECCF8FE018
:10CFB0008093640B9CCD80910A05882389F1893088
:10CFC00009F095CD7BEAA72E72E0B72EEAEFCE2EC0
:10CFD000ECE0DE2EE12C00E010E0F50181915F0134
:10CFE0000E940023F82E882369F0133011F4082FD3
:10CFF000FE2C0E948822D6016D937D938D939C9385
:10D000001397EF2C1F5FB4E0CB0ED11C143029F71F
:10D01000EE2009F457C00E94A0C70E9481D367CDBB
:10D020006BEAC62E62E0D62EF12CE12C00E010E077
:10D03000F60181916F010E940023382E8823D9F1D7
:10D040000E9488224B015C01133059F0F701E55B27
:10D05000F34F20813181428153810F9461244B0130
:10D060005C01F701E650F34F208131814281538109
:10D07000C501B4010F9461242B013C012DEB37E372
:10D0800046E855EB0F94C22687FD0AC02DEB37E327
:10D0900046E855E3C301B2010F94841D18165CF4F1
:10D0A0001330C1F48092060D9092070DA092080DE6
:10D0B000B092090D032D1F5FF4E0EF0EF11C143048
:10D0C00009F0B6CF002309F4A8CF86E09DE00E94C6
:10D0D00014C2A3CF97012059344F5901A3019201E3
:10D0E000D5016D917D918D919C910F946224F501F4
:10D0F0006083718382839383812F0E946DC5DBCF10
:10D1000080910B0590910C058737910511F40C94D3
:10D11000DF7108F06CC28D34910509F4C3C608F0C4
:10D12000D1C08A31910509F4E5C508F092C0843177
:10D13000910509F42BC508F06FC08131910509F400
:10D14000EAC408F042C0029708F0BACC80E50E9419
:10D150000023C12CD12C7601882321F00E946C1C65
:10D160006B017C0183E50E940023882361F00E940B
:10D17000882220E030E04AE754E40F94EA1D0F943F
:10D18000D5256B017C010E9403C280910E05909110
:10D190000F05892B09F4BAC40E94A1F080910B05F8
:10D1A00090910C0561E97DE0892B11F469E87DE03F
:10D1B00030E020E049E95DE082E00E94423540E055
:10D1C000C701B6010E94C86092CC429709F078CCA2
:10D1D00083E50E940023882311F40C943C710E9483
:10D1E000C4F36093991170939A1180939B1190935B
:10D1F0009C110E94882220E030E04AE754E40F941A
:10D20000EA1D0F94D525609308027093090280935C
:10D210000A0290930B026BCC8731910509F4EBC4A1
:10D2200070F48531910509F4E2C4469709F048CCC1
:10D2300080918E1482FD5BCC0E94DE9158CC8831A7
:10D24000910509F4EDC4499709F03ACC0E94D562E2
:10D250004ECC8F31910509F4F2C5D0F48C31910593
:10D2600009F4B5C508F459C58D31910509F4B7C560
:10D270004E9709F025CC80918E1483FF38CC0E9404
:10D28000E1EF80910E0590910F050E94CD952FCC76
:10D290008934910509F4F2C550F48032910509F4FE
:10D2A000A5C5819709F00CCC0E94EC5520CC8B349D
:10D2B000910509F4F3C58C34910509F001CC0E9465
:10D2C00085D715CC8B36910509F418C708F0F9C03D
:10D2D0008435910509F47CCF30F58135910509F449
:10D2E000ABC790F48E34910509F0EACB70E060E0B2
:10D2F00083E50E941B238E34910509F0D8C50E9456
:10D300005EB10F945710F3CB8235910509F4ACC789
:10D310008335910509F0D4CB8091640B8F7E8062B8
:10D320008093640BE4CB8836910509F444C608F079
:10D330009AC08535910509F4E2C78C35910509F04D
:10D34000BFCB0E949B4E87FDD2CB8091060584FD0A
:10D350000AC08091080587FD06C080910905837089
:10D3600011F40C94AC711BEAC12E12E0D12E08E925
:10D37000E02E0CE0F02E10E0D6018D916D010E94A0
:10D380000023882309F465C0133009F0DDC70E942B
:10D3900088224B015C0120E030E040EA51E40F9428
:10D3A000841D87FF4EC0A50194016091B80C709157
:10D3B000B90C8091BA0C9091BB0C0F945C252B0199
:10D3C0003C01AC019B016091F0087091F1088091E3
:10D3D000F2089091F3080F94EA1D6093F00870939F
:10D3E000F1088093F2089093F308A30192016091F1
:10D3F000C80C7091C90C8091CA0C9091CB0C0F9401
:10D40000EA1D6093C80C7093C90C8093CA0C90936A
:10D41000CB0C6091730570917405809175059091A6
:10D4200076050F94891DA30192010F94EA1D0F94B4
:10D43000D52560937305709374058093750590935B
:10D4400076058092B80C9092B90CA092BA0CB0926A
:10D45000BB0C1F5FF4E0EF0EF11C143009F08CCF11
:10D460000E94DFC144CB8936910509F41CC68A3677
:10D47000910509F025CB6091F80C80E50E942A23E4
:10D48000F82E91E0981708F432CB81E40E94B22282
:10D490000FEF10E0882341F0E091F80CF0E0EB5939
:10D4A000F44F6081062F10E083E50E94002388235B
:10D4B00019F00E94D91C8B01B8018F2D0E94CEA0BB
:10D4C00016CB8037910509F412CB08F04EC08D368B
:10D4D000910509F49FC508F40ACB8E36910509F42D
:10D4E0001CC68F36910509F0EBCA83E50E94B22273
:10D4F000882331F060E083E50E942A238093630B48
:10D500000E94974E81E99EE00E94382A8091630B29
:10D51000882309F415C610E000E020E08091630B39
:10D5200090E0B0E0A0E0002E04C0B695A7959795D6
:10D5300087950A94D2F780FF12C0FF24F394F20E6D
:10D54000222319F08CE20E94FF29F801EE0FFF1F41
:10D55000E957F14F859194910E94382A2F2D0F5F42
:10D560001F4F05301105D1F6FFC38337910509F42C
:10D57000F8C678F48137910509F4E5C5823791053D
:10D5800009F09ECA0E9425ED80EC92E10E94E3A082
:10D59000AECA8537910509F4E8C68637910509F0CA
:10D5A0008FCA00910E0510910F0594E0F12C40E018
:10D5B000915009F4F3C6F8018081282F2B7F213484
:10D5C00009F0E5C62181213309F0E8C6813409F468
:10D5D000F3C6853409F441E098012E5F3F4F89017D
:10D5E0002F5F3F4FF80180818032C9F3E1CF803354
:10D5F00031E0930711F40C94FD7408F0C1C18D3C27
:10D60000910509F48AC708F0D0C08B39910509F457
:10D61000ECC508F58937910509F4DEC608F4D3C6D0
:10D620008D37910509F412CE8C38910509F048CA5E
:10D630008091630B83FD5BCA83E50E9400238823EE
:10D6400009F455CA0E9484220E94161A61E080E003
:10D650000F949E114CCA893C910509F4C9C608F083
:10D660006BC08E3B910509F48DC5883C910509F08E
:10D6700027CA0E949B4E182F87FD39CAF0906F0B66
:10D6800084E40E940023082F882309F4ADC60E9479
:10D6900088226B017C0120E030E0A9010F94841DF9
:10D6A000882309F4A3C624E01202F0011124E959E9
:10D6B000F44FC082D182E282F38220E030E0A901FF
:10D6C0006091670B7091680B8091690B90916A0B68
:10D6D0000F94841D81110CC080E090E0A0EEBFE3A8
:10D6E0008093670B9093680BA093690BB0936A0BC0
:10D6F00020E030E0A90160916B0B70916C0B809180
:10D700006D0B90916E0B0F94841D81110CC080E005
:10D7100090E0A0EEBFE380936B0B90936C0BA09313
:10D720006D0BB0936E0B602F83E50E947A2480937B
:10D730006F0B0E94AEC4DBC98B3C910509F482C615
:10D740008C3C910509F0BCC98091070587FD9DC6F9
:10D75000809108058E7009F098C64091CC0C5091CC
:10D76000CD0C6091CE0C7091CF0C82ED9EE00E94AA
:10D7700018364091D00C5091D10C6091D20C709120
:10D78000D30C8FEC9EE00E9418364091D40C50913F
:10D79000D50C6091D60C7091D70C8EE09BE10E9465
:10D7A00018368AE00E94FF29A2C98D3D910511F427
:10D7B0000C94E07308F09FC0833D910509F434C7D1
:10D7C00008F050C0ECE7EE2EEBE0FE2E10E08E3CB1
:10D7D000910509F075C988E5810F0E94B22288235E
:10D7E00051F00E948822F7016083718382839383C2
:10D7F000812F0E946DC51F5FF4E0EF0EF11C133006
:10D8000051F78091080587FD08CC80910905837048
:10D8100009F003CC40917C0B50917D0B60917E0B05
:10D8200070917F0B84E19FE00E9418364091800B3D
:10D830005091810B6091820B7091830B8BEB9BE27B
:10D840000E9418364091840B5091850B6091860B95
:10D850007091870B88EB9BE20E9418368AE00E9449
:10D86000FF2945C9893D910509F4A6C78C3D91055D
:10D8700009F026C982E40E94B222882341F08091F7
:10D8800065029091660290930D0280930C0282E5EE
:10D890000E94B222882341F080910C0290910D02E7
:10D8A000909366028093650283E50E94002388239B
:10D8B00031F00E94842290936602809365028091E9
:10D8C000060590910705A0910805B0910905892BDF
:10D8D0008A2B8B2B09F00BC960916502709166024F
:10D8E00084E49FE00E943A3685E20E94FF298AE0A4
:10D8F0000E94FF29FCC88D32B1E09B0711F40C9403
:10D900007B74F0F48232F1E09F0709F48CC78C320B
:10D91000914009F0D5C864E071E083E50E940D23D1
:10D920008C0168EE73E080E50E940D23893823E1C5
:10D93000920710F088E893E1B8010E94672FD7C8DA
:10D940008E3231E0930711F40C9471758F3291404F
:10D9500009F0B6C870E060E085E40E941B23F82E51
:10D960003FEF831711F40C94E675882311F40C949F
:10D97000B7758EEC9FE00E94382A0E94D0E6B7C8A7
:10D98000883FB1E09B0711F40C94A47608F048C0DE
:10D99000853AF1E09F0711F40C94E975D0F48A39C7
:10D9A00031E0930709F4A3C838F48039914009F0B5
:10D9B00087C80E9403C29BC88D39E1E09E0711F41D
:10D9C0000C94FF77843A914009F07AC80E94CF4FB7
:10D9D0008EC8853F21E0920711F40C949C7668F480
:10D9E0008C3AA1E09A0711F40C94ED75843F9140B4
:10D9F00009F066C80E94D4AD7AC8863FE1E09E0770
:10DA000011F40C94A076873F914009F059C861E069
:10DA100083E50E947A2491E089270E94C7DC67C8C9
:10DA20008C3623E0920709F462C808F58B35A2E032
:10DA30009A0711F40C94C77668F48C30E2E09E07E4
:10DA400011F40C94B6768835924009F039C80E94DA
:10DA5000AC614DC88D3B22E0920711F40C944777DE
:10DA60008E3B924009F02CC80E94C14E40C8873EB0
:10DA7000A3E09A0711F40C94EF77C0F48438E3E044
:10DA80009E0711F40C944B77803A934011F00C945C
:10DA9000606520910E0530910F0590918E14926073
:10DAA00090938E14C9010E94359621C8883E23E0C8
:10DAB000920711F40C941878893E934011F00C945D
:10DAC00060658091841481110C941C780E948F24CD
:10DAD0000E943AF90E942FD66D3371058105910598
:10DAE00020F083E990E10E9472788FE890E10E9433
:10DAF000727884EE80935D058BE790E10E94382A6E
:10DB000087E790E10E9472780C94776582EA9DE045
:10DB10000E94EB1943CB8091060584FD18C08091CB
:10DB2000080587FD14C080910905837081F460E0C9
:10DB300085EB9DE00E9413345F988A9880910801DC
:10DB40008170809306010F94DB100C94776588E553
:10DB50000E94B22281115F9889E50E94B222811150
:10DB60008A988AE50E94B222882329F080910801D0
:10DB700081708093060185E40E94B222882311F40B
:10DB80000C9477650F94DB100C94776580918E145C
:10DB900083FF25C08DEC9DE00E94382A80918E1471
:10DBA00083FF17C08EEA94E10E9455928BE1EEEA62
:10DBB000F4E1DE01119601900D928A95E1F770E093
:10DBC00060E0CE0101960E947197CE0101960E94FD
:10DBD000B7248EEB9DE00E94382A0C9477650E9452
:10DBE000974E8EED9DE00E94382A0C9477650E9436
:10DBF000EF910C94776580910E0590910F05FC01D3
:10DC00002191222331F02032D9F7DF0111971C92A4
:10DC1000F7CF60E00E947E9610925D050C947765C8
:10DC200083E50E940023882321F00E94D91C0E94D2
:10DC3000001B84E50E9400238823A9F00E94D91CC0
:10DC40006B017C010E94D8D6C092C708D092C80848
:10DC5000E092C908F092CA08CD28CE28CF2819F042
:10DC600081E08093A2118091A1118823F9F080E0D6
:10DC700090E0A0EAB1E489839A83AB83BC831C8ED5
:10DC80001D8E1E8E1F8E18A219A21AA21BA210E0B2
:10DC900000E020E0AE014F5F5F4FBE01645E7F4F4A
:10DCA000CE0180960E947B5F0C9477650E94A5252B
:10DCB000882381F00E94CC890E94F3D68BEC9BE0F4
:10DCC0000E947D911092030E1092040E1092050E88
:10DCD0001092060E61E082E794E10E94E0334FE586
:10DCE00054E168EE7DE085E00E94C7E60F9457108E
:10DCF0000C94776580918E1483FD02C00C94776537
:10DD000083E50E940023882311F40C9477650E9418
:10DD1000D91C0E94001B0C94776583E40E94B222F8
:10DD2000882361F18EEF9DE00E94382A8091F515DD
:10DD30008823F9F0BE016F5F7F4F82EF95E10E946B
:10DD40001091CE0101960E94C28DCE0101960E94D3
:10DD50009B9280910612882339F080E20E94FF296D
:10DD600086E092E10E94C28D8AE00E94FF290C9415
:10DD7000776584EF9DE00E94382AF6CF83E50E9404
:10DD80000023882301F10E94E91C182F8C3308F02E
:10DD90008CE38093E1040E94C4F36B017C01212F8A
:10DDA00030E0A8EEB3E00F941C24C60ED71EE81E88
:10DDB000F91EC092DD04D092DE04E092DF04F092FE
:10DDC000E0040C9477650E948A890C9477658091B1
:10DDD0000E0590910F050E9435960C947765809101
:10DDE0008E148E7F80938E140C94776580918E14A0
:10DDF00082FD0E9403C280918E1483FD02C00C94A8
:10DE0000776560E080E50E947A24182F682F809162
:10DE10000E0590910F050E947E9683E50E940023D7
:10DE2000882321F00E94D91C0E94001B0E94CC89EB
:10DE300011110C9477650E94F3D60C9477650E94BB
:10DE40002FD66C8F7D8F8E8F9F8FBE016F5F7F4F20
:10DE5000CE014C960E94211ACE0101960F941F10FC
:10DE60000E94974EBE016F5F7F4F8DE09EE00E9443
:10DE7000C6538AE00E94FF290C94776580E50E94D2
:10DE8000B222882311F40C9477650E94E91C853630
:10DE900008F084E680935D050C9477650E94F3D6C4
:10DEA0000C94776581E00E9461D60C94776588E7D1
:10DEB0009EE00E94382A60918F0A7091900A8FE646
:10DEC0009EE00E9406366091910A7091920A82E665
:10DED0009EE00E94063660918F0A7091900A8091B0
:10DEE000910A9091920A681B790B8091A21181503E
:10DEF00021E030E0823010F030E020E0621B730B54
:10DF000087E59EE00E9406368AE00E94FF298FE4A2
:10DF10009EE00E94382A8091930A9091940AA091E1
:10DF2000950AB091960A8C8F9D8FAE8FBF8FBE01E0
:10DF30006F5F7F4FCE014C960E94211ABE016F5F2A
:10DF40007F4F82E49EE00E94C6538091970A909191
:10DF5000980AA091990AB0919A0A8C8F9D8FAE8FE2
:10DF6000BF8FBE016F5F7F4FCE014C960E94211A7A
:10DF7000BE016F5F7F4F82E39EE00E94C65320E0A8
:10DF800030E04AE754E460919B0A70919C0A8091CA
:10DF90009D0A90919E0A0F945C25AB01BC018AE119
:10DFA0009EE00E9418368DE60E94FF298AE00E94BA
:10DFB000FF290C9477658091630B83FF02C00C945A
:10DFC00077650E949B4E182F87FF02C00C947765DF
:10DFD00083E50E9400238823C9F00E948422212F18
:10DFE000110F330BF901EE0FFF1FE65FF64F918320
:10DFF00080834091F80C4217130611F00C9477655A
:10E000000E9485C161E080E00F949E110F9467111A
:10E010000C9477658091630B83FF02C00C94776545
:10E020000E949B4E182F87FF02C00C94776583E5F2
:10E030000E940023082F811105C082E50E94002361
:10E04000882321F30E948422212F012E000C330B00
:10E05000F901EE0FFF1FE65FF64F91838083409139
:10E06000F80C4217130611F00C9477650E9485C1D5
:10E0700061E081E00F949E1120915412309155126D
:10E0800080915212909153128217930714F001114C
:10E0900002C00E9424E80F946711602F812F0E9414
:10E0A000E79A0C9477650E949B4E182F87FD0AC053
:10E0B00080E89EE00E94382A812F0E94FC988AE026
:10E0C0000E94FF298CA98093EB04E5960FB6F89483
:10E0D000DEBF0FBECDBFDF91CF911F910F91FF909B
:10E0E000EF90DF90CF90BF90AF909F908F907F90F8
:10E0F0006F905F904F903F902F9008956091F80C33
:10E1000080E50E942A23823010F00C94776570E03D
:10E1100060E00E94CEA00C9477658EE40E940023FC
:10E12000882311F40C9477650E94D91C60938C0DA0
:10E1300070938D0D80938E0D90938F0D0C94776559
:10E1400083E89EE018CE83E50E940023882369F0CF
:10E150000E94E91C8D3320F4809307020C947765AC
:10E160008CE3809307020C9477650E94974E609130
:10E17000070288E99EE00E9410368AE00E94FF298B
:10E180000C9477658091630B83FF02C00C947765D4
:10E1900083E50E940023182F8823E9F00E9484223F
:10E1A0000E94161A60E081E00F949E112091EA11FE
:10E1B0003091EB118091E8119091E911821793074A
:10E1C0008CF08FE99EE060E00E941334812F0E9462
:10E1D0006F990C94776582E50E9400238111DECF50
:10E1E0000C9477658EEA9EE0EECF83E50E940023D3
:10E1F000882311F40C9477650E94E91C182F8C3346
:10E2000008F08CE38093E6040E94C4F36B017C0168
:10E21000212F30E0A8EEB3E00F941C24C60ED71EC9
:10E22000E81EF91EC092E204D092E304E092E404F6
:10E23000F092E5040C9477650E94CC9C0E94C3C3C5
:10E2400081E00E9461D60E94E22568EE73E080E0E2
:10E2500090E00E943D250E94331960E08DEB9EE026
:10E260000E9413340C9477658091640B8F7D8061DC
:10E270008093640B0C9477658091060584FD0CC037
:10E280008091080587FD08C080910905837021F4FD
:10E290000E94C3C30C9477650E9403C288E50E9464
:10E2A000B222882331F05F9A8091970C8E7F809301
:10E2B000970C89E50E94B222882331F08A9A8091D6
:10E2C000970C8D7F8093970C8AE50E94B222882359
:10E2D00059F08091080180958170809306018091AA
:10E2E000970C8B7F8093970C85E40E94B222882341
:10E2F00011F40C9477650E9430190C94776583E5CE
:10E300000E94B222882311F40C9477650E94C4F312
:10E310006093991170939A1180939B1190939C1123
:10E320000E94882220E030E04AE754E40F94EA1D7E
:10E330000F94D5256093E7047093E8048093E90473
:10E340009093EA040C9477650E948822F701648B0D
:10E35000758B868B978B7DC881E00E94A6EF0C940D
:10E3600077650E943F330C94776580910E059091FC
:10E370000F05009741F0DC012C91222321F00F942E
:10E380001F100C9477650F9457100C9477658035A7
:10E3900029F4818180538A3008F41EC941110E94FA
:10E3A000974EFF2021F08CEC9EE00E94382AC80195
:10E3B0000E94062A0C947765FF24F3940DC90E94ED
:10E3C0002DD40C94776581E08093A00A80939F0AF6
:10E3D0000E9449D40C9477651092A00A10929F0A6B
:10E3E0000E9449D40C9477650F2D9DC980E09FC988
:10E3F0000E949B4E87FF02C00C9477650BEA12E0E7
:10E40000A8E9EA2EACE0FA2EBFEACB2EB2E0DB2E72
:10E41000D8018D918D010E94B222882359F00E946B
:10E4200088220F94D525F7016083718382839383BB
:10E430000E9491C1F4E0EF0EF11CC016D10641F725
:10E440000C9477650E949B4E87FF02C00C94776501
:10E45000FBEAEF2EF2E0FF2E10E000E0D7018D91F5
:10E460007D010E94B222882349F00E948822F8018F
:10E47000E856F34F64A375A386A397A30C5F1F4FC1
:10E480000031110559F70C94776583E50E9400234C
:10E49000882391F00E9488226093CC0C7093CD0C5D
:10E4A0008093CE0C9093CF0C6093D40C7093D50CCA
:10E4B0008093D60C9093D70C80E50E94002388238C
:10E4C00051F00E9488226093CC0C7093CD0C809305
:10E4D000CE0C9093CF0C82E50E940023882351F04C
:10E4E0000E9488226093D00C7093D10C8093D20C40
:10E4F0009093D30C84E50E940023882311F40C949C
:10E5000077650E9488226093D40C7093D50C809319
:10E51000D60C9093D70C0C94776580910605827188
:10E5200051F4809108058C7831F48091090583704D
:10E5300011F40C94776582E40E94B222882351F092
:10E540000E946C1C6093A80C7093A90C8093AA0C79
:10E550009093AB0C83E50E94B222882351F00E9475
:10E5600088226093D80C7093D90C8093DA0C909326
:10E57000DB0C84E50E94B222882351F00E9488229D
:10E580006093DC0C7093DD0C8093DE0C9093DF0CB9
:10E5900088E50E94B222882351F00E94882260936D
:10E5A000E4087093E5088093E6089093E70889E50E
:10E5B0000E94B222882351F00E9488226093E808CA
:10E5C0007093E9088093EA089093EB088AE50E942B
:10E5D000B2228823B1F00E9488226093EC087093E5
:10E5E000ED088093EE089093EF082DEC3CEC4CEC9A
:10E5F0005DE30F94841D181624F082EE9EE00E94C5
:10E60000382A85E40E94B222882311F40C9477659D
:10E610000E9488226093F0087093F1088093F208BA
:10E620009093F3080C94776540904B0C50904C0CF1
:10E6300060904D0C70904E0C20914D0230914E0226
:10E6400040914F0250915002C301B2010F946224D5
:10E6500068A779A78AA79BA780904F0C9090500C31
:10E66000A090510CB090520C209151023091520266
:10E670004091530250915402C501B4010F94622499
:10E680006CA77DA78EA79FA7C090530CD090540C69
:10E69000E090550CF090560C2091550230915602A6
:10E6A0004091570250915802C701B6010F9462245D
:10E6B00068AB79AB8AAB9BAB2091590230915A027F
:10E6C00040915B0250915C02C301B2010F9462243D
:10E6D0002B013C0120915D0230915E0240915F026E
:10E6E00050916002C501B4010F9462244B015C019A
:10E6F0002091610230916202409163025091640264
:10E70000C701B6010F9462246B017C010E94974EF1
:10E7100084E39FE00E94382A83E50E94B222882386
:10E7200021F00E94FD1C80934B0280914B028823B4
:10E7300009F43FC08FE19FE00E94382A8CE29FE0FD
:10E740000E94382A48A559A56AA57BA58FE79AE1BA
:10E750000E9418364CA55DA56EA57FA58BEB9BE2AC
:10E760000E94183648A959A96AA97BA988EB9BE29F
:10E770000E9418368AE29FE00E94382A82E29FE0D7
:10E780000E94382AB301A2018FE79AE10E9418364D
:10E79000B501A4018BEB9BE20E941836B701A601DC
:10E7A00088EB9BE20E9418368AE00E94FF290C94B5
:10E7B00077658BE19FE0C0CF0E9423420C94776580
:10E7C0000E949B4E082F87FF02C00C94776583E55B
:10E7D0000E940023882341F00E948422BC01802FE4
:10E7E0000E947D1F0C9477650E94974E002E000CAE
:10E7F000110B85E40E94FF2980E3800F0E94FF290E
:10E80000000F111FF801EA5CFD4F6081718188E4FF
:10E810009FE00E943A3685E20E94FF298AE00E942A
:10E82000FF290C9477658AE50E940023882339F13B
:10E830000E94882220E030E040E050EC0F94841DDC
:10E8400087FD48C00E94882220E030E040E050E48C
:10E850000F94C22618160CF442C00E948822209100
:10E86000B40C3091B50C4091B60C5091B70C0F948C
:10E87000EA1D0F94CE25CB010E94FDF305C083E570
:10E880000E9400238111D4CF8091080587FD2CC000
:10E8900080910905837041F50E94974E4091E008F0
:10E8A0005091E1086091E2087091E3088BE59FE0E8
:10E8B0000E9418368AE00E94FF2960919D11709194
:10E8C0009E1180E59FE00E943A368AE00E94FF296F
:10E8D0000C94776560E070E080E090ECC0CF60E081
:10E8E00070E080E090E4BBCF82E50E94B22281110B
:10E8F000D3CF0C94776560E085E40E942A238111D0
:10E9000074C080E50E94B222882351F00E948822C0
:10E9100060935712709358128093591290935A1221
:10E9200089E40E94B222882381F00E9488222CEA86
:10E9300035EC47E25EE30F94EA1D60935B1270933F
:10E940005C1280935D1290935E1284E40E94B22266
:10E95000882381F00E9488222CEA35EC47E25EE3AE
:10E960000F945C2560935F12709360128093611224
:10E97000909362120E94974E4091571250915812F4
:10E980006091591270915A1280E79FE00E941836E8
:10E990002CEA35EC47E25EE360915B1270915C1209
:10E9A00080915D1290915E120F945C25AB01BC01C9
:10E9B0008CE69FE00E9418362CEA35EC47E25EE3D5
:10E9C00060915F1270916012809161129091621259
:10E9D0000F94EA1DAB01BC0188E69FE00E94183647
:10E9E0008AE00E94FF290C9477650E94AE4D84E76F
:10E9F0009FE00E94382A0C94776580E50E94B2223D
:10EA0000882351F00E9488226093ED117093EE11DB
:10EA10008093EF119093F01189E40E94B222882331
:10EA200081F00E9488222CEA35EC47E25EE30F94E5
:10EA3000EA1D6093F1117093F2118093F31190939A
:10EA4000F41184E40E94B222882381F00E9488227B
:10EA50002CEA35EC47E25EE30F945C256093F511F8
:10EA60007093F6118093F7119093F8110E94974ECE
:10EA70004091ED115091EE116091EF117091F011F4
:10EA80008EE89FE00E9418362CEA35EC47E25EE300
:10EA90006091F1117091F2118091F3119091F41144
:10EAA0000F945C25AB01BC018AE89FE00E941836F8
:10EAB0002CEA35EC47E25EE36091F5117091F611B6
:10EAC0008091F7119091F8110F94EA1DAB01BC01F0
:10EAD00086E89FE00E9418368AE00E94FF290C9485
:10EAE000776583E50E94B222182F882369F00E947F
:10EAF00084229C0190933B0280933A0291E0232B65
:10EB000009F090E09093620B80E50E94B222882386
:10EB100061F020913A0230913B02232B11F00E94C8
:10EB2000FD1C8093620B0C94776511110C94776532
:10EB30000E94974E8EEA9FE00E94382A8091620BD5
:10EB4000882391F086E99FE00E94382A60913A027A
:10EB500070913B028DE99FE00E943A3689E99FE07F
:10EB60000E94382A0C94776582E99FE0EDCF04EB90
:10EB700010E083E50E940023882319F00E9484227C
:10EB80008C0165E070E083E40E941B23E82E60E0C6
:10EB900085E50E947A24D82E60E081EC9FE00E94F7
:10EBA0001334B801110F880B990B0F948B1D6983D7
:10EBB0007A838B839C832D2D4E2D6F2DCE01019654
:10EBC0000E94C3D70F9457100C94776506E410E0A9
:10EBD000D0CF0E94B24D0C9477650F9486108111AE
:10EBE0000C94776561EAC62E65E1D62E8AEF9CE02B
:10EBF00099A788A7DE0111961D017D0110E000E0B4
:10EC0000F6016591759185919491E8A5F9A581909A
:10EC10009190A190B190F9A7E8A7A50194010F9454
:10EC200061242B013C01D7014D925D926D927C9243
:10EC3000139720E030E040EA51EC0F94C22687FDA4
:10EC40000AC020E030E040EA51E4C301B2010F9471
:10EC5000841D18167CF4F801E959F44DE4911E1650
:10EC60004CF4B7FAB094B7F8B094F701808291826F
:10EC7000A282B382D7018D909D90AD90BD907D0111
:10EC800020E030E040EA51ECC501B4010F94C22607
:10EC900087FD3FC020E030E040EA51E4C501B40107
:10ECA0000F94841D1816ACF10F5F1F4FB4E0CB0E0C
:10ECB000D11C0330110509F0A3CF5CE7E52E5BE022
:10ECC000F52E10E0F10181919191A191B1911F0177
:10ECD000F70181939193A193B1937F01812F0E94BA
:10ECE0006DC51F5F133071F70E9481D360E082EF22
:10ECF0009FE00E94133463E972E084E690E00E9492
:10ED0000672F6AEB72E084E690E00E94672F0C9414
:10ED100077650E94AE4D80E190E10E94382A61E063
:10ED200082E090E10E94133468E270E088EC90E0A9
:10ED30000E94672F0C9477650E9415E40C94776508
:10ED40000E9454D40C9477652093F4080E9409E43F
:10ED50001092F408882311F40C9477650E94974E62
:10ED60008EE290E10E94382A0C94776580918E148F
:10ED700082FF05C0806480938E140C94776583FDB8
:10ED800002C00C9477650E94E1EF0C9477650E94B5
:10ED90009B4E082F87FF02C00C94776585E50E9483
:10EDA000B222882359F10E9488224B015C01E02E97
:10EDB000002E000CFF0820E030E0A9010F94C226CD
:10EDC00087FF04C0B7FAB094B7F8B09420E030E8F9
:10EDD0004BE354E4C501B4010F94C226970143E00C
:10EDE000220F331F4A95E1F72153374F1816D4F1FC
:10EDF000D9018D929D92AD92BC9213978CE40E94A2
:10EE0000B222882311F40C9477650E9488226B014A
:10EE10007C01002E000C110B20E030E0A9010F94C2
:10EE2000C22687FF04C0F7FAF094F7F8F09420E0C8
:10EE300030E84BE354E4C701B6010F94C2269801B1
:10EE400093E0220F331F9A95E1F72153374F18169D
:10EE50009CF0D9011496CD92DD92ED92FC92179719
:10EE60000C94776580E090E8ABE3B4E4F90180832B
:10EE70009183A283B383C2CF80E090E8ABE3B4E494
:10EE8000F90184839583A683B7830C9477650E94E8
:10EE9000795E0C9477656091F80C70E084E50E94CF
:10EEA0001B23823080F08FE30E94FF2984E50E94BB
:10EEB000FF2984E490E10E94382A89E390E10E94CE
:10EEC000382A0C94776599278C01000F111F000FC9
:10EED000111FF801EC5CF64F80809180A280B38016
:10EEE0008BE40E940023882339F10E9488226B0161
:10EEF0007C0120E030E0A9010F94C22687FD0AC002
:10EF000020E030E040E251E4B601C7010F94841DD7
:10EF10001816A4F48FE30E94FF298BE40E94FF29B6
:10EF200084E490E10E94382A8CE390E10E94382A20
:10EF300089E390E10E94382A640175019601A701D6
:10EF4000B401C5010F94841D882359F00E9403C2A7
:10EF5000F801EC5CF64FA601B70140835183628350
:10EF600073838091060590910705A0910805B091E3
:10EF70000905892B8A2B8B2B11F00C9477650E9445
:10EF8000974E88E590E10E94382A80E20E94FF298E
:10EF900080E30E94FF298AE30E94FF2960913409DF
:10EFA00070913509809136099091370942E00E94AD
:10EFB000589880E20E94FF2981E30E94FF298AE39A
:10EFC0000E94FF29609138097091390980913A09AE
:10EFD00090913B0942E00E9458980C94B46E81E0F5
:10EFE0008093E40A1092E31160E083E50E947A24A2
:10EFF00081110C9477650E94F4EA0C94776583E59F
:10F000000E94B222882341F00E94FD1C8093DF08F9
:10F010000E9497240C9477650E94974E82E690E1B7
:10F020000E94382A8091DF080E94FA350C94776597
:10F030000E94E4780C9477650E947CF981110C940D
:10F0400077650C94666D10910B050E94C4F3609374
:10F05000991170939A1180939B1190939C11812F19
:10F06000012E000C990B2091F80C2817190651F06D
:10F0700060E083E50E947A24682F812F0E94A2C756
:10F080000C94776581E0F8CFDF92EF92FF920F93B7
:10F090001F93CF93DF93EC01E090F80AF090F90A08
:10F0A0008AE0D82E6AE070E0CE010F94B0278C0180
:10F0B000009711F0FC011082CE010E94131E81E026
:10F0C0000E94A2630115110519F0E801D992EACF57
:10F0D000C701DF91CF911F910F91FF90EF90DF90CB
:10F0E0000C94131E4F925F926F927F928F929F9219
:10F0F000AF92BF92CF92DF92EF92FF920F931F9346
:10F10000CF93DF93CDB7DEB77C014DB65EB660908E
:10F11000F80A7090F90A8DB69EB66AE070E0C701F1
:10F120000F94BF1C6C018C010E191F09892B21F44F
:10F13000C7010F94D11C8C01C80101962DB73EB7B1
:10F14000281B390B0FB6F8943EBF0FBE2DBF8DB7ED
:10F150009EB701965C01A801B7010F94F21CF5015E
:10F16000E00FF11F1082C5010E94131E81E00E9472
:10F17000A263C114D10451F076019FEFE91AF90A94
:10F180000FB6F8949EBE0FBE8DBEC5CF0FB6F894D5
:10F190009EBE0FBE8DBEC3010E94131E0FB6F89413
:10F1A0005EBE0FBE4DBEDF91CF911F910F91FF90BC
:10F1B000EF90DF90CF90BF90AF909F908F907F9017
:10F1C0006F905F904F9008952F923F924F925F9271
:10F1D0006F927F928F929F92AF92BF92CF92DF9267
:10F1E000EF92FF920F931F93CF93DF93CDB7DEB7CC
:10F1F000C059D1090FB6F894DEBF0FBECDBF0E9433
:10F20000A5248823B9F183E50E94B222882309F45A
:10F210004BC08FE69CE00E94382A8AE00E94FF29BA
:10F220008EEF8093590581E080936C02109258050F
:10F2300081E09AE59093FD138093FC138CE490E0B9
:10F240009093FF138093FE1387E08093F01382E87E
:10F250008093F31384E890E0A0E0B0E08093F4138F
:10F260009093F513A093F613B093F71380EA93E10C
:10F270000E947D26C057DF4F0FB6F894DEBF0FBE49
:10F28000CDBFDF91CF911F910F91FF90EF90DF9055
:10F29000CF90BF90AF909F908F907F906F905F9036
:10F2A0004F903F902F90089583E40E94B2228823CC
:10F2B00049F00E948F240E943AF90E9485890E9499
:10F2C0000330D8CF2090340C3090350C4090360C61
:10F2D0005090370C80913D0C80FF05C09091630BDE
:10F2E00098609093630B869581708093620B83E3A3
:10F2F0009DE00E9472788091C30B9091C40B9E0197
:10F300002F5F3F4F7901009799F09F938F938AE287
:10F310009DE09F938F933F932F930F941B1DC701E5
:10F320000E9444780F900F900F900F900F900F90C5
:10F330008091C10B9091C20B009799F09F938F938E
:10F3400081E29DE09F938F93FF92EF920F941B1D9C
:10F35000C7010E9444780F900F900F900F900F906C
:10F360000F906E0131E8C30ED11C60919B0B709120
:10F370009C0B80919D0B90919E0B860123E041E0B8
:10F380000F9451189F938F938FE09DE09F938F93DD
:10F39000FF92EF920F941B1DC7010E94447887E0F3
:10F3A0009DE00E94727887E08093970C80933309E8
:10F3B00099EB692E9BE0792E0F900F900F900F9094
:10F3C0000F900F90B12CA12C2AEF822E2CE0922EC0
:10F3D000F30161917191819191913F01860123E047
:10F3E00041E00F9451189F938F93BF92AF929F92D9
:10F3F0008F92FF92EF920F941B1DC7010E944478D9
:10F400000FB6F894DEBF0FBECDBFAA94AB2809F0AB
:10F4100065C18091B80B811115C08091B70B1F9207
:10F420008F938EEE9CE09F938F93FF92EF920F94B9
:10F430001B1DC7010E9444780F900F900F900F90F2
:10F440000F900F908091B70B1F928F9388EE9CE0E6
:10F450009F938F93FF92EF920F941B1DC7010E9401
:10F4600044788091C50B0F900F900F900F900F90E4
:10F470000F908823A1F01F928F931F921F928BED04
:10F480009CE09F938F93FF92EF920F941B1DC701F7
:10F490000E9444780FB6F894DEBF0FBECDBF8091B6
:10F4A000C60B8823A9F01F928F931F9281E08F9340
:10F4B0008BED9CE09F938F93FF92EF920F941B1D17
:10F4C000C7010E9444780FB6F894DEBF0FBECDBFCF
:10F4D0008090C70B9090C80BA090C90BB090CA0B3E
:10F4E00020E030E0A901C501B4010F94841D811111
:10F4F00004C080913D0C82FF20C0860121E041E0E4
:10F50000C501B4010F9451189F938F9380913D0CC6
:10F5100082FB882780F91F928F938EEC9CE09F934B
:10F520008F93FF92EF920F941B1DC7010E944478A6
:10F530000FB6F894DEBF0FBECDBF8AEC9CE00E94F0
:10F54000727860918D0B70918E0B80918F0B9091E2
:10F55000900B8E010F581F4F23E041E00F9451187C
:10F56000B82EA92E6091890B70918A0B80918B0B1C
:10F5700090918C0B860123E041E00F945118AF92DB
:10F58000BF929F938F9389EB9CE09F938F93FF9201
:10F59000EF920F941B1DC7010E9444786091910B5C
:10F5A0007091920B8091930B9091940B23E041E02A
:10F5B0000F9451188EEA9CE00E947278DF92CF92ED
:10F5C00084EA9CE09F938F93FF92EF920F941B1D10
:10F5D000C7010E94447880919A0B8F938091990B78
:10F5E0008F938DE99CE09F938F93FF92EF920F94FE
:10F5F0001B1DC7010E9444786091950B7091960B7A
:10F600008091970B9091980B23E041E00F94511853
:10F610009F938F9383E99CE09F938F93FF92EF9248
:10F620000F941B1DC7010E9444788CE0EFE9FBE0BA
:10F63000ACE7BBE001900D928A95E1F78CE0EBEA34
:10F64000FBE0A0E7BBE001900D928A95E1F780E036
:10F650000E946DC581E00E946DC582E00E946DC56B
:10F6600080913C0C8093640B81E08093DF080E94C2
:10F6700097248BEC9BE09F938F9380ED97E29F9371
:10F680008F93FF92EF920F941B1D0FB6F894DEBF7D
:10F690000FBECDBFC7010E94447880913B0C8F9371
:10F6A00080913A0C8F938091390C8F938091380C14
:10F6B0008F935F924F923F922F9285E89CE09F93A9
:10F6C0008F93FF92EF920F941B1DC7010E94447805
:10F6D0000FB6F894DEBF0FBECDBFCCCDAA24A39445
:10F6E000B12C76CE4F925F926F927F928F929F92C3
:10F6F000AF92BF92CF92DF92EF92FF920F931F9340
:10F70000CF93DF9300D000D01F921F92CDB7DEB70A
:10F7100060E083E50E942A23863028F084EF9BE096
:10F720000E94382A3BC0833009F460C1B0F48130B4
:10F7300021F1823009F44CC081EE9BE00E94382A0E
:10F740000E94F8248823A1F08091F90C0E94FA35D8
:10F750000E947B350E9481D321C0843009F490C17E
:10F76000853051F780E00E94DD240E94BD24F2CF55
:10F7700083ED9BE00E94382AEDCF0E94BD241092B9
:10F780000602109205028EE40E94B22281111DC071
:10F7900081EC9BE0909364128093631228960FB6DD
:10F7A000F894DEBF0FBECDBFDF91CF911F910F91B7
:10F7B000FF90EF90DF90CF90BF90AF909F908F9091
:10F7C0007F906F905F904F90089587EC9BE0E2CF21
:10F7D000809105029091060297FF03C088E99BE0A3
:10F7E0009FCF009709F0A8C01D821E821F82188635
:10F7F0008DEC9CECACE4BEE389839A83AB83BC8341
:10F80000BE016B5F7F4FCE0101960E9454C780916D
:10F81000050290910602893191050CF0B3C021E0F8
:10F8200020934C029C012F5F3F4F309306022093A0
:10F83000050265E00F942B2480FF03C024E0291B00
:10F84000922F24E09202F0011124E159FB4E8080B6
:10F850009180A280B38094E08902F0011124E55ADE
:10F86000FB4E40805180628073808DEC9CECACE458
:10F87000BEE38D839E83AF83B88719821A821B8271
:10F880001C82CE0101966C01E12CF12C00EA10E4FF
:10F89000A3019201C501B4010E947AC619821A829D
:10F8A0001B821C82B601CE0105960E9454C780922D
:10F8B000FA0C9092FB0CA092FC0CB092FD0C4092C2
:10F8C000FE0C5092FF0C6092000D7092010D0091A1
:10F8D00005021091060289E1F82EE12C093111058B
:10F8E00014F4F02EE12E6F2D7E2D81E39BE00E941B
:10F8F0003A3669E170E08CE29BE00E943A368AE099
:10F900000E94FF29101611060CF024CF1F9289E1E6
:10F910008F93EF92FF9285E19BE09F938F9383E219
:10F920009BE09F938F931F920E940AE80FB6F89472
:10F93000DEBF0FBECDBF0ECF815065E00F942B24EC
:10F9400080FF03C024E0291B922F25E09202F001E2
:10F950001124E80FF11D87FDFA95EE0FFF1FEE0F42
:10F96000FF1FE250F54F8091020D9091030DA09181
:10F97000040DB091050D80839183A283B38310920F
:10F980004C0245CF80E090E0A0EAB0E48093020D05
:10F990009093030DA093040DB093050D87E492E0BE
:10F9A0000E945BC60E9403C28FEF9FEF90930602F6
:10F9B0008093050284E89BE00E94382A82E79BE05E
:10F9C0000F941F1063E972E084E690E00E94672FB5
:10F9D0006AEB72E084E690E00E94672F8CE69BE081
:10F9E0000E94727881E00E94DD2471CF89E40E9438
:10F9F0000023882371F00E948422182F853068F03C
:10FA000064E070E089E59BE00E943A3686E59BE081
:10FA100087CE8AE40E94DA33C1CE8AE40E940023B2
:10FA20008823B9F30E948422082F853048F064E0CF
:10FA300070E083E49BE00E943A3680E49BE070CE65
:10FA40008AE50E9400238823C9F00E94882225E0CD
:10FA50001202F0011124E00FF11D07FDFA95EE0FDF
:10FA6000FF1FEE0FFF1FE250F54F6083718382830B
:10FA70009383602F812F0E94D4EE6CCE8AE5CACF8B
:10FA80008AE50E9400238823C9F30E94882260939C
:10FA9000E0087093E1088093E2089093E3085ACE5F
:10FAA000CF93DF93C091080EC093660581E6C89F8F
:10FAB000E0011124C65FD14F8091630B80FF05C028
:10FAC0000E94974ECE010E94062ACE010E94131E6C
:10FAD00080E0DF91CF910C94A263CF938091961137
:10FAE000C1E08823C9F080919711909198114091BD
:10FAF0008E1150918F116091901170919111DC01D4
:10FB0000ED91FC910288F389E02D2EE83FE01995F4
:10FB1000C82F811104C0C0E08C2FCF91089540916F
:10FB2000921150919311609194117091951141151A
:10FB3000510561057105B9F0809197119091981167
:10FB4000DC01ED91FC910288F389E02D2EE83FE085
:10FB50001995882301F3109292111092931110922B
:10FB600094111092951110929611D6CF0F931F9366
:10FB7000CF93DF93CDB7DEB760970FB6F894DEBFB3
:10FB80000FBECDBF8C01DC01ED91FC910280F381B1
:10FB9000E02DBE016F5F7F4F1995882309F464C083
:10FBA0008981807CC9F56F81637070E0762F66274C
:10FBB000770F770F8885B4E08B9FC0011124682BE5
:10FBC000792B89858295869586958370682B6F5FE2
:10FBD0007F4F90E080E02A852370220F3B8537FB22
:10FBE000332730F9232B3E813F70230F3327331FF8
:10FBF0002750310904C0660F771F881F991F2A9567
:10FC0000D2F760960FB6F894DEBF0FBECDBFDF917E
:10FC1000CF911F910F910895803419F568856695ED
:10FC2000669570E090E080E0CB01772766272A8513
:10FC3000622B098510E0102F0027012E000C220BEB
:10FC4000330B602B712B822B932B6F5F7F4F8F4F6A
:10FC50009F4F4AE0660F771F881F991F4A95D1F77B
:10FC6000D0CF8BE0F801848360E070E0CB01C9CF96
:10FC70000895FC0182810895BC0120912D0A3091E4
:10FC80002E0A40912D0A50912E0A2417350731F47F
:10FC900081E02617370709F080E008959A01F1CF37
:10FCA000EF92FF920F931F93E092F508F092F608FF
:10FCB0000093F7081093F8086093F9087093FA0816
:10FCC0008093FB089FEFFF27621B730B840B30F4BC
:10FCD000809570956195790B890B992790930A040B
:10FCE000A6E06A9F0092FE03512DEE277A9F500DE9
:10FCF000E11D8A9FE00D5093FF03E0930004AFE005
:10FD00006A9F00920204512DEE277A9F500DE11D4B
:10FD10008A9FE00D50930304E0930404AAE06A9FD5
:10FD200000920604512DEE277A9F500DE11D8A9F07
:10FD3000E00D50930704E09308041F910F91FF908A
:10FD4000EF9008959F92AF92BF92CF92DF92EF9281
:10FD5000FF920F931F93CF93DF9300D01F921F92B8
:10FD6000CDB7DEB7E6EAF7E10027BB27462F572FCE
:10FD7000A82FAA2341F4A52F542FB85FAA2319F462
:10FD8000A52F5527B85FA03138F45295A295452F7D
:10FD90004F70507FA42BBC5FA03428F4550FAA1FCE
:10FDA000550FAA1FBE5FA03818F4550FAA1FB395B0
:10FDB000550FAA1FEA0FF01F449151E0AA27B8502F
:10FDC00081F1C8F0B0FF02C0440F551FB1FF04C05D
:10FDD000440F551F440F551FB2FF06C05295429560
:10FDE000142F1F70407F512BB3FF1BC0A52F542F22
:10FDF00044270C94117FB195B0FF02C055954795EB
:10FE0000B1FF04C05595479555954795B2FF05C07C
:10FE10005295407F4295452B5F70B3FF02C0452F3E
:10FE20005527DD24CC24BB24B2E0649FD018C10840
:10FE3000B00AB00B749FC018B108B00B849FB01803
:10FE4000B109659FC018B108B00B759FB018B10912
:10FE5000859FB0196A9FB018B1097A9FB0194D9D5E
:10FE6000A12C99243327992722275D9DA00C911C52
:10FE7000301F901F201FAD9D900C311D901F201F23
:10FE80004C9DA00C911C301F901F201F5C9D900C5E
:10FE9000311D901F201FAC9D300D911D201F4B9DCB
:10FEA000900C311D901F201F5B9D300D911D201F58
:10FEB000AB9D900D211D4B9F300D911D201F5B9F11
:10FEC000900D211DAB9F200DB1E0BB24CC24DD247F
:10FED000639FD018C108B00AB00B739FC018B10857
:10FEE000B00B839FB018B109699FC018B108B00B5F
:10FEF000799FB018B109899FB019629FB018B109F4
:10FF0000729FB019D61AC70AB80A20F0B1E03B0FA9
:10FF1000901F201F1124792F632F90E0822F0F90C4
:10FF20000F900F900F900F90DF91CF911F910F9135
:10FF3000FF90EF90DF90CF90BF90AF909F9008958B
:10FF400080919A1290919B12891B877019F490E00E
:10FF500080E0089590919712992351F0833030F406
:10FF60008FEF890F19F080939712F1CF10929712AB
:10FF700080919B1228E6829FC001112489579A4FD5
:10FF8000FC01208120FDE3CF20919B122F5F277081
:10FF90002093981230919B1220919912321304C031
:10FFA000209198122093991208952F923F924F9288
:10FFB0005F926F927F928F929F92AF92BF92CF92F9
:10FFC000DF92EF92FF920F931F93CF93DF93CDB702
:10FFD000DEB764970FB6F894DEBF0FBECDBF7A8B45
:10FFE000698BDC018D909D90AD90BC901397149619
:10FFF0002D913D914D915C9117972D833E834F83B9
:020000021000EC
:10000000588720E030E040EA51E4C501B4010F9484
:10001000612421EC3FE04CE75CE30F94EA1D0F9470
:10002000CE2564300CF427C163E0E62E660FFF088E
:10003000F701EE0FFF1FEE0FFF1FE159FB4E40804F
:100040005180628073801701BFEF2B1A3B0A20E0BA
:1000500030E040EA51E46D817E818F8198850F9474
:10006000612421EC3FE04CE75CE30F94EA1D0F9420
:10007000CE2564300CF403C163E0062F660F110B2C
:10008000F801EE0FFF1FEE0FFF1FE159FB4E20811D
:1000900031814281538129833A834B835C83A80158
:1000A0004F5F5F4F5C8B4B8BA5E0AE9DC001AF9D5A
:1000B000900D11249A878987FC01E00FF11FEE0F44
:1000C000FF1FEE0FFF1FE250F54FC080D180E2808E
:1000D000F380F101EE0FFF1FEE0FFF1FE159FB4E02
:1000E000A301920160817181828193810F946124C7
:1000F0006B877C878D879E87A3019201C501B40120
:100100000F9461242B013C0125E0229DF001239DE9
:10011000F00D1124F88BEF87E00FF11FEE0FFF1F9A
:10012000EE0FFF1FE250F54FA7019601608171812C
:10013000828193810F9461242B853C854D855E855A
:100140000F945C25A30192010F94EA1DA70196016B
:100150000F9462246B017C01E985FA854B895C89E7
:10016000E40FF51FEE0FFF1FEE0FFF1FE250F54FDC
:1001700080809180A280B380EF85F889E40FF51F1D
:10018000EE0FFF1FEE0FFF1FE250F54FA501940188
:1001900060817181828193810F9461242B853C85DC
:1001A0004D855E850F945C25A30192010F94EA1D95
:1001B000A50194010F946224A70196010F94612474
:1001C0004B015C01EB89FC89EE0FFF1FEE0FFF1F57
:1001D000E159FB4E29813A814B815C8160817181BB
:1001E000828193810F9461249B01AC01C501B4010C
:1001F0000F945C254B015C0129813A814B815C8124
:100200006D817E818F8198850F9461249B01AC0163
:10021000C501B4010F94EA1DA70196010F94622451
:10022000A989BA892D913D914D915C910F94EA1D58
:100230002091E0083091E1084091E2085091E308F4
:100240000F94622464960FB6F894DEBF0FBECDBF44
:10025000DF91CF911F910F91FF90EF90DF90CF90A2
:10026000BF90AF909F908F907F906F905F904F90D6
:100270003F902F90089567FFD8CE60E0D6CE67FFFD
:10028000FCCE60E0FACE90916F0081E091FD02C05B
:1002900080E0089590916F009D7F90936F00089586
:1002A0008F929F92AF92BF92CF92DF92EF92FF9286
:1002B000CF93DF93EC018090470C9090480CA09076
:1002C000490CB0904A0C20E030E0A901C501B4010E
:1002D0000F94841D882309F454C0C880D980EA8013
:1002E000FB80A7019601C501B4010F94841D181667
:1002F0000CF04CC020913F0C3091400C4091410CCF
:100300005091420CC701B6010F94841D882331F12E
:10031000C0923F0CD092400CE092410CF092420C03
:100320002091430C3091440C4091450C5091460C67
:10033000688179818A819B810F94EA1D9B01AC01C0
:1003400060E070E080E89FE30F94612460930E0208
:1003500070930F02809310029093110260910E022D
:1003600070910F028091100290911102DF91CF9154
:10037000FF90EF90DF90CF90BF90AF909F908F90C5
:10038000089560E070E080E89FE3F0CF60E070E007
:10039000CB01ECCF24E0829FC0011124FC01E55A7F
:1003A000FA4E4591559165917491DC01A55BBD4F65
:1003B00012964D935D936D937C931597815B9A4E46
:1003C000FC0145915591659174911E964D935D93F5
:1003D0006D937C9351970895CF93C82FCB010E94C2
:1003E000382A80E295E10E94382A81E195E1CC2308
:1003F00011F086E195E10E94382A8AE0CF910C94B1
:10040000FF290F931F93CF93811113C0C42F8B012A
:100410000E94974E86E899E10E94382AC8010E94FE
:10042000382ACC2331F08AE0CF911F910F910C94A0
:10043000FF29CF911F910F910895CF93DF93EC0186
:100440008D810E94B55360E08B81DF91CF910C9438
:100450002FF2DF92EF92FF920F931F93CF93DF93D0
:100460008C01C62FD22FF32EE42ED52E0E941D8292
:100470000E94CEF88C2F80640E94A9538D2D0E947B
:10048000A9538E2D0E94A9538F2D0E94A9538D2F01
:100490000E94A95387E8C11101C085E90E94A953B0
:1004A000CC3011F40E94AE53C0E00E94AE53F8016C
:1004B000868387FF04C0CF3F11F0CF5FF6CFDF9177
:1004C000CF911F910F91FF90EF90DF90089561E021
:1004D000FC0183810E942FF28FEF0C94A9530F939C
:1004E0001F93CF938C010E941D820E94CEF8C82FCB
:1004F000882371F08DEF0E94A9530E94CEF8C82F77
:10050000C8010E9467828C2FCF911F910F9108958F
:1005100082E1F8018483F4CF8F929F92AF92BF92D1
:10052000CF92DF92EF92FF920F931F93CF93DF93BF
:10053000EC016A017B01590120E030E0A90167E389
:100540000E942982A501980167E1CE010E942982BB
:10055000811127C08F81833039F089E0CC0CDD1CFC
:10056000EE1CFF1C8A95D1F7A701960169E1CE0127
:100570000E94298211E0882319F010E087E08C8323
:10058000CE010E946782812FDF91CF911F910F9141
:10059000FF90EF90DF90CF90BF90AF909F908F90A3
:1005A000089589E08C8310E0EBCFCF93DF93EC01CB
:1005B0006EBDFA01CA019E5F0DB407FEFDCF20811A
:1005C0002EBD0DB407FEFDCF21812EBD3296E8175A
:1005D000F90791F70DB407FEFDCF8FEF0E94A953E5
:1005E0008FEF0E94A9530E94AE538E838F71853086
:1005F00049F083E18C83CE010E94678280E0DF9125
:10060000CF91089581E0FBCF0F931F93CF93DF939A
:10061000EC018B010E941D820E94CEF881110CC05A
:1006200085E18C8310E0CE010E946782812FDF91EB
:10063000CF911F910F910895A8016CEFCE010E94F8
:10064000D582182F882361F3EECF0F931F93CF939A
:10065000DF93EC0189018F81833039F089E0440F09
:10066000551F661F771F8A95D1F79A01AB0168E184
:10067000CE010E94298281112AC0A8016EEFCE010D
:100680000E94D582182F8823B1F00E94CEF8182F2F
:100690008823D1F020E030E0A9016DE0CE010E9476
:1006A0002982882321F086E18C8310E004C00E9417
:1006B000AE538111F8CFCE010E946782812FDF9166
:1006C000CF911F910F91089587E18C83F4CF86E03D
:1006D000EBCF1F93CF93DF93EC010E941D8220E0AC
:1006E00030E0A9016CE0CE010E94298211E088234C
:1006F00019F010E083E08C83CE010E946782812F85
:10070000DF91CF911F9108951F93CF93DF93EC0159
:100710008F81833039F089E0440F551F661F771FA2
:100720008A95D1F79A01AB0162E1CE010E9429823C
:1007300011E0882319F010E085E08C83CE010E943F
:100740006782812FDF91CF911F9108958F929F92A1
:10075000AF92BF92EF92FF920F931F93CF93DF93CD
:100760008C01EB017A010E94C4F34B015C012CE285
:10077000820E21E0921EA11CB11C0E94AE53F80112
:1007800086838F3F69F40E94C4F3681979098A0946
:100790009B0997FDF2CF81E1F8018483C0E021C07D
:1007A0008E3F71F5F1E0EF1AF1088FEF8EBDFE017B
:1007B0002FEF0DB407FEFDCF8EB581932EBDCF0177
:1007C0008C1B9D0B8E159F05A0F30DB407FEFDCF6E
:1007D0008EB5CE0DDF1D88830E94AE530E94AE53AE
:1007E000C1E0C8010E9467828C2FDF91CF911F91D9
:1007F0000F91FF90EF90BF90AF909F908F900895D2
:100800008FE0CACF0F931F93CF93DF93EC018B013F
:100810000E941D8240E052E0B801CE01DF91CF91ED
:100820001F910F910C94A6830F931F93CF93DF9387
:10083000EC0189018F81833039F089E0440F551F25
:10084000661F771F8A95D1F79A01AB0161E1CE014E
:100850000E94298281110AC040E052E0B801CE0115
:10086000DF91CF911F910F910C94A68384E08C832C
:10087000CE010E94678280E0DF91CF911F910F919E
:1008800008958F929F92AF92BF92CF92DF92EF9294
:10089000FF920F931F93CF93DF93EC01162F1F82CC
:1008A0001C824B830E94C4F36B017C0120EDC20EBD
:1008B00027E0D21EE11CF11CA89561E08B810E940B
:1008C0002FF28B810E94ACEA209A289A219A2398D1
:1008D000229A81E00E94B55385E08D830E94B55332
:1008E0000AE08FEF0E94A9530150D9F7A89520E0A4
:1008F00030E0A90160E0CE010E9429828E83813020
:1009000081F00E94C4F36C197D098E099F0997FD3F
:10091000EECF81E08C83CE010E9467821A8280E054
:100920006AC0A8952AEA31E040E050E068E0CE01D4
:100930000E942982853041F581E08F83A8958F81BF
:10094000812C912C5401823029F4812C912CA12CE2
:1009500080E4B82E20E030E0A90167E3CE010E94D8
:100960002982A501940169E2CE010E9429828E8329
:100970008823F1F00E94C4F36C197D098E099F0948
:1009800097FDE8CF8AE0C6CF04E00E94AE538E8385
:100990000150D9F78A3A11F482E0CFCF0E94C4F314
:1009A0006C197D098E099F0997FDBCCF82E0B2CFFB
:1009B0008F818230C1F420E030E0A9016AE3CE01EA
:1009C0000E942982882311F088E0A4CF0E94AE53B0
:1009D000807C803C11F483E08F830E94AE530E94A0
:1009E000AE530E94AE53CE010E94678281E08A839B
:1009F000173070F41D83DF91CF911F910F91FF90FD
:100A0000EF90DF90CF90BF90AF909F908F90089520
:100A100088E18C8384CF0F931F93CF93DF93EC01F6
:100A20008B0120E030E0A90169E00E942982811158
:100A30000AC040E150E0B801CE01DF91CF911F9193
:100A40000F910C94A68380E18C83CE010E94678273
:100A500080E0DF91CF911F910F910895CF93C82F20
:100A60000E94438194E0C99F90011124F901E05D47
:100A7000F54F245C354FD9014D915D916D917C917D
:100A8000408351836283738391E090932F0A88237C
:100A900019F0CF910C942025CF910895CF92DF9239
:100AA000EF92FF928091AD09659B62C08160809357
:100AB000AD09909103018091AD0991FF5BC0826007
:100AC0008093AD098091AD094B9B56C084608093A3
:100AD000AD09C090200AC0FE10C08091A10A80FF1D
:100AE0000CC08091AD0980FF08C08091E30A81604D
:100AF0008093E30A80E00E942E85D12CF12CE12C1A
:100B0000D701C601B695A7959795879580FF11C027
:100B10008091A10A869580FF0CC08091AD0981FF6C
:100B200008C08091E30A82608093E30A81E00E941A
:100B30002E8582E0F694E794D794C7948A95D1F7EE
:100B4000C0FE1CC08091A10A8695869580FF16C0C4
:100B50008091AD0982FF12C08091E30A8460809386
:100B6000E30A82E0FF90EF90DF90CF900C942E8507
:100B70008E7F9DCF8D7FA4CF8B7FA9CFFF90EF90ED
:100B8000DF90CF900895CF93DF9380919A12909148
:100B90009B12891B8095877019F40E94B156F5CF7E
:100BA00080919A128F5F8770A0919A1298E6A99F00
:100BB000D0011124FD01E957FA4FEF0119929A95DE
:100BC000E9F798E09083A456BA4F90E1E0ECF2E1A7
:100BD00001900D929A95E1F720919A1290919B12B3
:100BE000291303C094E69093971280939A12DF9191
:100BF000CF910C9420250F930091F40821E0022757
:100C00002AED39E04CE050E0BC0184ED99E00E940F
:100C1000EE250F9108950F930091F40821E002272B
:100C20002AED39E041E050E0BC0184ED99E00E94FA
:100C3000EE250F9108950F930091F40821E002270B
:100C40002AED39E041E050E0BC0184ED99E00E94DA
:100C5000EE250F9108950F930091F40821E00227EB
:100C60002AED39E042E050E0BC0184ED99E00E94B9
:100C7000EE250F9108950F930091F40821E00227CB
:100C80002AED39E048E050E0BC0184ED99E00E9493
:100C9000EE250F9108950F930091F40821E00227AB
:100CA0002AED39E04CE050E0BC0184ED99E00E946F
:100CB000EE250F9108950F930091F40821E002278B
:100CC0002AED39E044E050E0BC0184ED99E00E9457
:100CD000EE250F9108950F9301E02AED39E041E0F0
:100CE00050E0BC0184ED99E00E94EE250F9108953B
:100CF0000F93AB010091F40821E002272AED39E0BF
:100D0000BC0184ED99E00E94EE250F9108952AED33
:100D100039E042E050E0BC0184ED99E00C94785158
:100D20002AED39E04CE050E0BC0184ED99E00C94F0
:100D300078512AED39E041E050E0BC0184ED99E0C2
:100D40000C9478512AED39E041E050E0BC0184ED8B
:100D500099E00C9478512AED39E04CE050E0BC0168
:100D600084ED99E00C9478512AED39E044E050E0AC
:100D7000BC0184ED99E00C9478512F923F924F92F0
:100D80005F926F927F928F929F92AF92BF92CF921B
:100D9000DF92EF92FF920F931F93CF93DF93CDB724
:100DA000DEB76C970FB6F894DEBF0FBECDBF8C01D7
:100DB0005B015A834983FC01EE5AFF4F2081318148
:100DC0004281538129873A874B875C87CA01B901E1
:100DD0000F94891D6B017C01D5012D913D914D91A1
:100DE0005C910F94EA1D0F9440252B013C01E98191
:100DF000FA812081318142815381C701B6010F946C
:100E0000EA1D0F9440254B015C01C301B2010F9410
:100E1000D525698B7A8B8B8B9C8B68377105810507
:100E2000910540F428E730E040E050E0298B3A8B10
:100E30004B8B5C8BC501B4010F94D5256D877E87E4
:100E40008F87988B683771058105910540F448E7D5
:100E500050E060E070E04D875E876F87788BF80127
:100E6000E25AFF4F4080518062807380C301B2011B
:100E70000F948B1D69837A838B839C8369897A891C
:100E80008B899C890F94891D6D8B7E8B8F8B988F9E
:100E900020E030E0A90169817A818B819C810F94E7
:100EA000841D882309F4E1C1A7019601C701B60199
:100EB0000F94EA1D4B015C012D893E894F89588DA5
:100EC000CA01B9010F94EA1D9B01AC01C501B4012F
:100ED0000F9461244B015C0129813A814B815C8133
:100EE000CA01B9010F9462249B01AC01C501B40190
:100EF0000F945C250F9440250F94D5256D837E8338
:100F00008F83988766277727CB016419750986092F
:100F100097090F948B1D4B015C016D857E858F8534
:100F200098890F94891D2B013C0120E030E0A90134
:100F3000C501B4010F94841D882309F49AC1A3014B
:100F40009201C301B2010F94EA1D698F7A8F8B8FD2
:100F50009C8FA7019601C701B6010F94EA1D9B0162
:100F6000AC01698D7A8D8B8D9C8D0F9461246B0102
:100F70007C01A5019401C501B4010F9462249B0179
:100F8000AC01C701B6010F945C250F940426D8016B
:100F900095968D909D90AD90BC9098977501640149
:100FA0002D813E814F815885C21AD30AE40AF50A81
:100FB0000F94D525C61AD70AE80AF90AF7FE8EC09B
:100FC0002D893E894F89588DCA01B9010F94EA1DB8
:100FD0006B017C0129813A814B815C81CA01B90195
:100FE0000F94622469877A878B879C8720E030E0A2
:100FF000A90169817A818B819C810F94841D88234A
:1010000009F43BC1C501B4010F94891D29853A85B6
:101010004B855C850F94EA1DA70196010F9461240E
:101020006D837E838F839887A3019201C301B201F0
:101030000F94EA1D9B01AC016D817E818F819885A3
:101040000F9462242B013C0120E030E040E850E4A2
:1010500069817A818B819C810F94EA1D9B01AC018F
:10106000C301B2010F945C250F9440252B013C0174
:1010700020E030E0A9010F94C22618161CF0412C84
:10108000512C3201C301B2010F94D5256D837E83AB
:101090008F83988786169706A806B90620F48D8256
:1010A0009E82AF82B8866D817E818F8198850F94F4
:1010B000891D29853A854B855C850F94EA1DA7011A
:1010C00096010F9462240F9410270F94D5256987F9
:1010D0007A878B879C87C12CD12C760169857A858C
:1010E0008B859C8529893A894B895C89621B730BA6
:1010F000840B950B0F94891D29813A814B815C816A
:101100000F945C2520E034E244EF59E40F94EA1D8B
:101110000F94D5254B015C0169857A858B859C856B
:101120002D853E854F855889621B730B840B950B6B
:101130000F94891D29813A814B815C810F945C2534
:1011400020E034E244EF59E40F94EA1D0F94D525D2
:101150002B013C013FE683169104A104B10408F081
:1011600090C0F401EE0FFF1FEE0FFF1FE651FA4E85
:1011700085919591A591B4918983292E3A2EBD8BA5
:101180004FE6441651046104710408F083C0F20173
:10119000EE0FFF1FEE0FFF1FE651FA4E45915591DE
:1011A000659174919A01CB014D815E816F81788543
:1011B000D8019A964D935D936D937C939D974C0DBA
:1011C0005D1D6E1D7F1DF80146A757A760AB71AB73
:1011D000EA5AFF4F49895A896B897C894083518338
:1011E00062837383D6968D929D92AD92BC92D9976D
:1011F000F80142AE53AE64AE75AEFE9649814083AF
:10120000218232825D8953833496208331838283A5
:10121000938369857A858B859C85D2966D937D9322
:101220008D939C93D59778962D853E854F855889CB
:1012300020833183428353836C960FB6F894DEBFCC
:101240000FBECDBFDF91CF911F910F91FF90EF9017
:10125000DF90CF90BF90AF909F908F907F906F90D6
:101260005F904F903F902F90089560E070E0CB0129
:1012700041CE60E070E0CB0188CE60E070E0CB0151
:10128000F3CEC501B4010E94A27E6983272E382EB9
:101290009D8B76CFC301B2010E94A27E9B0184CFB9
:1012A0008BE1EEEAF4E1A9ECB4E101900D928A95AC
:1012B000E1F780918E14806280938E14089580915E
:1012C00083148823C1F0815080938314EEEAF4E103
:1012D000882351F08150990B2BE1289FF001299F21
:1012E000F00D1124EC51FB4E8BE1A9ECB4E101901F
:1012F0000D928A95E1F780918314811105C0909138
:101300008E14906290938E14089581E080938414DB
:101310000C947CF9CF92DF92EF92FF9280918E1421
:1013200082FF29C0C0908A14D0908B14E0908C1456
:10133000F0908D1486EA98E20E94382A4AE0C701AC
:10134000B6010E94D0F98FE20E94FF2960918614B5
:101350007091871480918814909189144AE00E94BA
:10136000D0F98DE00E94FF298AE0FF90EF90DF9096
:10137000CF900C94FF2988EB98E2FF90EF90DF90DC
:10138000CF900C94382ABC018AED97E20E94C65394
:1013900087ED97E20C94382A80918E1483FF03C066
:1013A000846080938E140895CF92DF92EF92FF9223
:1013B0000F931F93CF93DF93CDB7DEB7EDB6FEB695
:1013C000DC010D900020E9F79D01281B390B285FF7
:1013D0003F4FEDB7FEB7E21BF30B0FB6F894FEBF1D
:1013E0000FBEEDBF0DB71EB70F5F1F4F9F938F93BB
:1013F00080ED97E29F938F931F930F930F941B1D84
:101400006801F4E0CF0ED11C0F900F900F900F9059
:101410000F900F90D6018D916D01882349F0082E11
:10142000000C990B0F947427F60131978083F2CF4B
:101430006BEC77E2C8010F94B41C4FE350E0B801A5
:1014400083EA9AE00F94D0270FB6F894FEBE0FBE41
:10145000EDBEDF91CF911F910F91FF90EF90DF9044
:10146000CF900895FC01938591FD13C0987121E000
:10147000903109F020E080918E1420FB84F9809354
:101480008E14903141F08085873419F481858E3730
:1014900011F480E0089581E00895FC0120E03EE22F
:1014A000DB014D91BD01403249F0283011F4308309
:1014B0003196DB0111974C91408331962F5F2B3091
:1014C00079F710820895EF92FF920F931F93CF93B5
:1014D000DF93CDB7DEB7A0970FB6F894DEBF0FBE8F
:1014E000CDBF7C018B01BE016F5F7F4FC7010E94A2
:1014F00014E51816A4F4CE0101960E94328A8823BE
:1015000091F3BE016F5F7F4F89EF91E10E944D8A99
:1015100069EF71E1C8010F949227892B21F7A096FA
:101520000FB6F894DEBF0FBECDBFDF91CF911F91F4
:101530000F91FF90EF900895CF92DF92EF92FF927C
:10154000CF936B017C01C42F80918E1190918F11EC
:10155000A0919011B09191118C159D05AE05BF051C
:1015600029F10E946D7D811108C0C0E08C2FCF91C0
:10157000FF90EF90DF90CF90089580919711909118
:101580009811DC01ED91FC910088F189E02D2EE8A5
:101590003FE0B701A6011995882339F3C0928E1157
:1015A000D0928F11E0929011F0929111CC2321F002
:1015B00081E080939611DACFC1E0D8CF4F925F924D
:1015C0006F927F928F929F92AF92BF92CF92DF9253
:1015D000EF92FF920F931F93CF93DF93EC01423072
:1015E00051056105710590F480E0DF91CF911F9165
:1015F0000F91FF90EF90DF90CF90BF90AF909F90B2
:101600008F907F906F905F904F90089589859A8515
:10161000AB85BC850196A11DB11D84179507A60752
:10162000B70710F38F898031C9F5852E962EA72E26
:10163000BB248B899C89AD89BE89880E991EAA1E00
:10164000BB1E280139016A017B0141E0C501B401DB
:101650000E949C8A882341F29F89903181F5DD2484
:10166000EE24FF24F601EE0FFF1FE257F04F118327
:1016700000839A89923008F4B8CF4D815E816F81E2
:101680007885840E951EA61EB71E809292119092A8
:101690009311A0929411B0929511A7CF803209F0C6
:1016A000A3CF8B899C89AD89BE894A015B01E7E0A4
:1016B000B694A79497948794EA95D1F7BECFE8940F
:1016C000C7F8DD24EE24FF24F601EE0FFF1FEE0F16
:1016D000FF1FE257F04F4082518262827382C9CF6E
:1016E000CF92DF92EF92FF920F931F93CF93DF93EE
:1016F000FC0181859285A385B4850196A11DB11D4C
:1017000084179507A607B70750F480E0DF91CF91C3
:101710001F910F91FF90EF90DF90CF9008958789F0
:101720008031A9F5BB27A72F962F852FC388D48892
:10173000E588F6888C0D9D1DAE1DBF1DE9016A016F
:101740007B018F0140918E1150918F11609190110A
:101750007091911184179507A607B70749F5F8010D
:101760008789803169F5B701A60155276627772754
:10177000440F551F4257504FFA0180819181B0E0CC
:10178000A0E088839983AA83BB8381E0BFCF8032A6
:1017900009F0BBCFC388D488E588F688DB01CA018D
:1017A000C7E0B695A79597958795CA95D1F7C2CF0B
:1017B00040E0BC01CD010E949C8A8111D0CFA5CF11
:1017C000B701A6014F77552766277727440F551F86
:1017D000440F551F4257504FFA0180819181A281D9
:1017E000B381BF70CECF4F925F926F927F92AF92D4
:1017F000BF92CF92DF92EF92FF920F931F93CF93FE
:10180000DF9300D01F92CDB7DEB78C0149835A8396
:101810006B837C835901C12CD12C7601412C82E051
:10182000582E612C712C49815A816B817C819E01DB
:101830002F5F3F4FC8010E94708B882319F1F80178
:101840008585A301920104C0220F331F441F551F39
:101850008A95D2F7DA01C901C80ED91EEA1EFB1E0D
:1018600049815A816B817C8187898031F1F481E0E3
:10187000483F5F4F61057105B0F2F501C082D1822A
:10188000E282F3820F900F900F900F90DF91CF9133
:101890001F910F91FF90EF90DF90CF90BF90AF908E
:1018A0007F906F905F904F90089581E0483F5F4F29
:1018B0006F4F7F4008F4B7CFE0CF0F931F93CF93C4
:1018C000DF93FC012381222331F080E0DF91CF916F
:1018D0001F910F9108958B01EC01FB0187898031E5
:1018E00039F582E08B831D8A1E8A1F8A188E808DAF
:1018F000918DB0E0A0E025E0880F991FAA1FBB1FC3
:101900002A95D1F7898B9A8BAB8BBC8B1A8F098F59
:1019100081E08983188619861A861B861C821D829F
:101920001E821F82188A1C861D861E861F86CECFA9
:10193000803259F683E08B83428D538D648D758D93
:101940004D8B5E8B6F8B788F9E012F5E3F4FC80152
:101950000E94F38B8111DACFB8CF3F924F925F9202
:101960006F927F928F929F92AF92BF92CF92DF92AF
:10197000EF92FF920F931F93CF93DF93CDB7DEB714
:101980002C970FB6F894DEBF0FBECDBF5C01DC0113
:1019900059968D909C90F40181859285A385B4859C
:1019A0009C01AD012F5F3F4F4F4F5F4F29873A8713
:1019B0004B875C87D50114964D905D906D907C901F
:1019C0001797411451046104710409F459C0BFEF21
:1019D0004B1A5B0A6B0A7B0A312C730162011D8270
:1019E0001E821F821886F40181859285A385B485A5
:1019F0002D813E814F815885281739074A075B079B
:101A000008F056C089859A85AB85BC858C159D05E7
:101A1000AE05BF0550F482E0C82ED12CE12CF12C8C
:101A200092E0492E512C612C712C9E012F5F3F4F6B
:101A3000B701A601C4010E94708B8823C9F1898176
:101A40009A81AB81BC81892B8A2B8B2B01F12601DA
:101A500037019FEF491A590A690A790A2D813E8197
:101A60004F8158852F5F3F4F4F4F5F4F2D833E83F0
:101A70004F8358873FEFC31AD30AE30AF30AB3CF61
:101A8000408051806280738033243394A6CFC41485
:101A9000D504E604F70411F70FEF1FEF2FEF3FE037
:101AA000B701A601C4010E94DE8A782E81111AC0F6
:101AB000712C872D2C960FB6F894DEBF0FBECDBFCC
:101AC000DF91CF911F910F91FF90EF90DF90CF901A
:101AD000BF90AF909F908F907F906F905F904F904E
:101AE0003F900895F50144815581668177814115C4
:101AF00051056105710539F097018601C4010E9405
:101B0000DE8A8823A9F2D5011496CD92DD92ED925A
:101B1000FC921797332051F0D701C6010196A11D01
:101B2000B11DF40180839183A283B383F50185897C
:101B30009689A789B08D892B8A2B8B2B09F0B9CF79
:101B4000C58AD68AE78AF08E818180688183B1CF89
:101B5000CF93DF93EC01462F41706C857D858E8598
:101B60009F850E949C8A882351F0888920E2829F69
:101B7000C00111248257904FDF91CF91089590E0DA
:101B800080E0FACFCF93DF93EC018991882319F09D
:101B90000E94FF29FACFDF91CF910895CF93DF9371
:101BA000EC018B81882349F1898187FF22C061E0A4
:101BB000CE010E94A88DFC01892BF9F08081853E21
:101BC000E1F08B81823040F489899A89AB89BC89A4
:101BD000848F958FA68FB78F8D899E89938F828FE3
:101BE0008D899E89AF89B88DB58BA48B89818F77BC
:101BF0008983DF91CF910C946D7D81E0888380E0B3
:101C0000DF91CF9108958F929F92AF92BF92CF9222
